:020000040800F2
:100000000020001039BF0208CD6E020815A20008BA
:10001000C96E0208C56E0208C16E02080000000029
:10002000000000000000000000000000BD6E02089B
:10003000B96E020800000000B56E02081DB7000886
:10004000A1BF0208A1BF0208A1BF0208A1BF020808
:10005000A1BF0208A1BF0208A1BF0208A1BF0208F8
:10006000A1BF0208A1BF0208A1BF0208914E00086B
:10007000814E0008714E0008614E0008514E000884
:100080003D4E0008294E0008A1BF0208A1BF02088A
:10009000DD720208A1BF0208A1BF0208A1BF0208C9
:1000A00061A80008C1A8000851A80008E9A8000834
:1000B000B1A80008A1A8000891A80008A1BF0208E3
:1000C000A1BF0208A1BF0208A1BF0208A1BF020888
:1000D000A1BF020825B80008A9B70008A1BF0208FF
:1000E000A1BF0208A1BF0208A56E0208A1BF0208B5
:1000F00071A80008A1BF020881A80008A1BF0208DA
:10010000000000000000000000000000A1BF020885
:10011000A1BF0208A1BF0208A1BF0208A1BF020837
:10012000154E0008014E0008ED4D0008D94D00089D
:10013000C54D0008A1BF020800000000000000003B
:10014000A1BF0208A1BF0208A1BF02080000000071
:10015000000000000000000000000000000000009F
:100160000000000000000000A1BF0208A1BF0208BB
:10017000A1BF020800000000000000000000000015
:0801800000000000A1BF02080D
:100188002DE9F04FB0F908502DED048B0D81EDB23B
:10019800382D8FB00C4600F02984804634D9802D44
:1001A80000F0DB8079D8522D00F08B8040F2FE837E
:1001B800542D00F04E846E2D40F0F680704B0A6886
:1001C8001B88704DFF2BA8BFFF23511C21601370A3
:1001D800A96881F3100189B2204604F009F96A4B35
:1001E8002046198804F004F9296801F30F0189B23F
:1001F800204604F0FDF801252B46284663810FB000
:10020800BDEC048BBDE8F08F042D00F0168440F29D
:10021800B583202D00F0858040F2D383242D00F093
:100228002584282D40F0C0800B68DFF87881574E70
:10023800591C022221601A70236806275A1C226062
:100248001F7023680A22591C21601A70236801252F
:100258005A1922601D70B8F80010204604F0C8F83A
:10026800B8F80210204604F0C3F823685A1922602F
:100278001F7023685022591921601A7023680022C0
:10028800591921601A703188204604F0B1F8718834
:10029800204604F0ADF82B46AFE7822D19D0C0F008
:1002A800F883A02D00F0E983FE2D7DD1384D05F1AE
:1002B800080635F8021B204604F09AF8AE42F8D139
:1002C80099E70A680021531C012523602B46117009
:1002D80093E70B682F4A2B4D11782F4A581C206042
:1002E8001970D188204604F083F8254B22681B88B2
:1002F800FF2B02F10101A8BFFF2321601370A96839
:1003080081F3100189B2204604F072F8296801F3DC
:100318000F0189B2204604F06BF8204B2268197847
:10032800D1E70B681C4D591C6A7821601A70236844
:100338002A78591C21601A702368AA78591C2160F0
:100348001A70E988204604F053F823682A79591C62
:1003580021601A7022686979B5E70B68104A581C41
:100368000A211288206019702168FF2A01F101030F
:10037800A8BFFF22012523602B460A703DE700BF76
:10038800005E0020045E00203C2E00209424002003
:10039800765E0020425E00207C600020C42B002096
:1003A800A42400202C1D0020A5F10A03E72B00F24D
:1003B800EA80DFE813F03B08E800E800E800E8001E
:1003C800E800E800E800E800E800E800E800E800E5
:1003D800E800E800E800E800E800E800E800E800D5
:1003E800E800E800E8000A08E800E800E800F90783
:1003F800E800E800E800F407E800B307E800E800D0
:10040800E800E800E8009707E8007107E8005E07E1
:10041800E800E800E8000A04C508E800BB08E800AE
:10042800E800B208E800E800E800E800E800FD039A
:10043800E800E800E800E8009608E8007408E8002A
:100448004D084607E800E800E800E800E800E80092
:10045800E8000207E800D706E800A806E8005E06FC
:10046800E8004D06E800E800E800E800EF05BC05F4
:10047800B3058B057905E800E80060055205E8003A
:100488001805FB04E800E800E800E800EF04E800CD
:10049800E800CD04E800E800E800BC04A304660412
:1004A800E800E800E800E8005504E8004A04E8002D
:1004B800E800E800E800E800E800E800E800E800F4
:1004C800E800E800E800E800E800E800E800EF05D8
:1004D800E800E800E800E800E800E800E800E800D4
:1004E800E800E800E800E800E800E800E800E800C4
:1004F800E800E800E800E800E800E800E800E800B4
:10050800E800E800E800E800E800E800E800E800A3
:10051800E800E800E800E800E800E800E800E80093
:10052800E800E800E800E800E800E800E800E80083
:10053800E800E800E800E800E800E800E800E80073
:10054800E800E800E800E800E800E800E800E80063
:10055800E800E800E800E800E800E800E800E80053
:10056800E800E800E800E800E800E800E800E80043
:10057800E800E800E800E800E800E800E800E80033
:10058800E8003D041204742DD8F8003000F0E88229
:10059800772D00F0D582292D00F0F282392D01F057
:1005A800DB85212D01F0B185D8F804600B3DF61AE2
:1005B800EF2D01F2E18301A252F825F0731600082D
:1005C800811D0008811D0008811D0008811D00088B
:1005D800811D0008811D0008811D0008811D00087B
:1005E800811D0008811D0008811D0008811D00086B
:1005F800811D0008811D0008811D0008811D00085B
:10060800811D0008811D0008811D0008811D00084A
:10061800811D0008811D0008811D0008C5150008FE
:10062800811D0008AB150008811D00088915000808
:10063800811D0008811D0008811D0008751500082E
:10064800811D00089B1D0008811D0008811D0008F0
:10065800811D0008811D0008811D00088B1D0008F0
:10066800811D0008131F0008811D00083D1D00089A
:10067800811D0008811D0008811D0008811D0008DA
:10068800FF010008811D0008E31C0008811D000807
:10069800811D0008C71C0008811D0008811D000875
:1006A800811D0008811D0008811D0008811D0008AA
:1006B800811D0008811D0008811D0008811D00089A
:1006C8007B1C0008811D00082D1C0008811D0008E6
:1006D800811D0008F91B0008811D0008811D000804
:1006E800811D0008811D0008811D0008811D00086A
:1006F800811D00089D1A0008811D0008731B000851
:10070800811D0008571A0008811D0008F719000804
:10071800811D0008C9190008811D0008811D0008F5
:10072800811D0008811D0008811D0008811D000829
:10073800811D0008811D0008811D0008811D000819
:10074800811D0008811D0008811D0008811D000809
:10075800811D0008811D0008811D0008811D0008F9
:10076800811D0008811D0008811D0008811D0008E9
:10077800811D0008811D0008811D0008811D0008D9
:10078800811D0008811D0008811D0008811D0008C9
:10079800811D0008811D0008811D0008811D0008B9
:1007A800811D0008811D0008811D0008811D0008A9
:1007B800811D0008811D0008811D0008811D000899
:1007C800811D0008811D0008811D0008811D000889
:1007D800811D0008811D0008811D0008811D000879
:1007E800811D0008811D0008811D0008811D000869
:1007F800811D0008811D0008811D0008811D000859
:10080800811D0008811D0008811D0008811D000848
:10081800811D0008811D0008811D0008811D000838
:10082800811D0008811D0008811D0008811D000828
:10083800811D0008811D0008811D0008811D000818
:10084800811D0008811D0008811D0008811D000808
:10085800811D0008811D0008811D0008811D0008F8
:10086800811D0008811D0008811D0008811D0008E8
:10087800811D0008811D0008811D0008811D0008D8
:10088800811D0008811D0008811D0008811D0008C8
:10089800811D0008811D0008811D0008811D0008B8
:1008A800811D0008811D0008811D0008811D0008A8
:1008B8001D190008811D0008DF180008811D0008A7
:1008C8006B1E0008511E0008F71E0008811D000855
:1008D800C5180008811D00089B1800088918000821
:1008E80029180008811D000801180008811D00084A
:1008F800811D0008DF170008AB17000897170008CC
:1009080069170008811D000847170008811D0008A5
:100918002F170008811D0008811D0008811D00088F
:10092800811D0008811D0008811D0008811D000827
:10093800811D0008811D0008811D0008811D000817
:10094800811D0008811D0008811D00081517000879
:10095800811D0008811D0008AB160008811D0008D4
:10096800811D0008811D0008811D0008811D0008E7
:10097800811D0008811D00085B150008022D00F08C
:10098800D68000F2C280012D7FF40EAD0B680022E4
:10099800591C21601A7023685A1C22601D70226835
:1009A8002421531C23602B46117026E4442D7FF428
:1009B800FBAC002A3FF41FACBA4B136001252B4651
:1009C8001BE4052D7FF4F0AC0B22B749204603F059
:1009D800DFFC0822B549204603F0DAFC012507228E
:1009E800B349204603F0D4FC2B4606E40A68B14B11
:1009F8000125511C216015702268052150192060BD
:100A0800117022680A215019206011702268002193
:100A180050192060117022681978501920601170DF
:100A280022685978501920601170226899785319F2
:100A380023602B461170FFF7E0BB2A469E492046EB
:100A480003F0A6FC0021204603F0D2FC2268002116
:100A580039E40B6800215A1C2260197022680125AC
:100A6800531923602B461170FFF7C7BB934B1968C6
:100A7800204603F0A5FCFFF7BEBB914B084619685A
:100A880003F09EFC8F4B2046196803F099FC8E4BAF
:100A9800EDE78E4A8E4E9368116803EB83034FF699
:100AA800FF725B009342A8BF13469142A8BF11464C
:100AB80023EAE37321EAE1719DB289B20A22002791
:100AC80013E0B368316803EB83034FF6FF725B00F2
:100AD8009342A8BF13469142A8BF114623EAE37385
:100AE80021EAE1719DB289B250222368581C206026
:100AF80020461A7003F07CFC01372946204603F093
:100B080077FC022FDDD1FFF776BB0B680222591C58
:100B180021601A70236801255A1922601D70226805
:100B28000021531923602B461170FFF766BB04227E
:100B380068492046012503F02BFC2B46FFF75DBBD7
:100B4800D8F804209A421EBF5A1CC8F80020197809
:100B5800614A08BF0021204609F0EAFAFFF74BBBBB
:100B6800D8F804209A421EBF5A1CC8F800201978E9
:100B78005A4A08BF0021204609F0DAFAFFF73BBBC2
:100B88005A1CC8F800201B780A2B01F06E83502BE2
:100B980041F0F280404603F0EFFB514E3080404672
:100BA80003F0EAFB4FF0FF3570802B46FFF725BBBB
:100BB800236800255A1C2260294620461D7003F030
:100BC800FFFB2946204603F0FBFB002120460125B8
:100BD80003F0F6FB2B46FFF710BB424B03F1700501
:100BE80022681978501C2060117022685978501CAE
:100BF8002060117022689978501C2060117022685A
:100C0800D978501C2060117022681979501C206016
:100C1800117022685979501C2060117022689979E6
:100C28000733501C9D4220601170D9D1FFF7E3BAF9
:100C38002D4D2046A98903F0DBFB69892046012553
:100C480003F0D6FB2B46FFF7D8BA284B2849B3F94F
:100C5800003081FB0321DB17C3EBA101FFF7C7BA03
:100C6800244D2046A98A03F0C3FBE98A204603F0F5
:100C7800BFFB298B2046012503F0BAFB2B46FFF763
:100C8800BCBA23681C4A19491078174A5D1C2560AC
:100C9800187023689278581C20601A702268897826
:100CA800FFF711BB3D9F0008C40E0308D00E0308D0
:100CB800DC0E0308CF740020BC0E0308442C00206F
:100CC800ACF7FF1FB0F7FF1FB4F7FF1F5824002031
:100CD80098240020B40E0308459E0008159F0008BC
:100CE8009424002020500020344C0020C0300020E4
:100CF80067666666FC310020E06000202268BA4B17
:100D0800BA491878551C2560107022685878551C07
:100D18002560107022689B78501C20601370C98869
:100D28002046012503F064FB2B46FFF766BAAF4D5A
:100D38002046298803F05CFB6988204603F058FBAD
:100D4800A9882046012503F053FB2B46FFF755BA27
:100D5800A74D05F16006A988204603F049FBE988FC
:100D6800204603F045FB2989204603F041FB236810
:100D7800AA7A591C21601A702368EA7A591C2160E2
:100D88001A7055F80C1B204603F01AFBB542E2D145
:100D9800FFF731BA974952232268501C206013701C
:100DA80011F8013F002BF7D1FFF725BA924D002328
:100DB8002268286803EB4301561C405C26601070CB
:100DC8002A6820680A44461C5278266002702A68FD
:100DD80020680A4401339278411C0A2B2160027072
:100DE800E6D1FFF708BA854D23682A68591C12789E
:100DF80021601A702B6822689978531C236000239D
:100E080011702A6821681A4401335279481C032B4F
:100E180020600A70F5D123682A68591C127A21606B
:100E28001A7023682A68591CD27821601A702368BE
:100E38002A68591C127921601A702B682046598932
:100E480003F0D6FA23682A68591C527A21601A706E
:100E58002B6822685978FFF736BA694B204619681B
:100E680003F0AEFA674B20461988012503F0C0FA53
:100E78002B46FFF7C2B9644D2046298803F0B8FA1B
:100E88006988204603F0B4FAB5F904305F49DA17E7
:100E980081FB0313C2EBA30399B22046012503F09B
:100EA800A7FA2B46FFF7A9B9594E3378002B3FF420
:100EB800A2A9584F002537F8021F204603F098FAD8
:100EC800337801359D42F6DBFFF795B9524D534E05
:100ED800DFF87081DFF87091DFED518ADFED519A0C
:100EE8009FED519A05F1200708E02046043503F0EC
:100EF8007FFABD4206F118063FF47DA9717C0029EE
:100F0800F3D095ED008AB0EE480A2BF06DFA98F808
:100F18000030002B41F0458181B2E6E710224349B9
:100F28002046012503F034FA2B46FFF766B9404EF8
:100F3800338AB3F5007F06F1340594BF01270427EF
:100F4800403655F8041B91FBF7F1204689B203F0AF
:100F58004FFAB542F5D1374D374F05F10C06B5ECD0
:100F6800010AD7ED087A80EE270A2BF03DFA81B204
:100F7800204603F03DFAAE42F1D1304D05F10C06A2
:100F880055F8041B204689B203F032FAAE42F7D175
:100F9800FFF731B90DF1140900220592DFF8ACA072
:100FA800274B03920492C9F80420904601214FF67A
:100FB800FF7B07E008F10108B8F10B0F00F0F78795
:100FC8001AF9011F4E1CF5D04BFA08F2D007F1D5DB
:100FD8001A8842FA08F2D207ECD54846019303F082
:100FE8003BFC019BE6E700BF9C1C002064570020E7
:100FF800E457002088E70208B05E0020FC86002045
:10100800BC1C0020B41E00202C5F002067666666AA
:10101800345F0020BA830020502E0020B46D0020D9
:10102800000040420040744400E08244402E00200A
:10103800D85E00201C690020F46000201C5F00209E
:10104800D02300202432002020370020B8E70208EF
:101058002368A74AA749D078A74A5D1C256018705D
:1010680023681278581C20601A702268C978FFF724
:101078002AB90021204603F0BBF90021204603F0DD
:10108800B7F90021204603F0B3F922689B4D0023ED
:10109800511C2160137022682968501C91F82F1088
:1010A8002060117022682968501C91F83A1020605D
:1010B800117022682968501C91F83B10206011704B
:1010C8002268511C216013702268511C2160137022
:1010D8002268511C216013702B682046D98F03F0B9
:1010E80087F92B682046998F03F082F923682A68CC
:1010F800591C92F8312021601A702B68226893F8E5
:101108003210FFF7E0B87E4D23686A797B4E591C90
:1011180021601A7033682046198C03F069F9336826
:101128002046598C03F064F96989204603F060F978
:10113800A989204603F05CF933682046998C03F0AE
:1011480057F933682046D98C03F052F9E9892046CB
:1011580003F04EF9298A2046012503F049F92B4668
:10116800FFF74BB8664EF378002B01F00D8023682B
:101178000822591C21601A702368012299182160DD
:101188001A7023685F4D591C2A7921601A702368E8
:10119800AA78591C21601A702988204603F028F97A
:1011A800698A204603F024F92368F279591C2160E2
:1011B8001A702268E978FFF786B827F03BF8FF280D
:1011C800064601F03A800EA9002501F82E5D0DF1C2
:1011D80009008DF809501AF0A5FE0EA800F82D5D3B
:1011E8001AF094FE0EA800F82C5D1AF083FE0EA8E3
:1011F80020F8245D26F0FEFF23685A1C22601E702A
:1012080023689DF80920591C21601A7023689DF8ED
:101218000A20591C21601A7023689DF80B20591C5C
:1012280021601A7023689DF80C20591C21601A70DF
:10123800BDF814102046012503F0DAF82B46FEF716
:10124800DCBF2268304B0125511C216015702268D3
:101258009978501920601170226819785019206007
:10126800117022685978531923602B461170FEF7C4
:10127800C4BF264D264E05F1280795F90210002314
:10128800F2568A4200F075860C333C2BF8D10835AB
:10129800BD42F2D1FEF7AFBF1E4B03F15A052268DB
:1012A8005979501C2060117022681978501C2060F0
:1012B800117022685978501C206011702268997842
:1012C800501C206011702268D978501C2060117061
:1012D800226819790633501CAB4220601170DED1A8
:1012E800FEF789BF0C4B2268597DFEF7ECBF00BFA3
:1012F800344C0020C0300020D0300020B05E0020E8
:10130800E0600020FC310020F175002058740020B6
:1013180090360020582C0020F0360020AE4D23686F
:101328002A7A591C21601A70A98B204603F060F8AC
:10133800298B204603F05CF8698B204603F058F8A7
:101348002368EA7C591C21601A70E98C204603F056
:101358004FF8298D204603F04BF82368AA7F591CC3
:1013680021601A70236895F82020591C21601A7092
:10137800A98C204603F03CF82368EA7A591C2160BE
:101388001A70E968204603F01BF823682A7C591C68
:1013980021601A70226895F82110FEF794BF8F4BD0
:1013A80022681978FEF78FBF8D4D2046298803F0F3
:1013B8001FF8A988204603F01BF829892046012533
:1013C80003F016F82B46FEF718BF864D864F05F139
:1013D800500600212878854A0B4607E00133242B64
:1013E80002F10C0200F0C28512F80C1C8842F5D1FB
:1013F80003EB4303226807EB8303511C93F8443043
:101408002160137023686A78591C21601A70236858
:10141800AA78591C21601A702368EA780435591C87
:10142800B54221601A70D4D1FEF7E5BE70482AF0A3
:10143800C1F800287EF7DFAE6D4B1D18226813F83F
:10144800011B501C9D4220601170F7D1FEF7D3BEDE
:101458002368684D01269A1922601E7017F0FAFD5C
:10146800002840F0E286644B2268511C216010700D
:10147800226841F2B410511C185C216041F27811C5
:10148800107059582046890A02F09AFFE96B2046E5
:101498004908012502F094FF2B46FEF7AEBE574ED1
:1014A8003378002B3EF4A7AE554F0025B846236885
:1014B80017F81520591C21601A7098F8011001EBD3
:1014C800810101EB810101F2EE2189B2204602F08F
:1014D8008FFF337801359D4208F10208E7DBFEF7FC
:1014E8008ABE2368474D591C2A7821601A702368E0
:1014F8006A78591C21601A706988204602F078FFC2
:1015080023682A79591C21601A70E988204602F05C
:101518006FFF2268297AFEF7D6BE08222E49204698
:10152800012502F035FF2B46FEF767BE2268364BD1
:10153800501C99782060117022685978FEF7C3BE54
:1015480022680121531823600D460B461170FEF7DF
:1015580054BE2E4B1B78DB0700F10E84012508F0E2
:101568008BFE09F0BBFC2B46FEF747BE5A1CC8F899
:1015780000201A4A1B78137001252B46FEF73DBE42
:10158800404602F0F9FE164E3060404602F0F4FE86
:101598007060404602F0F0FE0125B0602B46FEF771
:1015A8002CBE1B4E00233360404602F0CDFE33684C
:1015B8000125034333602B46FEF71FBE5A1CC8F8AB
:1015C80000201878132800F2D7839A1CC8F8002046
:1015D8005D78104A002125E0F036002054300020C4
:1015E800302A00205830002088E70208D0E7020897
:1015F8009C5E00204C7A00203C370020345F00209D
:10160800E44C0020802D0020301D0020358500206E
:10161800442C0020C4E702080131242902F10C02FD
:1016280000F0AA83167AAE42F6D1D14DD14A0C26E3
:1016380006FB0151DD1C91F83C1002F82010C8F897
:10164800005002EB800299785170191DC8F80010FB
:10165800D8789070581DC8F80000C7491B790868E9
:10166800D37014F01DFDFEF7C6BDC44B102E4FF00D
:10167800000228BF10261A605A609A60DA601A744D
:10168800002E3EF4B8ADD8F8002016440132C8F850
:10169800002012F8011C03F8011BB242F6D1FEF734
:1016A800AABD5A1CC8F800201A780F2A00F26483D1
:1016B800991CC8F80010C2EBC202B1495878885486
:1016C800D81CC8F800000A4499785170191DC8F848
:1016D8000010D9789170591DC8F800101979D17087
:1016E800991DC8F8001059791171D91DC8F8001052
:1016F8009979517103F10801C8F80010DB799371E9
:1017080001251DF0F1FF2B46FEF777BD404602F09C
:1017180033FE9C4EB081404602F02EFE01257081BA
:101728002B46FEF76ABD404602F026FE964A00EBBD
:1017380080004300012513802B46FEF75EBD40461E
:1017480002F01AFE914EB082404602F015FEF08279
:10175800404602F011FE012530832B46FEF74DBDB1
:101768001A46591CC8F80010894912F8020B08706B
:10177800C8F8002083495A788A70DA1CC8F8002013
:10178800814A9B78937001252B46FEF736BD7A4B2C
:10179800804918684A2201252CF019FF2B46FEF7CC
:1017A8002CBD19465A1CC8F800207B4A11F8020BB8
:1017B8001070C8F8001059785170D91CC8F800107A
:1017C8009B789370404602F0D7FD744B0125D88072
:1017D8002B46FEF712BD404602F0CEFD6F4E30801C
:1017E800404602F0C9FD7080404602F0C5FD012563
:1017F800B0802B46FEF701BD694F3B78002B3EF4C5
:10180800FAAC684E0025404602F0B6FD1EF014FC06
:101818003B78A6EC010A01359D42F4DBFEF7EBBCF0
:101828000F2E40F0A9825A1CC8F800201D78072DF9
:1018380000F2A2825C4F40460C2602F09DFD06FB9A
:1018480005F6BD19A880404602F096FDE88040469E
:1018580002F092FDD8F8003028811A46591CC8F8C1
:10186800001012F8021BA972C8F800205B78EB720E
:10187800404602F069FD0125B8512B46FEF7BDBC74
:10188800404602F079FD494B012518802B46FEF7AA
:10189800B4BC5A1CC8F800201878060600F12A853E
:1018A800434B1B78DD073EF5A6AC032828BF002074
:1018B800012508F0C5FC2B46FEF79FBC3C4B1B7866
:1018C800D8073EF598AC012508F09EFD09F006FB07
:1018D8002B46FEF792BC284A1068DA1C01462133D1
:1018E800951EC8F8005012F8035C0D70551EC8F814
:1018F800005012F8025C4D70C8F8002012F8015C24
:101908008D7003329A4201F10301E9D11DF080FF85
:10191800FEF771BCC6F34706122E00F22D82B6B14F
:101928000EAB0DF1120903EB46054F46263D404626
:1019380002F022FD27F8020FBD42F8D11D4B39F8FD
:10194800022F23F8022F4F45F9D1112E09D81A4A30
:101958007300023B13440021223223F8021F9A42EB
:10196800FBD1164A01231D461370FEF746BC00BF83
:1019780088E7020858300020B05E00209C5E0020F6
:1019880020500020344C0020C0300020FC310020C2
:10199800E0600020300103089C1C002064570020F0
:1019A800182E002068560020E4570020981C0020BC
:1019B80035850020CA4D0020CC4D0020C84D0020A0
:1019C8001A46591CC8F80010CC4912F8020BC87006
:1019D800C8F80020CA495A780A70DA1CC8F80020EA
:1019E800C84A9B78D37001252B46FEF706BC4046B3
:1019F80002F0C2FC404602F0BFFC404602F0BCFCCC
:101A0800D8F80030C04D9A1C2F68C8F800205A78C2
:101A180087F82F20DA1CC8F800209A7887F83A202F
:101A28001A1DC8F80020DA7887F83B200733C8F871
:101A38000030404602F0A0FCF88740462F6802F0CC
:101A48009BFC112EB88700F2898428685EE75A1C2F
:101A5800C8F80020AC4DAD4F1B78D5F800907B71CD
:101A6800404602F089FCA9F820004046D5F80090CD
:101A780002F082FC052EA9F8220000F29B8408F0EF
:101A880005FC21F039FF286801251DF0D5FF2B46FC
:101A9800FEF7B3BB404602F06FFC054626F0CAFBD2
:101AA800FF283EF4A8ABB5F57A7F80F03F840DF1AE
:101AB8003809002309F8243DEE08494603A88DF8A3
:101AC8000C3001361AF02EFA9DF80C30F6B205F0FB
:101AD8000705B34205F1010503D19DF81430AB4267
:101AE80003D02946304626F091FBD8F80030D8F8C4
:101AF8000420D21A012A7EF77EAB5A1C0EA8C8F819
:101B0800002000221D7800F82C2D1AF0FFF99DF80E
:101B18000C30AB420AD07E4B1B683BB19A79AA4283
:101B280004D31B681B690BB128469847D8F80030C6
:101B38005A1CC8F80020484600221D788DF8142049
:101B48001AF0D8F99DF81430AB423EF454AB704B00
:101B58001B68002B3EF44FAB1B685B69002B3EF4FF
:101B68004AAB28469847FEF746BB1A46591CC8F8A0
:101B78000010664E12F8021BB170C8F800206549C3
:101B88005A780A70DA1CC8F80020634D9A782A71CE
:101B98001A1DC8F80020DB78092BA8BF0923404686
:101BA800AB7002F0E9FBD8F80030D8F804202880A0
:101BB800D11A012907DD404602F0DEFBD8F80030D3
:101BC800D8F8042068829A4240F0178408F05EFB37
:101BD800D8F80030D8F804209A423EF40CAB5A1CCE
:101BE800C8F800201B78EB7001252B46FEF705BBD3
:101BF8004A4A1278012A3EF6FEAA19465A1CC8F823
:101C08000020474A11F8020B9070C8F80010597864
:101C18001170D91CC8F800109B78537001252B4609
:101C2800FEF7EBBA5A1CC8F800201E78112E00F2F5
:101C3800A3809A1CC8F800203A4D5B7805F8163046
:101C4800404602F099FB40F6CA039842A8BF1846DE
:101C580040F2EE23984205EB4601B8BF184601252D
:101C6800A0F2EE222B46192092FBF0F24A70FEF702
:101C7800C4BA1A46591C2C4DC8F8001012F8021B99
:101C88002970C8F800205B786B70404602F074FB3E
:101C9800D8F8003068805A1CC8F800201B782B71CF
:101CA800404602F069FBD8F80030E8805A1CC8F8B2
:101CB80000201B782B7201252B46FEF79EBA1B4A83
:101CC80003F108010133C8F8003013F8010C02F8D9
:101CD800010F9942F6D1FEF78EBA591C1A46C8F878
:101CE8000010134912F8020B8870C8F800205B78BE
:101CF8004B7001252B46FEF780BA00BF344C0020FC
:101D0800D0300020C0300020B05E0020E06000200D
:101D18003437002058560020FC310020F075002090
:101D2800F1750020E44C0020802D0020EF360020C3
:101D3800301D00200722B6FBF2F2C2EBC201711A75
:101D48001AD1D2B2571EFFB2002A3EF454AADFF8C5
:101D5800E49201378A465A1CC8F8002093F900100B
:101D6800B44B002593F902208A4200F08B8201359A
:101D7800052D03F10803F5D14FF0FF352B46FEF78B
:101D88003CBA5A1CC8F80020AB4A1B785375FEF7BA
:101D980032BA5A1CC8F80020A74D1B782B7240464F
:101DA80002F0EAFAA883404602F0E6FA28834046A1
:101DB80002F0E2FAD8F8003068835A1CC8F800200C
:101DC8001B78EB74082E7EF616AA404602F0D4FA69
:101DD800E884404602F0D0FA0C2E28857EF60BAA3D
:101DE800D8F800301A46591CC8F8001012F8021B1F
:101DF800A977C8F800205B7885F82030404602F0C3
:101E0800BBFA102EA8847EF6F6A9D8F800305A1C22
:101E1800C8F800201B78EB72404602F095FAD8F813
:101E28000030E8605A1CC8F800201A782A74162E68
:101E38007EF6E1A99A1CC8F800205B7885F8213065
:101E480001252B46FEF7D9B97C4B1B78D9073EF5FF
:101E5800D2A97B4B4FF4C87201251A802B46FEF796
:101E6800CCB9092E88D9774F1A46591C3D68C8F84D
:101E7800001012F8021B2970C8F800205A78AA70BE
:101E8800DA1CC8F800209A78642A03F10401A8BF74
:101E980064226A71C8F80010DA78642A03F105012F
:101EA800A8BF6422AA71C8F800101A79EA719A1DAD
:101EB800C8F800205A79642A28BF6422D91D2A72DA
:101EC800C8F800109A79EA7003F10802C8F80020EF
:101ED800DB792B71404602F04FFA0A2E688140F0F8
:101EE8001482012529F092F82B46FEF786B9534B48
:101EF8001B78DA073EF57FA9534A1378012543F08A
:101F0800040313702B46FEF778B95A1CC8F8002052
:101F18001A780E2A3FF630AF991CC8F800105D7881
:101F2800032D3FF629AF4948062101FB02F142186B
:101F3800DE1C5571C8F800609D784554191DC8F815
:101F48000010D9785170591DC8F80010197991708E
:101F5800991DC8F800105979D170D91DC8F800101A
:101F68009B79137101252B46FEF747B900231B7A8D
:101F7800FFDE23685A1C226019702988204602F067
:101F880037FA2368EA78591C21601A7023682A797D
:101F9800591C21601A702368AA79591C21601A708B
:101FA80023686A79591C21601A70FFF770B9DFF845
:101FB800A4B04FF000084FF0080A08F10108B8F182
:101FC800240F1BD0C8F120020AFA02F22BFA08F6F5
:101FD800A8F1200316432AFA03F31E4306F0010270
:101FE80000231343E9D05FFA88F014F053F800286F
:101FF800E3D04146484602F02FFCDEE70F4B1B7842
:10200800DF0700F12D810026114FB04602E00136AE
:10201800242E21D03146384602F02EFC0028F6D076
:102028003146484602F028FC002869D108F1010829
:10203800EDE700BF58740020F036002035850020F9
:102048001A870020FC860020942E0020582C00209F
:102058004C1C002090E33FF4C94BCA4EB3F8501013
:10206800204602F0C5F9C84B1988204689B202F00B
:10207800BFF9C64B1A68530103F02001C2F34003AD
:102088000B43C2F3800143EA4103C2F3C00143EAB0
:102098008103C2F3401143EAC10102F01002114367
:1020A800204602F0A5F903A90422204602F070F99F
:1020B80023683178B64A581C206019701188642941
:1020C800A8BF6421204602F093F9962D00F0BD8048
:1020D8000021204602F08CF92168B8F1190348BFA5
:1020E800A8F11203A3F3C4034A1C226020460B7014
:1020F8001A4604A9012502F04BF92B46FEF77DB8D4
:10210800414603A802F0A8FB90E71A46591CC8F8F4
:102118000010A04D12F8021B6970C8F800205A7808
:102128002A70DA1CC8F800209B78AB70404602F091
:1021380023F9D8F80030E880591C1A46C8F800106E
:1021480012F8021B2971C8F800205B786B714FF0F8
:10215800FF352B46FEF751B85A1CC8F800201A78EC
:102168000A2A7FF409AE9A1CC8F800208A4A5978CE
:102178001170D91CC8F8001099785170191DC8F849
:102188000010DB789370F7E52368B178834A581C10
:102198002060197023681278591C21601A70FEF7A4
:1021A800F0BFD9F8003013F48053B4EEE88A62D057
:1021B800F1EE10FAC0F29580B4EEC98AF1EE10FA89
:1021C8000DD8DFED777A9FED777A77EEC87AB4EE9F
:1021D800C78AF1EE10FAB0EE678A00F28280F7EE55
:1021E800007A78EE677AB6EE007AF0EE696AE7EE82
:1021F800876A40F2E932FDEEE67A17EE901AB1F5F9
:10220800FA6FA8BF4FF4FA619142B8BF114689B27C
:10221800002B3EF46AAEB5EE408AF1EE10FA40F2B9
:10222800DC5308BF1946FEF760BE95F824205E4BC4
:10223800002A4DD13046FFF717B9226801255319F6
:1022480023602B461070FDF7D8BF23680322591C62
:1022580021601A7023687278591C21601A703BE754
:10226800059B43F001030593CDE6404602F084F850
:102278004E4EFEF793BCF1EE10FAB0DA4FF47A71D5
:10228800FEF733BE09EBC5064046B17002F074F89C
:10229800D8F8002029F835001346511CC8F800105A
:1022A80013F8021BF170C8F8003053783371D31C4F
:1022B800C8F800309378B371131DC8F800300AF1DC
:1022C800010AD278727157457FF445ADFDF793BF87
:1022D8005978022908D003290CBF04203046FFF79B
:1022E800C3B84FF47A7196E7042A34BF022003205A
:1022F800FFF7BAB800F07F00032828BF00200125A7
:1023080010F0E6FA2B46FDF778BFD8F800303A68A7
:10231800591CC8F80010197851720B2E3FF4E1AD22
:10232800991CC8F800105B785370DAE50DF11409B0
:10233800484625F05FFFBDF81430AB423FF4D5ABFB
:102348001B4B1B68002B3FF4D0AB1B689B69002B11
:102358003FF4CBAB28469847FFF7C7BBD8F8003007
:102368002968581C1A46C8F8000012F8020B81F8B0
:102378003100C8F800205B7881F83230FFF765BB80
:10238800880F0020985E002098720020286900209D
:10239800C82B00207C600020CF74002058560020F5
:1023A80000C0884400C082443C3700202C1D002017
:1023B80034370020404601F0DFFF7881404601F0C5
:1023C800DBFFB8814046D5F8009001F0D5FFA9F8A9
:1023D80024004046D5F8009001F0CEFF0D2EA9F854
:1023E80026007FF64CAB404601F0C6FFF881404618
:1023F80001F0C2FF3882FFF742BB5A1CC8F8002020
:102408001B78003318BF0123F371FFF7DFBB00BF50
:10241800436A826970B4D154436A0469426B0133D8
:10242800A34228BF00234362DAB1116811F0010109
:1024380001D070BC7047856A86699D422E44D6607B
:102448000BD3641B546081621368002143F00103BD
:1024580080F8441070BC136070475D1B5560836240
:10246800F2E7026D136843F080031360E1E700BFF1
:10247800026B10B462B1036CC2684469D11A013BA3
:10248800615C5DF8044B08BF13460364C8B270472B
:10249800016A4369C4685B5C0131A14228BF1146E7
:1024A80001625DF8044BD8B2704700BF436B13B1AB
:1024B80090F844007047836A406A181AB0FA80F0AE
:1024C80040097047416A836A99420AD3CB1A416B23
:1024D800026961B14968501E0B4483420AD2C01A8E
:1024E800704702691144CB1A416B0029F2D1501E82
:1024F800C01A704700207047036B43B1026C5B68D9
:1025080093422FBF981AC0689B1AC0187047C269B7
:10251800036A9A422FBFD01AC0688018C01A704741
:102528000A4B30B503F1100493F900205D78072AAF
:10253800C8BF143A811804330D7313F8025C85542C
:1025480013F8012C0A76A342EED130BD74E90208D3
:1025580003682DE9F041DF691FB13B46BDE8F04152
:102568001847002A164611DD04460D460E4400E0C1
:1025780023689B68204698470028F9D0236815F8F7
:10258800011B1B6820469847AE42F1D1BDE8F08197
:1025980010B45A2158240022032304704170827019
:1025A800C3705DF8044B7047152303701623C3707E
:1025B800172383712D2343702E2303712F23C37197
:1025C800704700BF002870B51EDB0928044620DDCF
:1025D800012303EB83035B00B0FBF3F2092AF8D86D
:1025E8007BB10E4EB4FBF3F00928CCBF5722302242
:1025F800A6FB03E5024403FB1044EB0801F8012B9A
:10260800F0D100230B7070BD2D230B7040420131B7
:10261800DBE7303001F8010BF3E700BFCDCCCCCCC1
:10262800884230B44FF001042ED301FB04F4B0FB10
:10263800F4F58D42F9D284B1AAB901E0B0FBF4F502
:10264800092DCCBF572230222A4404FB150003F879
:10265800012BB4FBF1F4002CF0D100221A7030BC2D
:102668007047B0FBF4F5092DCCBF372230222A443D
:1026780004FB150003F8012BB4FBF1F4002CF0D196
:1026880000221A7030BC70470546002AEBD1D7E704
:1026980003685A1C02601970704700BF2DE9F047A3
:1026A800089C2578002B804689460CBF4FF0200AED
:1026B8004FF0300A661C35B3002A29DD334601E0A5
:1026C800024698B113F8011B501E0029F8D1971E35
:1026D80060B13D46013D51464046C8476B1C002B42
:1026E800F8DC257827EAE770013055B1041B294644
:1026F8004046C847301916F8015B002DF7D1BDE8F0
:10270800F087BDE8F087002A04DC2846BDE8F0879A
:102718000020EBE7571EDCE70A44914251D030B461
:1027280041F2210411F8013B80EA0320430010F430
:10273800004F84EA03059BB2ADB208BF1D466B008B
:1027480015F4004F84EA03009BB280B208BF184614
:10275800430010F4004F84EA03059BB2ADB208BFF2
:102768001D466B0015F4004F84EA03009BB280B24B
:1027780008BF1846430010F4004F84EA03059BB2D3
:10278800ADB208BF1D466B0015F4004F84EA030084
:102798009BB280B208BF1846430010F4004F84EA89
:1027A80003059BB2ADB208BF1D466B0084EA030067
:1027B80015F4004F85B298B218BF28468A42B1D1A5
:1027C80030BC704783684268D0ED037A00EB830120
:1027D8000133934281ED040A836004BF00238360C0
:1027E80000EB830393ED047A036870EE277A9A422C
:1027F800C0ED037A77EEC77AC0ED037A0CDA0133BD
:1028080007EE103AF8EEC76AB7EE007A87EEA60A26
:10281800036030EE070A704707EE102AB8EEC77A51
:1028280087EE870A704700BF90ED097A90ED004A5D
:10283800D0ED0A6AD0ED014AD0ED047A90ED035A42
:10284800D0ED025AA4EE007AB0EE406AB0EE470A24
:10285800B0EE667AA6EE247A67EEC07AA0EE457AE4
:10286800E6EE257A80ED097AC0ED0A7A704700BF56
:10287800D0ED057A90ED013AD0ED003AD0ED064A58
:1028880090ED024A90ED077A90ED035A90ED086AB0
:10289800D0ED045AC0ED067AF0EE406A27EE830ABE
:1028A800C0ED056AA3EEA60A80ED087AA4EE240A14
:1028B800A5EE470AA5EEC60A80ED070A704700BFD5
:1028C800D0ED007A90ED017A30EE670AE7EE007AF3
:1028D800B0EE670AC0ED007A704700BF704700BFCE
:1028E8002DE9F04FDFF8F8C1DFF8F8E1BCF80A701D
:1028F800DEF80060BCF80C30BCF808A03C028BB0D5
:10290800361B4FF00004CDE90034009CBCF80630BB
:102918004FEA17654FF0000767EB0507B946B04661
:10292800A4FB06670024CDE90634009C002304FBC1
:1029380009770024CDE90034AAFB0823CDE9022356
:10294800039AF30D00930AFB09230393009B43EAC0
:1029580047230093029B4FEAD31AFB150193039B6D
:102968004AEA436ADDE9002344464D46CDE9084575
:10297800069C12F5FA62A4FB086743F1000304FB06
:102988000977CDE90623BCF80440039BBCF8022074
:102998004FEAE31B230C059323040493340A44EA07
:1029A80007643D12DDE904674FEAC23816EB0A06F0
:1029B80047EB0B0718EB0408DDE906344FEA5249E8
:1029C80049EB0509B3F5FA6F74F10004B246BB464A
:1029D8003CDADDE90067BC00B20044EA9673B4183B
:1029E80047EB030522463C462B4602FB04F406FB54
:1029F8000344A2FB06232344940844EA83749D10ED
:102A08005B104FEA3202B8EB040869EB0509BAEB30
:102A1800020A6BEB030BDDE90623304C4FF0FF3560
:102A2800A242AB412CDBDDE90856A5FB052305FBDB
:102A380006F403EB4403D40F44EA4304DD17DDE94D
:102A48000623121B63EB0503CDE90623DEF80440D9
:102A5800A4FB082304FB0933540D44EAC3245D1581
:102A6800B4EB0A0A65EB0B0B4FEADA3343EA4B4344
:102A780000B1036009B1069B0B600BB0BDE8F08F95
:102A880040F6AC52B4184FF0000347EB030522465A
:102A9800A2FB022304FB05F403EB4403941843EB65
:102AA8000305A4185D414FEA850CA6004CEA947C06
:102AB800B41A6CEB0305DF00D6006D104FEA34043E
:102AC80047EA5277921B63EB0703B8EB040869EBFC
:102AD80005091AEB020A4BEB030BA4E724FAFFFFE4
:102AE800D8300020541C0020037F33B1012B03D1C0
:102AF8004FF400630382704770474FF4806303828A
:102B0800704700BF90F8493013B1002280F849207F
:102B18001846704770B5044682B01830256D94F891
:102B28005C106B460622A847A8B19DF804009DF8E2
:102B380000609DF801109DF802509DF803209DF853
:102B4800053041EA062143EA002342EA0522A1842E
:102B5800E2842385012002B070BD00BF70B5044631
:102B680082B00830256A6B4606223B21A847A8B1E7
:102B78009DF804009DF800609DF801109DF8025032
:102B88009DF803209DF8053041EA062143EA002319
:102B980042EA05226182A282E382012002B070BD6E
:102BA80030B490E81200057B43690222AA404A60CB
:102BB8002268586A996A4FF6FE752A408842226050
:102BC80004D1012283F8442030BC70479C695A6BB9
:102BD8000C44D4600DD818690024411A51609C62D5
:102BE8001168002041F0010183F8440030BC1160F5
:102BF8007047411A51609862F2E700BF70B40468E8
:102C0800037B2268022101FA03F31A4213D04269B6
:102C18000A49582000FB02124FF6FE765068528986
:102C2800C5680068296831402960C168D24392B2FA
:102C38000A40C260636070BC704700BF2832002041
:102C480030B4094B1C7864B1084B002503EBC4046D
:102C58001A6899885562D06808330143A342D16045
:102C6800F6D130BC704700BF483600204C360020F3
:102C7800F0B5064683B00D460024012714E0032969
:102C88000CBF03220122C3F3011E6946C3F381036B
:102C980030468DF805208DF806E08DF8073026F0CF
:102CA80019FE0134102C0FD02B8807FA04F21342B6
:102CB800F7D0AB78E9780092022903F003028DF887
:102CC8000420DCD10A46DEE703B0F0BDF0B4334C93
:102CD80000EB800004EB80046468002C5BD0304E6D
:102CE80049004FF42040CDB23060A169090444D4B2
:102CF80060682C4F45F08071384041F490310143B1
:102D08004FF420406160306003E0411E002838D055
:102D18000846A1698F07F8D54FF42040A2623060B9
:102D280002E0421E68B31046A2691106F9D562682E
:102D38001C4945F0007545F480350A4015434FF4A9
:102D480020406560306002E0421ED0B11046A269A2
:102D58009207F9D5A362A3694FF420409B0630601F
:102D680005D4431E68B11846A3699B06F9D52023EC
:102D78003060E3610120F0BC7047411E08B108468D
:102D8800B3E7094A138801339BB24FF0FF31316032
:102D98001380F0BC70472046F0BC70476C7200206E
:102DA80094720020009800FC9872002013460020BE
:102DB8000A4668218AE700BF30B50446006D617194
:102DC8000368A26823F00103036087B0A379009227
:102DD80013F004023DD04FF4805213F00203019225
:102DE80044D102934FF480630022039311F001034E
:102DF800059237D1049308238D07694648BF049389
:102E080016F026FC6079236DA17900F00202002AF1
:102E180015BF4FF440324FF480324FF40034002491
:102E280010F0010F586808BF2246CC074CBF024378
:102E380020EA02025A609A6809074CBF42F0080269
:102E480022F008029A601A6842F001021A6007B07C
:102E580030BD13F0020301920BD04FF40055134616
:102E68000295C1E7042304930C23C5E74FF40053EC
:102E7800B7E70293B8E700BF10B50446006DA1603C
:102E8800036823F001030360A37986B013F00402FA
:102E9800009141D04FF4805213F00203019244D1C3
:102EA80002934FF4806362790393D1074FF00003D4
:102EB8000493059345BF0423049308230C23694610
:102EC800920748BF049316F0C3FB6079236DA1797C
:102ED80000F00202002A15BF4FF440324FF480324E
:102EE8004FF40034002410F0010F586808BF224640
:102EF800CC074CBF024320EA02025A609A680907CD
:102F08004CBF42F0080222F008029A601A6842F0A8
:102F180001021A6006B010BD13F00203019207D037
:102F28004FF4005113460291BDE74FF40053B7E741
:102F38000293B8E7002326220360027027228270DA
:102F4800012243600271837170472DE9F3410569DD
:102F580006460F467DBBD0F80080C8F30A0323B3AA
:102F68000023D6F80080019318F050FC042819D1EA
:102F7800214C236943F001032361BBB2A8F8003058
:102F880018F044FC04282ED108F102030193019B98
:102F98003F0C1F8018F03AFC2369042823F0010332
:102FA800236125D06FF0010505E018F02FFC0428F7
:102FB80005D04FF0FF35284602B0BDE8F0810E4C31
:102FC800236943F002032361C4F81480236943F0A2
:102FD8004003236118F01AFC2369042823F0020334
:102FE8002361BDD0E5E7236923F001032361D9E715
:102FF800336804333360DEE700200240F8B5044646
:103008000D468E180027B54201D12069F8BDE36846
:10301800591CE160234415F8012B1A720429F2D1D6
:10302800A1682046FFF791FFE7602061EBE700BF4A
:1030380000B583B001AB03220021772021F036FDD3
:103048009DF805309DF804209DF806001B0243EA10
:103058000243184303B05DF804FB00BF08B5FFF74F
:10306800E7FF014B586008BD541C002008B5FFF766
:10307800DFFF014B186008BD541C0020682021F0B8
:1030880015BD00BFF0B583B004466B460622A821E3
:10309800192021F00BFD00B39DF801709DF8001078
:1030A8009DF803609DF802209DF805509DF80430B6
:1030B80041EA072142EA062243EA052309B212B28D
:1030C8001BB201EBD17102EBD27203EBD37349103F
:1030D80052105B106182A282E38203B0F0BD00BF90
:1030E80070B5044600F11805636D80226B212846EF
:1030F8009847642008F070FA636D284603226B2114
:103108009847636D94F848201921284698470F205E
:1031180008F062FA636D94F8462028461A21984709
:10312800636D284618221B219847636D284618228C
:103138001C2198472846636D02223721BDE870405C
:10314800184700BF03682DE9F041DF691FB13B460E
:10315800BDE8F0411847002A164611DD04460D4621
:103168000E4400E023689B68204698470028F9D061
:10317800236815F8011B1B6820469847AE42F1D119
:10318800BDE8F08103689B69184700BF0368DB68E6
:10319800184700BF03685B68184700BF03681B68CF
:1031A800184700BF014B1868F8E700BF6C8500207E
:1031B800054B53F8203033B11A689B88918A0B422B
:1031C80018BF1B0493617047D072002010B5040922
:1031D800013C052C17D80D4B33F8142000F00F00D4
:1031E80042FA00F313F001030DD0012303FA00F0B3
:1031F8000138104028F088FE054A064B125D10443D
:1032080003EBC00010BD002010BD00BF700503080F
:103218007C050308A46F00202DE9F04F4A484B4B6A
:103228004B4C4FF090414FF0010A4FF002094FF01C
:1032380004084FF0080C4FF0100E20274026802578
:1032480030F8022B12F0010F03D01960A3F804A084
:10325800083312F0020F03D01960A3F80490083362
:1032680012F0040F03D01960A3F80480083312F099
:10327800080F03D01960A3F804C0083312F0100F28
:1032880003D01960A3F804E0083312F0200F02D02D
:1032980019609F80083312F0400F02D019609E8099
:1032A800083312F0800F02D019609D80083312F4A1
:1032B800807F05D04FF4807B1960A3F804B00833F1
:1032C80012F4007F05D04FF4007B1960A3F804B016
:1032D800083312F4806F05D04FF4806B1960A3F89F
:1032E80004B0083312F4006F05D04FF4006B196076
:1032F800A3F804B0083312F4805F05D04FF4805B64
:103308001960A3F804B0083312F4005F05D04FF435
:10331800005B1960A3F804B0083312F4804F05D09D
:103328004FF4804B1960A3F804B00833D20B04D0D3
:103338004FF4004219609A80083301F58061A14278
:103348007FF47EAFBDE8F08F70050308A46F0020FE
:1033580000180048002867D003682DE9F04F03F1F2
:1033680038445C4EA40A0125345D04F01F06640944
:10337800022C05FA06F558D0032C00F0A580012C84
:1033880058D08088B0FA80F4C4F11F04A4B2E508CC
:1033980003EB850504F007042E6AA4000F27A74055
:1033A80026EA07062E622E6A01F00307A2407C1E59
:1033B8003243012CC1F3810CC1F300182A62C1F316
:1033C80041113CD9C60700F18980850700F1958035
:1033D800440700F1A380020700F1B180C60600F19E
:1033E800BF80850600F1CD80440600F1DB8002062F
:1033F80000F1E980C60500F1F780850500F1058137
:10340800440500F11381020500F12181C60400F191
:103418002F81850400F13D81440400F14B810204B1
:1034280000F15981BDE8F08F70472B4CA6693543F0
:10343800A561A6E7284C666935436561A1E70024C4
:1034480022464FF0010E4FF0030904E00132102A22
:1034580004F10204E6D00EFA02F636EA0005F5D1C8
:10346800D3F808A009FA04F5ED430AEA050AC3F8F7
:1034780008A0D3F808B00CFA04FA4AEA0B0AC3F811
:1034880008A0B3F804A01FFA8AFA2AEA06069E8062
:10349800B3F804A008FA02F646EA0A06B6B29E8015
:1034A8001E682E401E60D3F800A007FA04F646EA0C
:1034B8000A061E60D3F80CA001FA04F605EA0A0A07
:1034C80046EA0A05DD60C1E7034CE6693543E56174
:1034D80057E700BF84050308001002401A6822F06D
:1034E80003021A601A683A431A60DA6822F0030283
:1034F8000A438507DA607FF56BAF1A6822F00C0281
:103508001A601A6842EA87021A60DA6822F00C0226
:1035180042EA81024407DA607FF55DAF1A6822F05B
:1035280030021A601A6842EA07121A60DA6822F052
:10353800300242EA0112DA6002077FF54FAF1A68DB
:1035480022F0C0021A601A6842EA87121A60DA6822
:1035580022F0C00242EA8112C606DA607FF541AF66
:103568001A6822F440721A601A6842EA07221A603E
:10357800DA6822F4407242EA01228506DA607FF5B1
:1035880033AF1A6822F440621A601A6842EA872246
:103598001A60DA6822F4406242EA81224406DA605C
:1035A8007FF525AF1A6822F440521A601A6842EA79
:1035B80007321A60DA6822F4405242EA0132DA60CD
:1035C80002067FF517AF1A6822F440421A601A689B
:1035D80042EA87321A60DA6822F4404242EA8132CB
:1035E800C605DA607FF509AF1A6822F440321A601E
:1035F8001A6842EA07421A60DA6822F4403242EA5C
:1036080001428505DA607FF5FBAE1A6822F4402294
:103618001A601A6842EA87421A60DA6822F440227D
:1036280042EA81424405DA607FF5EDAE1A6822F479
:1036380040121A601A6842EA07521A60DA6822F4DD
:10364800401242EA0152DA6002057FF5DFAE1A68DD
:1036580022F440021A601A6842EA87521A60DA684D
:1036680022F4400242EA8152C604DA607FF5D1AE04
:103678001A6822F040721A601A6842EA07621A60F1
:10368800DA6822F0407242EA01628504DA607FF566
:10369800C3AE1A6822F040621A601A6842EA87626A
:1036A8001A60DA6822F0406242EA81624404DA6011
:1036B8007FF5B5AE1A6822F040521A601A6842EADD
:1036C80007721A60DA6822F0405242EA0172DA6040
:1036D80002047FF5A7AE1A6822F040421A601A6801
:1036E80042EA87771F60DA6822F0404242EA817135
:1036F800D960BDE8F08F00BF002852D0036803F1FD
:1037080038422DE9F04F920A504DAA5C02F01F058D
:1037180052090124022A04FA05F443D0032A00F0CE
:103728009080012A43D001F003077A1E012AC1F3D1
:10373800810CC1F300188088C1F341113CD9C60738
:1037480000F18880850700F19480440700F1A28089
:10375800020700F1B080C60600F1BE80850600F1C0
:10376800CC80440600F1DA80020600F1E880C60544
:1037780000F1F680850500F10481440500F112810D
:10378800020500F12081C60400F12E81850400F1B4
:103798003C81440400F14A81020400F15881BDE8EB
:1037A800F08F70472A4A95692C439461BBE7284AF1
:1037B80055692C435461B6E7002422464FF0010EA8
:1037C8004FF0030904E00132102A04F10204E6D0A4
:1037D8000EFA02F636EA0005F5D1D3F808A009FA80
:1037E80004F5ED430AEA050AC3F808A0D3F808B0BF
:1037F8000CFA04FA4AEA0B0AC3F808A0B3F804A0C2
:103808001FFA8AFA2AEA06069E80B3F804A008FA84
:1038180002F646EA0A06B6B29E801E682E401E6070
:10382800D3F800A007FA04F646EA0A061E60D3F8A1
:103838000CA001FA04F605EA0A0A46EA0A05DD6060
:10384800C1E7034AD5692C43D4616CE784050308B2
:10385800001002401A6822F003021A601A683A43FC
:103868001A60DA6822F003020A438507DA607FF5F6
:103878006CAF1A6822F00C021A601A6842EA8702D2
:103888001A60DA6822F00C0242EA81024407DA6020
:103898007FF55EAF1A6822F030021A601A6842EAB1
:1038A80007121A60DA6822F0300242EA0112DA607E
:1038B80002077FF550AF1A6822F0C0021A601A6832
:1038C80042EA87121A60DA6822F0C00242EA8112DC
:1038D800C606DA607FF542AF1A6822F440721A60B1
:1038E8001A6842EA07221A60DA6822F4407242EA49
:1038F80001228506DA607FF534AF1A6822F4406247
:103908001A601A6842EA87221A60DA6822F440626A
:1039180042EA81224406DA607FF526AF1A6822F46B
:1039280040521A601A6842EA07321A60DA6822F4CA
:10393800405242EA0132DA6002067FF518AF1A688F
:1039480022F440421A601A6842EA87321A60DA683A
:1039580022F4404242EA8132C605DA607FF50AAFB6
:103968001A6822F440321A601A6842EA07421A605A
:10397800DA6822F4403242EA01428505DA607FF5CE
:10398800FCAE1A6822F440221A601A6842EA87429A
:103998001A60DA6822F4402242EA81424405DA6079
:1039A8007FF5EEAE1A6822F440121A601A6842EAED
:1039B80007521A60DA6822F4401242EA0152DA60C9
:1039C80002057FF5E0AE1A6822F440021A601A6810
:1039D80042EA87521A60DA6822F4400242EA8152C7
:1039E800C604DA607FF5D2AE1A6822F040721A6017
:1039F8001A6842EA07621A60DA6822F0407242EAFC
:103A080001628504DA607FF5C4AE1A6822F040626C
:103A18001A601A6842EA87621A60DA6822F040621D
:103A280042EA81624404DA607FF5B6AE1A6822F091
:103A380040521A601A6842EA07721A60DA6822F07D
:103A4800405242EA0172DA6002047FF5A8AE1A68B1
:103A580022F040421A601A6842EA87771F60DA68E3
:103A680022F0404242EA8171D960BDE8F08F00BF80
:103A780010B1036882881A85704700BF10B10368C7
:103A880082889A61704700BFF0B5174F83B0064629
:103A9800B868FFF7EDFFE82021F044F96C460DF116
:103AA8000605002021F03EF904F8010BAC42F8D1DC
:103AB800B868FFF7E3FF9DF804009DF800509DF8F3
:103AC80001109DF802409DF803209DF8053041EA59
:103AD800052143EA002342EA04220120B184F2844A
:103AE800338503B0F0BD00BF541C002038B1002955
:103AF8008388026814BF002110218B4093617047AE
:103B080010B40A4B0A4A1C7801238340234052F818
:103B1800200029B9B3FA83F149095DF8044BE5E7B8
:103B2800191C18BF01215DF8044BDFE7CC72002097
:103B3800D07200202DE9F041044618460D4616467D
:103B4800984627F037FD2768E6722844A072294670
:103B58007D69434632462046AC46BDE8F0416047A1
:103B6800036810B504461B689847236820469B687D
:103B78009847A37B0133A37310BD08B5FFF726FB55
:103B880038B12C2282710022C2712021BDE8084080
:103B9800B2E508BD038823F040031B041B0C038017
:103BA800038841F4807191FAA1F20029B2FA82F2F5
:103BB8009BB208BF4FF0FF32013A23F0380343EAC3
:103BC800C2039BB2038003889BB243F04003038087
:103BD800704700BF70B5204D204C002228460D21AB
:103BE8001C26EA71AE71A560FFF786FD2846FFF72F
:103BF80045FF04211A48FFF7CDFF2846FFF738FF95
:103C0800242021F08FF8802021F08CF8A068FFF79D
:103C180035FF642007F086FCA068FFF729FF202005
:103C280021F080F8AF2021F07DF8A068FFF726FF8B
:103C3800012007F077FCA068FFF71AFF232021F086
:103C480071F8602021F06EF8A068FFF717FF642074
:103C5800BDE8704007F0C0BC7C710020541C0020F7
:103C680000300140F8B505015A4C5B4B62596119A7
:103C78009A4204EB050704BF01230B730646387A02
:103C880020F084FD3B7A03F01F015B090122022B1F
:103C980002FA01F278D0032B71D0012B67D0631997
:103CA80001361879FFF792FAF6B2074610B11223D7
:103CB800C671837163195879FFF788FA10B1132315
:103CC800C671837163199879FFF780FA10B11423CC
:103CD800C671837166190E21F2793846FFF73AFBEF
:103CE8007079FFF773FAF2790E21FFF733FBB07999
:103CF800FFF76CFAF2790E21FFF72CFB6359374A6C
:103D0800934251D0344A934259D0354A934240D0D5
:103D18002C44227B002A2FD1012002249A8822F4E5
:103D280080521204120C9A80998889B241F4805109
:103D380099801A8802F4415242F4457202432243A0
:103D48001A809A8822F470621204120C42F4E0621B
:103D58009A809A8B22F400621204120C07219A832B
:103D680019821A8892B242F040021A80F8BD1D4B9F
:103D7800996A0A439A6292E700200446CEE7194BF3
:103D880019690A431A618AE7164BD9680A43DA6047
:103D980085E702F5EA32116941F4004111611169C0
:103DA80021F400411161B3E702F56042D16841F4A2
:103DB8008051D160D16821F48051D160A8E702F523
:103DC800EC32116941F480411161116921F480419B
:103DD80011619DE79C7200200038004000300140CE
:103DE800003C004000100240427A02B9704710B50A
:103DF80004460368406804F10A0198470023637287
:103E080010BD00BF437A5A1C0344D2B24272997261
:103E1800037A934200D802B9704710B50446036884
:103E2800406804F10A0198470023637210BD00BF7F
:103E380030B40B4D002305F1100101E0272B0BD006
:103E480011F8132082424FEA430403F10103F5D12C
:103E58002C44607C30BC7047002030BC704700BFE9
:103E680074E9020870B5448806460D46C4F30B048D
:103E78002246002128462AF0CFFB3369094A93429B
:103E880009D3094A934206D2224628461946BDE874
:103E980070402AF09CBB23B121462846BDE87040FB
:103EA800184770BD6043030806440308064B0749DA
:103EB8008B4202D30023184670471A88C2F30B02BC
:103EC8009042F8D01433F3E7503F030860430308E7
:103ED800024A136823EA000010607047442C00204F
:103EE800F8B51A4D2B789F2B2ED16B78BE2B2BD182
:103EF80005221749A81C2AF0DAFB28BB0722294605
:103F08004FF6FF70FEF708FC124FEC1D22884AB1ED
:103F1800A618BE4218D2052A16D92146FEF7FCFB80
:103F28003446F3E721460222FEF7F6FB0222A118E7
:103F3800FEF7F2FB0634084B641B1C8041F60F5356
:103F4800C31A58425841F8BD0020F8BD00F00308D4
:103F58007D10030800000408C62B00202DE9F04F4F
:103F6800DFF854914F4F8DB00326A7EB09071822AD
:103F78000DEB020000212AF04FFB4B4BCDF81890B7
:103F880007971A69120604D5484A5A6002F188321E
:103F98005A6001228DF82C203422DA60444B454CBB
:103FA80018689A8804909B79ADF8142004A9072210
:103FB80006A88DF81630FFF721F8072204A94FF656
:103FC800FF70FEF7A9FBDFF8F4B080464FF0000A57
:103FD8005C4536D30CAC002524F82C5D0222214622
:103FE80006A8FFF70BF8022221464046FEF794FB8D
:103FF80040BAC043ADF80800022202A906A8FEF79D
:10400800FDFF099860B108ABC0F1040229461844C5
:104018002AF002FB089906A8FEF797FF09950A906F
:104028009DF82C300A9A23B11F490B6943F080038D
:104038000B61013E2DD0002A99D1FFF751FF50B3F3
:104048002CE065888DF80DA0C5F30B05AA1DADF809
:1040580008202288C2F30B01120BADF80A108DF864
:104068000C2002A9062206A8FEF7C8FF062202A90C
:104078004046FEF751FB616880462A4606A8FEF7CF
:10408800BDFF616840462A46FEF746FB1434804669
:104098009EE7002AD1D0052006F0F4FD0DB0BDE85A
:1040A800F08F00BF0000040800200240230167458C
:1040B800D2E90208503F030800F0030860430308F0
:1040C8000378202B024600F10100F9D0092BF7D024
:1040D8002D2B2CD02B2B03BF5378B7EE000A0246AA
:1040E800B7EE000AA3F13001C8B209289FED467A5D
:1040F80010D8F2EE046A07EE901AF8EEE77A12F892
:10410800013FE7EE267AA3F13001C8B20928B0EEE4
:10411800677AF0D92E2B4CD003F0DF03452B0BD058
:10412800F7EE007A67EE276A20EE260A7047537882
:10413800BFEE000A0246D5E710B451782D2959D0B0
:104148002B290ABF9178501C901C0024A1F1300340
:10415800092B53D8002303EB830301EB430310F827
:10416800011FA1F13002092AA3F13003F3D9B3F5F5
:104178009A7F28BF4FF49A73072B42D9DFED236A41
:104188001A46F7EE007A083A072A67EEA67AFAD8AE
:1041980003F007032BB1F2EE046A013B67EEA67A3F
:1041A800FBD124B3C7EE276A5DF8044B20EE260A3C
:1041B80070475378A3F13001C8B2092802F101020F
:1041C800AAD8F2EE046AF0EE665A07EE901AF8EEF4
:1041D800E77A12F8013F87EEA66AA3F13001C8B268
:1041E800092866EEA56A37EE067AEED994E767EEF7
:1041F800276AD9E7901C91780124A7E7F7EE007A9F
:10420800CFE7F7EE007AC5E70000000020BCBE4CFF
:10421800B5EEC00ADFED317AF1EE10FACCBF30EE20
:10422800270A30EE670ADFED2E7A20EE270A30B52E
:10423800FDEEC07A87B017EE904A054684EAE4702E
:10424800002303A9A0EBE47001930093029317F0F5
:10425800FFFC002CACBF20232D2303A88DF80030D1
:1042680027F0A8F9012803A924D002282DD0032873
:1042780005BF3023684668468DF801302AF0F2F908
:10428800684627F097F90338C4B22246694628469B
:104298002AF046FA00232B55284627F08BF92E22C0
:1042A800431C2A540DEB0401E8182AF0F8F92846B3
:1042B80007B030BD302368468DF801308DF80230E4
:1042C8008DF803302AF0CEF9DAE7302368468DF806
:1042D80001308DF802302AF0C5F9D1E76F12033AA0
:1042E80000007A442DE9F041064615460846B6FB1B
:1042F800F2F43CB905FB1464124B1B5D00F8013B5A
:10430800BDE8F081B4FBF2F767B90E4B05FB174720
:1043180005FB1464DA5D00F8012B1B5D00F8013B16
:10432800BDE8F081B7FBF2F8B8F1000F02D04046C3
:10433800FFF7D8FF05FB1878024B13F8082000F8A0
:10434800012BE3E78410030830B402681146531CBC
:10435800036011F8024B0160D31C51780360937815
:10436800151D05601B0443EA0123D078234343EA63
:10437800006030BC704700BF0368591C1A460160D2
:1043880012F8021B0260587841EA0020704700BF0B
:1043980038B50446006815462AF019F922682A44F7
:1043A800226038BD036810B40A0A5C1C04601A70E5
:1043B80003685A1C026019705DF8044B704700BF0F
:1043C80003685A1C026010B4197003680A0A5C1C5E
:1043D80004601A7003680A0C5C1C04601A70036895
:1043E800090E5A1C026019705DF8044B704700BF33
:1043F80003685A1C026019700368090A5A1C026093
:10440800197070472DE9F047002488B080460F46A0
:104418001E46A14605AD531C0393117839B32529CF
:1044280033D1931CCDF810900393507830284ED098
:104438004FF0000AA0F13003DBB2092B42D96C28F7
:1044480019D0642800F0938024D825281CD063D97B
:10445800582876D063281BD131784046B847039A4C
:10446800531C03931178043601340029D7D1204610
:1044780008B0BDE8F087039B5A1C03921B78642B95
:104488007CD02AD8252B54D1252140460134B84761
:10449800039AC0E7732833D044D975284FD106F161
:1044A800040E30682B4600220A217646FEF7B8F83B
:1044B800049A0095534639464046FEF7EFF8039AAA
:1044C8000444A8E704AA03A917F09EFBB7E7D31C86
:1044D800039390784FF0010AACE7732B10D05BD9A7
:1044E800752B3AD0782B96D1A3F15802B2FA82F202
:1044F800306852092B4610210436FEF791F8D7E7A9
:104508003368049A0093394600234046FEF7C6F8FC
:1045180004360444039A7EE70028B9D1204608B03F
:10452800BDE8F0876E28B3D1039A336804361C605F
:1045380071E72AD9582BD7D0632B8DD06BE7782811
:10454800A6D1A0F15802B2FA82F2306852092B467D
:104558001021FEF765F80436AAE706F1040E306864
:104568002B4600220A217646FEF75AF8A0E7331DAB
:10457800306829461E46FEF725F899E7331D30684E
:1045880029461E46FEF71EF892E7002B7FF443AF3C
:10459800204608B0BDE8F0876E2BC6D03BE700BFC9
:1045A8000EB400B584B005AB019053F8042B06494E
:1045B800039301A8FFF726FF019B00221A7004B09D
:1045C8005DF804EB03B07047992600080FB430B5C6
:1045D80083B006AB0B490C4853F8042B09680068F4
:1045E8000193FFF70FFF094C0546206803685B69D4
:1045F80098470028F9D0284603B0BDE8304004B0F9
:10460800704700BFFC290020002A00206C8500208C
:10461800DFED2B7AB4EEE70AF1EE10FA4ADDDFEDB2
:10462800296A9FED297A01E0B0EE670AB4EEC70A5D
:10463800F1EE10FA70EE667AF6DC9FED247AF4EE6D
:10464800C77AF1EE10FA38D5DFED1E6A9FED207AB1
:1046580001E0F0EE407AF4EEC77AF1EE10FA37EEA8
:10466800A60AF6D4DFED1B7AB4EEE70AF1EE10FAEB
:1046780014DDDFED137A37EEC00A60EE006A9FEDB5
:10468800166A9FED167ADFED167AA6EE867A20EE88
:10469800266AE6EE877AA6EE270A7047DFED117ADA
:1046A800B4EEE70AF1EE10FA44BFDFED087A37EE10
:1046B800C00AE2E7F0EE407ABFE7B0EE670AD1E75A
:1046C800DB0F4940DB0FC940E4CB1641DB0F49C083
:1046D800E4CB16C1DB0FC93F92E741B99730083CDC
:1046E80015A82ABEDB0FC9BF41404A0011F0800F50
:1046F80082F0D503D2B2DBB208BF1346590013F0DB
:10470800800F81F0D502C9B2D2B208BF0A46510063
:1047180012F0800F81F0D503C9B2DBB208BF0B4697
:10472800590013F0800F81F0D502C9B2D2B208BF88
:104738000A46510012F0800F81F0D503C9B2DBB2EE
:1047480008BF0B46590013F0800F81F0D502C9B29B
:10475800D2B208BF0A46510012F0800F81F0D5038B
:10476800C9B2DBB208BF0B465A0082F0D50013F07D
:10477800800FD2B2C0B208BF1046704780EAE0731B
:10478800A3EBE0738B4205DB002801DD401A70477C
:1047980002D17047002070470844704709B909E002
:1047A800194690FBF1F301FB13030846002BF7D1E0
:1047B800084670470146FBE710B507EE901A2DED45
:1047C800028BB8EE678ADFED227A28EE008A04466B
:1047D80028EE278AB0EE480A27F052FEF0EE408A0B
:1047E800B0EE480A27F0AEFDF7EE007A9FED197A91
:1047F800F0EE675AE8EE875A0023A361B0EE676AC5
:10480800C7EEA56A63612362E361A3626362A8EEEF
:10481800C76ABDEC028B77EEC07AB6EE007AF8EE86
:10482800005A27EE877A20EE250A27EE267A26EE0A
:10483800266A67EEA67A20EE260A84ED046AC4ED9D
:10484800017A84ED007A84ED027A84ED030A10BDC2
:1048580027D4D236F304353F10B44C09012250F85E
:10486800243001F01F0102FA01F10B4340F8243013
:104878005DF8044B704700BF4B0901F01F0150F869
:104888002320012303FA01F1114214BF1846002026
:10489800704700BFB0F1FF3F0AD0022810B403DC14
:1048A8005DF8044BFEF712BA00205DF8044B704720
:1048B80000207047F0B585B005460DF107030122C9
:1048C80002210C2020F0F2F818B19DF80730DB0720
:1048D80003D40024204605B0F0BD02AB0622032114
:1048E8000C2020F0E3F80DF10703012209210C2028
:1048F80020F0DCF804460028EBD09DF8070010F003
:104908000C00E6D19DF809E09DF808109DF80B70A1
:104918009DF80A209DF80D609DF80C3041EA0E21A3
:1049280042EA072243EA0623C1EB8131C2EB823215
:10493800C3EB8333890092009B0029806A80AB8097
:104948000A2201230C21FFF7A5FFC3E700B50023C6
:1049580083B018460A220C21FFF79CFF142006F0AA
:104968003BFE0F230A220C210020FFF793FF0A20A9
:1049780006F032FE01AB032210210C2020F096F83D
:104988000A2006F029FE002318460A220C21FFF708
:1049980081FF0A2006F020FE0DF103030122022107
:1049A8000C2020F083F80DF10303012209210C20CB
:1049B80020F07CF801230A220C210020FFF76AFF6F
:1049C800012003B05DF804FB012348227721002071
:1049D80060E700BF01235822772100205AE700BF73
:1049E80010B580232422192104460020FFF752FF26
:1049F800642006F0F1FD9723202219210020FFF7FB
:104A080049FF0A2006F0E8FD10232322192100207F
:104A1800FFF740FF642006F0DFFD4FF48053238248
:104A280010BD00BFF0B5574B574A97B0196891426F
:104A380000AF00F09C805549554A00234FF47000A0
:104A4800C1F888003B607B60136843F480331360CF
:104A580003E03B68B3F5A04F09D0136803F40033B3
:104A68007B603B6801333B607B68002BF1D0484B8F
:104A78001B6813F4003318BF01237B607B68012B8C
:104A88004BD0424D424B434AEA60434A596A11604F
:104A98005A6A424E42F080725A625A6907F15804C3
:104AA80042F4FC0241F6FF715A6124F8501D0323B9
:104AB80021464FF09040BB72FEF7DAF84FF6FF73CD
:104AC800214637483B81FEF7D3F821463548FEF7A3
:104AD800CFF821463448FEF7CBF821463348FEF795
:104AE800C7F821463248FEF7C3F8204624F0FEFCFA
:104AF800BB683049304AA1FB031330499B0CF024B2
:104B080000204FF0070E5C370B60566085F8234095
:104B18009060C2F800E0BD46F0BD294A1C4B122146
:104B280011605A685A605A685A605A6842F480623A
:104B38005A605A6822F47C125A605A6842F4E812A1
:104B48005A601A6842F080721A601A689201FCD59D
:104B580059680F4A21F003015960596841F0020170
:104B68005960536803F00C03082BFAD189E7002237
:104B78001A6062B6134B1B6883F30888124B1B68D4
:104B88009847FEE7FC9F0020EFBEADDE00ED00E099
:104B9800001002400005FA051C3700203F190100EB
:104BA8000004004800080048000C004800100048B5
:104BB8000014004883DE1B4310E000E00873002067
:104BC8000020024000D8FF1F04D8FF1F064A002318
:104BD8005168814202F11C0204D001330C2BF7D139
:104BE80000207047D8B2704750000020074BC0EB38
:104BF800C00030B403EB8000054C056963692B43A2
:104C080063610176427630BC704700BF50000020D7
:104C1800001002402DE9F04F634C54F8204083B057
:104C2800002C7CD0656D1F466B682365A1604FF42E
:104C3800807304F15A019046064604F5AD725B484C
:104C480020606161A261E3602361287E1FF09EFD00
:104C5800E86858B1FFF7BAFF721CD2B20C21FFF70F
:104C6800C5FF236DEA6822632433E364A86870B340
:104C7800FFF7ACFF721CD2B20B218146FFF7B6FFDB
:104C88004B48DFF830E1EB7EDEF81410C9EBC909B8
:104C980000EB89009B0902690A43CEF81420DFF86B
:104CA80018E1417B446100228DF80530C0F808E026
:104CB800012301A88DF806208DF807308DF804101F
:104CC8001FF0E4FF236DAA6862632833A36494F895
:104CD8005900FEF77BFA814694F85800FEF776FAF9
:104CE8003A07824695F819B01DD5B9F1000F1AD0C8
:104CF80017F0110F4FF00B0306F1010614BF4E21F8
:104D08003E2189F8063089F807605A464846FEF77A
:104D180021FBFB0743D5236B6BB3636B5BB3204667
:104D280003B0BDE8F08F17F0010F0CBF2E274E27F8
:104D380018F0020F0DD0B9F1000F0AD00B22731C26
:104D480089F8062089F8073048465A463946FEF75A
:104D580001FB18F0010FDED0BAF1000FDBD00136ED
:104D68000C238AF807605A4639468AF806305046B6
:104D7800FEF7F0FACFE7AB7E8DF804302B7F0021E9
:104D88009B09012201A88DF805308DF806108DF8D1
:104D980007201FF07BFF204603B0BDE8F08F484690
:104DA800FEF766FEB7E700BF082A0020DCE9020824
:104DB8005000002000100240A92B00080348D0F83A
:104DC8003C3113B100F59A70184770475000002025
:104DD8000348D0F8203113B100F58C70184770479C
:104DE800500000200348D0F804310BB1FC301847BC
:104DF800704700BF500000200348D0F8E8300BB1DE
:104E0800E0301847704700BF500000200348D0F832
:104E1800CC300BB1C4301847704700BF5000002099
:104E28000348D0F8B0300BB1A8301847704700BF1E
:104E3800500000200348D0F894300BB18C3018474C
:104E4800704700BF500000200248836F0BB17030DC
:104E580018477047500000200248C36D0BB154300A
:104E680018477047500000200248036C0BB13830D7
:104E780018477047500000200248436A0BB11C30A5
:104E880018477047500000200248836803B118474C
:104E9800704700BF500000201749184B184A19489E
:104EA80010B4D1F8884044F47004C1F888401C68F4
:104EB80044F001041C605C6822405A601A6822F0C1
:104EC800847222F480321A601A6822F480221A60EE
:104ED8005A6822F4FE025A60DA6A22F00F02DA6295
:104EE8001A6B002410404FF0006218639C608A60BF
:104EF8005DF8044B704700BF00ED00E00010024071
:104F08000CC07FF8CCFC00FF2DE9F04F2DED028B93
:104F1800C54B1B7891B0072B099001F07B820023C9
:104F28000793C24BD3F800A01AF4806F40F0548660
:104F3800BF4B1B6806931C0700F1F885BD4BBE4D9F
:104F4800B3F80090BD4CBE4BBE491F68B1F906804E
:104F58007A89904580F29084BB4B4FF07E521A605C
:104F6800DFF8F8B294F90820B1F900C0BBF818606E
:104F7800207994F805E0002AACEB060314BF01225F
:104F88004FF0FF32002B40F3E284B3F5FA7FC0F212
:104F9800E4844FF4FA731B1A07EE903AF8EEE77AB6
:104FA800B445C5ED007A03DAF1EE677AC5ED007A0B
:104FB800B1F902C0ACEB0603002B40F3D584B3F57E
:104FC800FA7FC0F2D7844FF4FA731B1A07EE903AAF
:104FD800F8EEE77AB445C5ED017A03DAF1EE677ABF
:104FE800C5ED017AB1F90430991B0029D8BFF11A2F
:104FF800B1F5FA7F80F23A847145D8BF4FF0000EC0
:1050080000F3368402FB0EF207EE902AF8EEE77AF8
:10501800B342C5ED027ABCBFF1EE677AC5ED027AFC
:105028001AF48053059300F0E980B8F5FA6F424608
:10503800A8BF4FF4FA62B2F57A7FB8BF4FF47A721C
:10504800A2F57A728149DFF818E281FB0230D317A2
:10505800C3EB6013581C6FF0630C3EF910003EF967
:1050680013E00CFB0323A0EB0E0003FB00F381FB12
:105078000321DB17C3EB61139E440FFA8EFE07EE84
:1050880090EA059BB8EEE78A85ED038A002B40F08D
:10509800B08519F04003089340F0B984069B13F0DB
:1050A800140F03D019F4027F40F02A86684B1B784E
:1050B80023B1BBF81A30434580F29A8494F83260E1
:1050C8001EB119F0030F40F0598794F838209BF867
:1050D8001F30002A40F0BA859BF81E60002E00F0B1
:1050E800C380022E00F04487032E00F0268759491A
:1050F80049880233DBB2002A00F02C87002900F02F
:10510800298755480668B1FBF6F10EB2A4F8686025
:10511800ABB307EE906AF8EEE77AF7EE006A86EE30
:10512800A77A012BD5ED007AD4ED1F6A77EEE67ADF
:1051380067EE877AC4ED1B7A21D0D5ED017AD4EDDC
:10514800206A77EEE67A022B67EE877AC4ED1C7A3E
:1051580015D0D5ED027AD4ED216A77EEE67A032BE5
:1051680067EE877AC4ED1D7A09D0D5ED037AD4EDC0
:10517800226A77EEE67A67EE877AC4ED1E7A2A49C4
:105188000978092901F07084002E72DD93B394ED3B
:105198001F7AD4ED1B7A77EE877A012BC4ED1F7A3C
:1051A800C5ED007A21D094ED207AD4ED1C7A77EE03
:1051B800877A022BC4ED207AC5ED017A15D094EDDB
:1051C800217AD4ED1D7A77EE877A032BC4ED217A04
:1051D800C5ED027A09D0D4ED227A94ED1E7A77EEE5
:1051E800877AC4ED227AC5ED037A013B022BB8BF5A
:1051F8000223DBB2002A18BF02233BE0BBF81A10D7
:105208008845C0F2F383B8F5FA6FD4BFC1EB080341
:10521800C1F5FA634FF47A7202FB03F2C1F5FA6141
:10522800B2FBF1F20EE700BF563000202037002015
:1052380028690020D0230020445E0020981C00200C
:10524800FC860020BC830020B02300201F85EB5182
:1052580044000020345F00203C300020F03600205D
:10526800008700200AD7233CA4F86860002A00F0D1
:105278006F8102233A785FED056AB97807EE902AC4
:10528800F8EEE77AB0EE007A67EEA67AD34AF4EE43
:10529800C77AF1EE10FA107840F34484DFEDD06A53
:1052A80037EEC77AB0EE676AA7EE266AF0EE466A6E
:1052B80095ED007A9FEDCB6ADFF84CE3DFF84CC33D
:1052C80027EE066AF0EEC65ACEED005A8CED006A5B
:1052D80099B107EE101AB8EEC75A9FEDC37A66EE79
:1052E800064A25EE075AB7EE007A37EE457A64EE9D
:1052F800A54AA5EE247A26EE076A9FEDBC7A7A794C
:1053080026EE877A27EE067AAAB1DFEDB76A9FED17
:10531800B86A65EEA65A06EE902AF8EEE66A66EED8
:10532800A56AF4EEC66AF1EE10FA40F3D9859FED4E
:10533800B16A27EE067A0C289FEDAF8ADFEDAF6AD7
:10534800DFF8CC8200F0A785B4EEC87AF1EE10FA47
:1053580098BFB0EE478AB4EEE68AF1EE10FAB8BF0D
:10536800B0EE668A88ED008A002B00F0E680B0EE89
:10537800007AF4EEC77AF1EE10FA05DD37EEC77A57
:10538800DFED976AE7EE267A95ED017ADFED956A0B
:1053980027EE267AF0EEC75A8CED017ACEED015A47
:1053A80099B106EE901A9FED906AF8EEE66A27EE3C
:1053B800075A66EE866AB7EE006A36EE666A25EE2A
:1053C800255AA6EE856A27EE067ADFED886ABA794D
:1053D80067EEA67A67EE877AFAB107EE102AB8EE7A
:1053E800C77A9FED816ADFED826A27EE257A27EE7C
:1053F800067AB4EEE67AF1EE10FA00F36D85B5EEB2
:10540800C07AF1EE10FA01F15D80B7EE006A36EE6F
:10541800477AC6EE076A67EEA67A0C2800F01C8564
:10542800DFED756A9FED757AF4EEE67AF1EE10FA23
:1054380088BFF0EE667AF4EEC77AF1EE10FAB8BFDC
:10544800F0EE477A012BC8ED017A76DD7B78DFED47
:10545800666A07EE903AF8EEE77AB0EE007A67EE01
:10546800A67A7B7AF4EEC77AF1EE10FA05DD37EE0C
:10547800C77ADFED5B6AE7EE267A95ED027ADFED13
:10548800596A27EE267AF0EEC75A8CED027ACEEDED
:10549800025A9BB106EE903A9FED536AF8EEE66A1F
:1054A80027EE075A66EE866AB7EE006A36EE666A37
:1054B80025EE255AA6EE856A27EE067ADFED4B6AB9
:1054C800FB7967EEA67A67EE877AFBB107EE103AAA
:1054D800B8EEC77A9FED446ADFED456A27EE257A74
:1054E80027EE067AB4EEE67AF1EE10FA00F3F084CD
:1054F800B5EEC07AF1EE10FA00F1E087B7EE006A77
:1055080036EE477AC6EE076A67EEA67A0C2800F0F0
:105518009B84DFED396A9FED397AF4EEE67AF1EE95
:1055280010FA88BFF0EE667AF4EEC77AF1EE10FA58
:10553800B8BFF0EE477AC8ED027A092800F07B84FC
:105548009BF82150002D40F03184002384F8383036
:105558002B4D2C4F95F82420DFF8B880DFF8B8A041
:10556800531E082B00F20581DFE813F01E019A0193
:10557800A600030158000900AF0103019C0198F837
:105588000030002B40F0B4842B68287A03EB00200D
:1055980020F092FB2B7A0133DBB2022B2B7240F006
:1055A800548100201FF090FB00201FF08DFBFF208E
:1055B8001FF08AFB00F01F00052801F0498313F053
:1055C8000DFBEE68002E00F0988300222B696968B5
:1055D8000120B04795F82420C2E700BF56300020CC
:1055E800D7A368416F12033B0AD7233C0000484306
:1055F800A4707D3F0000C84200C0F94400C0F9C44F
:105608004C7A002004730020E0230020D4230020DB
:10561800B8230020DE2D0020580002404FF400710E
:10562800286813F08FFA012800F0DD84C0F0D485D3
:10563800022840F00A8113F003FB13F0CFFAEE685A
:10564800002E00F05A83002210462B696968B04783
:1056580095F8242084E71021D24813F073FA002823
:1056680040F0F180059001217F2023F003FC012800
:105678008146059B40F0E7801846022123F0FAFB9B
:10568800002801F09A81012840F0DD8016213A2097
:1056980023F0F0FB431C9B02EB6313F0D1FA306854
:1056A800FEF7E6F900210A2013F06AFA002840F014
:1056B800CF86032385F8243010210CA813F042FA72
:1056C800002840F0C2809DF83A209DF839009DF8E6
:1056D8003C109DF83D309DF83B60120442EA0062A0
:1056E8000A431B019DF83E109DF83100DBB243EAE6
:1056F800111342EA062203F5FA636A632B879DF8C1
:1057080032209DF8383042EA002201F00F011809D2
:1057180003F00F0385F83A106A859DF830109DF85C
:10572800332085F832309DF8343085F8281085F814
:105738002C209DF835109DF8362085F82D309DF8E1
:10574800373085F8303085F8310085F82E1085F827
:105758002F2013F075FAAB7E002B00F01281022186
:105768009148FEF717FA002304222B6285F82420BB
:105778000323DBB2022B6ED9042A00F0C280082A68
:1057880000F0BF80894B1B7823B9894EB278002A74
:1057980040F03685874B1B78072B00F07B8411B0CF
:1057A800BDEC028BBDE8F08F834E3068FEF760F9E0
:1057B8000021084613F0E4F9814613F041FAB9F1E3
:1057C800010F42D1002330686B76FEF751F940F2A1
:1057D800AB11082013F0D4F9052800F01084012833
:1057E80000F01D8613F02CFA6B7E002B01F0F3817C
:1057F800022385F824303068FEF73AF96B7E022BD5
:1058080014BF4FF000094FF080490021372013F0F2
:10581800B7F94946292013F0B3F9814613F010FA75
:10582800B9F1000F11D16B7E022B00F0038685F8C9
:105838001A903068FEF71CF90021092013F0A0F92E
:1058480000283FF408AF13F0FBF995F82420531E05
:10585800DBB2022B90D8594B69691B685B1AC82BBD
:105868008DD913F0BBF995F8242085E74FF4FA7128
:10587800A1EB0E0EFFF7C6BBB8F5FA6FC0F2AA800F
:105888003B7AC3F1640307EE903A9FED4D7A4D4B96
:10589800F8EEE77A67EE877AC3ED007AFFF760BB28
:1058A800454EA8E70826FF201FF00EFAFF2800F053
:1058B800FC83013EF7D16B693A68FA339342C4D24C
:1058C80013F08CF995F824204AE6FF201FF0FCF924
:1058D800FF284FF0080606D0013EECD0FF201FF04D
:1058E800F3F9FF28F8D12B6A0022012B2A7641F21E
:1058F8005784EA69013B01322B620823EA6185F883
:105908002430314D13F054FD6B78022B00F0D9830D
:10591800032B7FF437AF41F2B813EB5C002B41F057
:10592800698041F2A403EB5C002B41F06D8041F2E9
:10593800E803EB5C002B41F0628041F22C13EB5C36
:10594800002B3FF41FAF214821F030FC1AE7A6EBEB
:105958000C03B3F5FA7FBFF61CAB9842FFF61BABFE
:10596800DFED1B7AFFF71CBBA6EB0C03B3F5FA7F40
:10597800BFF629AB9842FFF628ABDFED157AFFF7A3
:1059880029BB0D4E3068FEF773F84FF400711020F4
:1059980013F0F6F8064613F053F9002E3FF4DFAE85
:1059A8008EE700BF8C7A002000380040755E00202A
:1059B800F175002056300020E02D002004730020EF
:1059C8000AD7233CB02300203C3700206848002039
:1059D80000000000387AA8EB020303FB00F3C2F5CD
:1059E800FA6293FBF2F3C3F164034CE71A4615E439
:1059F800D14B1B78012B00F04283192B00F03F8319
:105A08000E2B3FF45BAB082B3FF458AB3CE3CB4B7E
:105A1800CB49B3F904306289DFEDCA6A9FEDCA7ACF
:105A280081FB0301DB17C3EBA1039B1A1BB207EE33
:105A3800903AF8EEE77A67EEA67A77EE876ABDEED7
:105A4800E66A16EE103A2033402B40F24E83DFED23
:105A5800BF6ABDEEE77A17EE103A2033402B00F20A
:105A680041839FEDBB7AF4EEC77AF1EE10FA40F36A
:105A7800DF87DFEDB85A9FEDB86A01E0F0EE477AAC
:105A8800F4EEC67AF1EE10FA37EEE57AF6DCDFEDE1
:105A9800B37AB4EEE77AF1EE10FA40F1CD87DFED94
:105AA800AD5A9FEDAF6A01E0B0EE677AB4EEC67A00
:105AB800F1EE10FA77EE257AF6D49FEDA37AF4EE9C
:105AC800C77AF1EE10FA00F395829FEDA67AF4EE0C
:105AD800C77AF1EE10FA44BF9FEDA07A77EE677AA5
:105AE80067EEA75A9FEDA05A9FEDA06A9FEDA07A96
:105AF800A5EE856A27EEA55AA5EE867AE5EE077A21
:105B080095ED016AD5ED005A27EEC67A65EEA77ABB
:105B1800A5EEA67AE6EE267A85ED007AC5ED017A3D
:105B2800FFF7BCBAF0EE676AFFF7C2BB914D924B24
:105B3800D5ED027AB3F80090804B814AB3F904306E
:105B48008E4CB2EE0E7AF0EEE76AF4EEC76AF1EE2A
:105B580010FA82FB03124FEAE37338D519F0040FE9
:105B680035D02188C3EBA2035B1A9BB21AB212F19B
:105B7800B30FBCBF03F5B4731AB2B32AC8BFA2F5FA
:105B8800B4737F49C8BF1AB2237A0978002B4FF63D
:105B9800FF7318BF012308077FF5D5A9794909685C
:105BA80012FB03F30A7E78499BB212FB03F381FBD5
:105BB80003121A44DB17C3EB221307EE103AB8EEB0
:105BC800C77A77EEC77AC5ED027AFFF7BCB9C3EB9F
:105BD800A2032380FFF7B7B96C488368002B3FF412
:105BE800A7A900F144019847694BD3F800A0FFF733
:105BF8009FB91D216748FEF73FFE00283FF449AAD8
:105C0800654BDB78002B7FF444AADFED647A6449A6
:105C180038EE678AC6F5FA63FDEEC87A1BB2CDED99
:105C2800087ABDF92020120381FB0201D217C2EBCA
:105C3800A11203FB02F343F30F33334407EE903A08
:105C4800F8EEE77AC5ED037AFFF723BA55485149CC
:105C5800D0F8EC00096844F62066B042A8BF304688
:105C6800B0F57A7FB8BF4FF47A7080B2C906608702
:105C780040F1C9810599002900F028844149D1F8EB
:105C880000C0BCF836E04FEA5E0E454EE16BD5ED3C
:105C9800037AA6FB00608609642090FBF6F01428BE
:105CA800BDEEE77A04EB4108A8BF14200131814218
:105CB800E16317EE109AA4BF0021E16304EB4101F0
:105CC800A8F84090B1F9401007EE101AB8EEC77A5C
:105CD80077EEC77AFDEEE77ACDED057ABDF91400C7
:105CE80080EAE071A1EBE071714500F392862E49DC
:105CF8004FF07E500860FFF7EFB995F824202FE4A5
:105D08001F4B1B7813F0100300F08D81227B236951
:105D180095ED017A002A0CBF01224FF0FF3203FBF8
:105D280002F307EE903AF8EEE77A77EE877AC5ED58
:105D3800017AFFF7BBB900BF543000202C5F002068
:105D48006766666635FA8E3CDB0FC93F00000000C7
:105D5800DB0F4940DB0FC940E4CB1641DB0F49C0DC
:105D6800E4CB16C1DB0FC9BF92E741B99730083CB5
:105D780015A82ABE445E0020D0230020981C0020CD
:105D8800942E0020B05E002089888888F460002066
:105D9800203700208C2E00205460002000007A4418
:105DA800D34D6210880F0020080000201E21D4481F
:105DB800FEF762FD00283FF4C8AB089B002B7FF478
:105DC800C4AB94F88C30AB4240F07086CD4BD4ED28
:105DD800247AD3ED006A98ED025ADFEDCB5A9FED95
:105DE800CB6A27EEC57A68EE277AA8EE267AE5EE22
:105DF800267AB4EEE57AF1EE10FA88BFB0EE657A4D
:105E0800B4EEC67AF1EE10FAF4EEE57AB8BFB0EE69
:105E1800467AF1EE10FA88BFF0EE657AF4EEC67AAB
:105E2800F1EE10FAB8BFF0EE467A88ED007AC8EDC8
:105E3800027AFFF78ABBFDEEC87AB54A17EE903AA8
:105E48009680D380FFF77CBBBDEEE77AB04B17EEA8
:105E5800102A9A80FFF75DBB9FEDAB7ADFEDAB6A46
:105E6800AB49F4EEC77AF1EE10FA98BFB0EE677A54
:105E7800FDEEE77AB4EEE67AF1EE10FA17EE902A24
:105E8800B8BFB0EE667A012B88ED017A4A803FF7F9
:105E9800DDAAFFF755BBB4EEC87AF1EE10FA98BF49
:105EA800B0EE478ABDEEC77AB4EEE68ADFF86092B4
:105EB800F1EE10FA17EE102AB8BFB0EE668A88ED38
:105EC800008AA9F80020002B7FF451AAFFF738BBFD
:105ED800DFED906AFFF718BBDFED8E6AFFF79BBA1C
:105EE800F7EE005A75EEE66A85EEA66AFFF721BA64
:105EF800894B19688E037FF542AC4FF400325A6023
:105F0800DAF80020854B4FF6FE710A40CAF80020E7
:105F18001A89D2077DD41FF081FE0028FBD17F4A61
:105F2800938823F002031B041B0C938098F800301D
:105F3800002B7FF436ABFFF727BB9BF82010C1EB93
:105F4800411001EB8001C900023389B2DBB2002A9B
:105F58007FF4D4A8B4F86860013E36B2002EA4F8E5
:105F680068603FF713A9002A7FF483A9FFF7F0BA06
:105F7800618F01F57A7189B2FFF7BBB8684BDFED25
:105F8800697A93ED080AB4EEE70AF1EE10FA40F2E6
:105F98007C8226F0BFFAD4ED0D7A20EE270A26F08F
:105FA80023FAB0F5617F00F3988207EE900AF8EEC5
:105FB800E76ADFED5D7A66EEA76A07EE906AB8EEEB
:105FC800E77AFDEEE67A17EE903A2033402B40F25E
:105FD80055869FED560A26F007FA00B207EE900A9A
:105FE800B8EEE77A53E26B693A6864339342FFF498
:105FF80022AB2AE49FED567A77EE677A70E585F84A
:106008001990FFF7EFBB1AF0805F7FF433AEFFF70C
:1060180063B89A891A89D007FBD41FF0FFFD0028BE
:106028007FF479AF7BE7E179002940F06F82B4F91A
:106038001430A079A8EB030282EAE276A6EBE276B6
:10604800864240F3068502EBD27201215210A26209
:1060580084F82C10217722691344B3F5FA6FA8BF8E
:106068004FF4FA63B3F57A7FB8BF4FF47A7307EE4B
:10607800903AF8EEE77AC5ED037AFFF717B82C4B9C
:106088009B7B002B7FF41AA82A4A0023AB609360FD
:10609800FFF714B805F0FAF9079A1D4B801A988093
:1060A80011B0BDEC028BBDE8F08F12F0C9FD0423DE
:1060B80085F82430204D13F07BF96B78022B7FF4A0
:1060C80027ACAB784FF001082746072B00F2228453
:1060D800DFE813F0C6034E04E0035103ED03900319
:1060E8009A035D03DFED117A0AE5F4EEC77AF1EE63
:1060F80010FA40F36885DFED135A9FED106A31E01E
:106108008C2E00200000002000C0F94400C0F9C413
:10611800765E00200000C8420000024000380040BF
:10612800D82B00208FC2753CD06D393A0000000092
:10613800D46E0020B82300203C370020E4CB164161
:10614800DB0F49C0DB0FC940E4CB16C1DB0FC93FE9
:10615800DB0F494092E741B99730083C15A82ABEA1
:10616800F0EE476AF4EEC66AF1EE10FA36EEE57A1A
:10617800F6DC5FED0D6AB4EEE67AF1EE10FA40F166
:106188001E855FED105A1FED106A01E0B0EE667AC9
:10619800B4EEC67AF1EE10FA77EE256AF6D41FED62
:1061A800157AF4EEC76AF1EE10FA40F362811FED3A
:1061B800187A77EE666A66EEA65A1FED1A5A1FED30
:1061C8001A6A1FED1A7AA5EE856A26EEA55AA5EE7B
:1061D800867AE5EE076A3CE412F032FDEE680423A5
:1061E800002085F824302876002E3FF48AAB2B69EE
:1061F8002A686968B04795F82420531EFFF728BB22
:10620800D14F3B78013B0A2B59D8DFE813F09202B3
:10621800840278025E02580058004A02E201BF0177
:10622800A1020B00022A38D1C84BDFF85CA31B7807
:10623800002B40F0BC87DAF8005045B32B7833B315
:1062480095F82820002A40F02A812B7EAA6385F839
:106258003C20042285F8282013F008036A6AEA62C1
:106268002A6303D0BA4A41F29413D3586B634FF0B0
:106278000008C5F82480C5F80880C5F80C802846B1
:1062880022F0AEFD0523C5F8408085F828300022AD
:106298000423CAF800208AF81430AE4BAE4A5B6873
:1062A8001268C833934204D318F020FB002800F08A
:1062B8003082B278032A01F01B8001233B70022A46
:1062C80000F0ED80F378002B3FF464AAA34B1B6821
:1062D800D90440F15B85A24B9B8807EE903AF8EE13
:1062E800E77AA04991ED012AD1ED022A91ED033A0E
:1062F800D1ED043A91ED054AD1ED064A91ED075AE0
:10630800D1ED085A91ED096AD1ED0A6A91ED0B7A3F
:10631800B4EE672AF1EE10FAF4EE672A14BF0123EF
:106328000023F1EE10FAB4EE673A18BF43F0010308
:10633800F1EE10FAF4EE673A18BF43F00103F1EEFC
:1063480010FAB4EE674A18BF43F00103F1EE10FAF1
:10635800F4EE674A18BF43F00103F1EE10FAB4EE09
:10636800675A18BF43F00103F1EE10FAF4EE675ACA
:1063780018BF43F00103F1EE10FAB4EE676A18BFD4
:1063880043F00103F1EE10FAF4EE676A18BF43F028
:106398000103F1EE10FAB4EE677A18BF43F0010377
:1063A800F1EE10FA18BF43F00103002B40F0ED8323
:1063B80091ED007AB4EE677AF1EE10FA40F0E583D9
:1063C800654DD4F89C102B68994200F2E5833B7820
:1063D800012B3FF4DFA994F89B20002A3FF4DAA9A7
:1063E8000B2B0DD801229A4040F6030112EA010650
:1063F8000BD112F4C06F03D0093B012B40F2FD878B
:10640800544B2A685A600B233B70002384F89B3056
:10641800FFF7C0B905F03AF80790FEF782BD0CA85F
:106428001FF086FC9DF83330AB2B04BF02236B763C
:10643800FFF7D8B93068FDF71BFB49463A2012F040
:106448009FFB81460CA81FF073FCB9F1000F07D021
:1064580012F0F6FB12F0C2FB95F82420FFF780B883
:1064680012F0EEFB0C9B1BBAC3F38073AB76FFF7FD
:10647800E0B99FED3D7AF4EEC76AF1EE10FA44BF39
:106488009FED3A7A77EE666A95E69FED397AD5ED13
:10649800037A77EE877AC5ED037AFEF716BE2C4AA3
:1064A80041F2B513D35C002B00F0C68794F89B30FB
:1064B80001223A70002B3FF46DA9A6E7F7EE006AB7
:1064C800FFF722B8F7EE006AFEF7A5BF2949D1F811
:1064D80000C0BCF936E0FFF7D8BB07EE906ADFEDE5
:1064E800266AB8EEE77A66EEA65A9FED245A9FED23
:1064F800246ADFED247AA5EE856A26EEA55AE5EE34
:10650800867AE5EE276A26EE870A64E5B4F9141060
:10651800A279A8EB010686EAE670A0EBE670904245
:1065280040F38E828845C8BF524207EE902A95ED07
:10653800037AA361F8EEE77A012077EE277A2077CD
:10654800C5ED037AFEF7B2BDF07500201C300020BF
:106558003C37002030300020047300202037002012
:106568006457002068560020DB0FC9BFDB0F49C005
:1065780000000000B05E002084F9223F92E741B994
:106588009730083C15A82ABE204D00201A200FF08D
:1065980081FDD0B1A24B1B88BBB9A24B45201D6819
:1065A80018F0E4F90E2018F0E1F9284613F018FA6B
:1065B800099D284613F014FA9B4A4FF480510A2388
:1065C800284611803B7013F0ADFA13F099FDB278AC
:1065D80075E618F04DF9954B93ED000A25F004FF88
:1065E800934B93ED000A804625F0FEFE814640203D
:1065F80018F020F9002840F08C808E4D8E4A2B68C8
:1066080092F801E0492B00F28285DFE813F02307B6
:106618001807DF06D906D206CB06C406BD06B4069F
:10662800A8064B0A410A3A0A2C0A250A1E0A170A22
:106638000C0A010AF609EB09E009D509CA09BF09DC
:10664800AE09D408C408B408A408940884087408D7
:1066580064085C084C0844083C0834082C082408E2
:106668001B08120809080108F907F007E707DF0700
:10667800D70773076B0765075F07580751074A076E
:106688004207A60993098C0985097E097709220919
:106698001B0914090D090609FF08F808F108EB0899
:1066A800E40818F0E5F8654B002105208DE80300A3
:1066B800A3F108020291532013F042FD48BB5D4B41
:1066C800B278186008233B70F9E518F0D1F85C4AF5
:1066D8000292A2F10C03292101930091A2F10A036D
:1066E8005021163A492013F02BFD90B9514BB2783E
:1066F80018604FF0FF31596007233B70DFE54D4DBF
:1067080018F0B6F84F4A6B68126864339342C0F0C9
:106718000C85B278D3E5022A00F09B83494B4549A2
:106728001B684B60484800230B60032103603970E5
:10673800C5E5464B1B78D9077FF5C1AD802015F01C
:1067480051FC08B10DF0A4F813F0E4FDB278B6E5F9
:106758003F4B1B78002B00F03A821A200FF09AFC6E
:10676800002840F0348294F89B30002B40F02F82B0
:1067780009233B7029E741F270133C46EB5C002B80
:106788003FF400A8334820F011FDFEF7FBBF0323B8
:106798003C466B70FEF7F6BF2B690622652BAA7084
:1067A80032D92A78032A14BF6FF0FF026FF07F02F4
:1067B800A3F1650303EA020303F1010314BF4FF4D5
:1067C800807280229A422B611ED23268EC680232B3
:1067D8001E19964280F087851F4A6C60D16FAE60A3
:1067E800490203FB01F30521146042F81C3C42F8FE
:1067F800183CA970AA681949012020F043F901281A
:1068080040F066850623AB70002112481FF0AEFCED
:10681800012840F05D85AB780133DBB2AB7054E4FE
:10682800962E0020982E0020802E0020A42E0020D6
:106838005857002030300020985E002058EC02089D
:106848007AEA020804730020BC4D00203585002038
:10685800A8300020AC480020D04800204037002055
:1068680000230DF1300841461846092212F0F6F9C6
:1068780001283C467EF486AF0C9A92F8FE31552BDF
:1068880000F0428241F2B41202210123A9546B7034
:10689800FEF778BFD24B00930320A870302305225F
:1068A800D049D1483C4620F05BF8FEF76BBF2A7808
:1068B8002B7DCE4EDFF88CA3032A14BF4FF48079CA
:1068C8004FF08009002B3ED0012BFBD1C84BD5F8E7
:1068D80004C01B6832684FEA432E00244FF0FF3390
:1068E800B3FBFEFE1EEB0C0044F100010024A142A4
:1068F80002F1020208BF904238BF0CEB0E02BD49FC
:10690800022012F0EBFA032800F2B681DFE800F06B
:10691800020502053C46FEF735BF6C68AB6829697D
:106928001A1B8A4284BFEC602A6103283FF434AF03
:106938000133B3FBF9F209FB12320AB14B449B1A3B
:1069480000226B602A75326851460232002012F02C
:10695800C5FA032800F2908101A353F820F000BF84
:106968001D690008B76900081D690008A1670008CB
:106978003C460DF1300841F2FC164146A859002367
:10698800092212F06BF901287EF4FCAE00230C9A60
:106998002B70B2F80B30B3F5007F00F0338441F26E
:1069A800B41203210123A9546B70FEF7EBBE6B6888
:1069B80085F814800133AB6088E704212C2022F08D
:1069C80059FA032106904E2022F054FA0C21059022
:1069D800362022F04FFA059A069B911C421C8A40E9
:1069E80009FA03F3A2FB0301420A42EAC152EA632D
:1069F800FEF753BE804820F0D9FBFEF792BF7F48D0
:106A080020F0D4FBFEF799BF7D4820F0CFFBFEF7BE
:106A18008EBFBCF838109FED7B7A07EE901AF8EE1F
:106A2800E77A794967EE877AC1ED007AFEF754BBB9
:106A3800B0EE677AFFF72BB8F0EE477AFFF73DB86C
:106A4800227F12B1626A2377226223690B44FFF71F
:106A580004BB227F002A3FF4FEAA626A84F82C1045
:106A680021772262FFF7F7BA95ED000A059306929F
:106A780025F0BAFC6549DFF8D0E1D1F8EC10DFF871
:106A8800CCC1069AACF800008EFB013EC917C1EBD9
:106A9800AE1107EE901AF8EEE77A059BFDEEE77A5D
:106AA80017EE901AACF80210FEF76EBB07EE905A7C
:106AB800DFED576A9FED577A84F88C50F8EEE77A45
:106AC80067EEA67A77EE876ABDEEE66A16EE103AAA
:106AD8002033402B40F26A81DFED4F6A4F4BBDEE09
:106AE800E77AC3ED006A17EE103A2033402B00F224
:106AF8005A819FED4B7AF4EEC77AF1EE10FA40F323
:106B08002A84DFED485A9FED486A01E0F0EE477AA3
:106B1800F4EEC67AF1EE10FA37EEE57AF6DCDFED40
:106B2800437AB4EEE77AF1EE10FA40F11084DFED23
:106B38003D5A9FED3F6A01E0B0EE677AB4EEC67A3F
:106B4800F1EE10FA77EE257AF6D49FED327AF4EE6C
:106B5800C77AF1EE10FA40F370819FED317A77EE43
:106B6800677A67EEA75A9FED335A9FED336A9FED18
:106B7800337AA5EE856A27EEA55AA5EE867AE5EE64
:106B8800077AC4ED247AFFF726B92D4B1B6803F565
:106B98009C530833C4F89C303B78012B7EF4FAAD43
:106BA80094F89B30002B7EF4F5AD032A00F0158491
:106BB80013F0B0FB012384F89B30FEF7EBBDF0EE39
:106BC800476AFFF7ECBAB0EE667AFFF7D2BA0998CF
:106BD80012F0A8FFF9E485F82430FEF7D3BD00BF12
:106BE800C15E0208AC100308AC48002044490020EC
:106BF8004C49002044370020F44800202448002055
:106C0800E04700206F12833A08000020880F002018
:106C180035FA8E3CDB0FC93F000000000000002061
:106C2800DB0F4940DB0FC940E4CB1641DB0F49C0FD
:106C3800E4CB16C192E741B99730083C15A82ABEA3
:106C48000473002040370020D34D6210765E002088
:106C58008B4BEE681B686B61072385F82430002E88
:106C68003EF490AD2B692A6869680120B04795F811
:106C78002420531EFEF77DBD2B7D23E6DFED817AB0
:106C8800F4EEE76AF1EE10FA40F3D383DFED7E5AB3
:106C98009FED7E6A01E0F0EE676AF4EEC66AF1EEF7
:106CA80010FA76EEE57AF6DCDFED796AF4EEE67A4C
:106CB800F1EE10FA40F1B383DFED735A9FED756A78
:106CC80001E0F0EE667AF4EEC67AF1EE10FA77EEAD
:106CD800A56AF6D4DFED707AF4EEE76AF1EE10FA01
:106CE80005DDDFED687A77EEE66AFFF7FCBBDFEDDE
:106CF8006B7AF4EEE76AF1EE10FA44BFDFED647ADE
:106D080077EEE66AFFF7EFBB92F8FF31AA2B7FF424
:106D1800B9ADD2F8C6314BB192F8C211A1F10B004E
:106D280001282DD901F0F701062929D0D2F8D6314A
:106D38004BB192F8D211A1F10B00012820D901F032
:106D4800F70106291CD0D2F8E6314BB192F8E211CE
:106D5800A1F10B00012813D901F0F70106290FD082
:106D6800D2F8F631002B3FF48DAD92F8F221A2F162
:106D78000B01012904D902F0F702062A7FF482AD3B
:106D880041F2FC1101226B50AA70F4E5444B1B78C8
:106D9800002B40F0F581434B1B8B07EE903AF8EE41
:106DA800E77AFFF79EBADFED407AEAE6F4EEC77AB3
:106DB800F1EE10FA40F3B482DFED335A9FED336AF7
:106DC80001E0F0EE476AF4EEC66AF1EE10FA36EE2C
:106DD800E57AF6DCDFED2E6AB4EEE67AF1EE10FA2B
:106DE80040F19B82DFED285A9FED2A6A01E0B0EE60
:106DF800667AB4EEC67AF1EE10FA77EE256AF6D422
:106E08009FED257AF4EEC76AF1EE10FA40F3BC81E3
:106E18009FED1C7A77EE666A66EEA65A9FED235AB6
:106E28009FED236A9FED237AA5EE856A26EEA55A83
:106E3800A5EE867AE5EE076A50E69FED187AF4EE3D
:106E4800C77AF1EE10FA44BF9FED117A77EE677AB0
:106E580087E6DFF864A09AF81430052B3FF659ACA2
:106E680001A252F823F000BFD37000081B67000886
:106E780057700008236F0008596F00081171000847
:106E880004730020DB0F4940DB0FC940E4CB1641F7
:106E9800DB0F49C0E4CB16C1DB0FC93FDB0FC9BF0D
:106EA80024320020FC3100200000000092E741B9A4
:106EB8009730083C15A82ABE204D0020DAF8042097
:106EC80092F91A104B1C5C460AD0BE4B01F5817131
:106ED80003EB0113FF20D9796FF30001D971907684
:106EE80092F91B104D1C15D0B64D01F5817105EBBB
:106EF800011305EB0115DB79E979C3F34503012B90
:106F0800C6BF03F1FF33DBB20023FF2063F3460162
:106F1800E971D07603238AF81430AB48DAF8041004
:106F28000378002B7FF4F5AB002900F0998291F8E3
:106F38002830002B7FF4EDAB2838442227F047FB9C
:106F48000021DAF804001FF0C5F90023CAF804305C
:106F5800DAF81050DFF89092DFF890E2DFF890C28C
:106F68009A4B05F1010BA9FB0B58ACFB0B5CAEFB74
:106F78000BE50695964DA5FB0BE50895069D0FCBF1
:106F8800AD090695089D4FEAD80E4FEA5C1C6D0BBB
:106F98000DF13008CDF814C00895A9FB0EC5C446FC
:106FA800ACE80700059A06988CF80030A9FB022186
:106FB800ED08A9FB00020898069B05EB8505A9FBCF
:106FC8000009C908AEEB4500D208059D01EB810117
:106FD80002EB8202A5EB410141F2A40CA3EB4202B1
:106FE8004FEAD909089B774D09EB89090EEB8E0EFC
:106FF800ABEB4E0EA3EB490915F80C3030300EF10F
:10700800300C303201F1300E09F1300901218DF8D0
:1070180036008DF837C08DF835E08DF834208DF8BE
:1070280033908AF81410002B00F0818141F2E803B4
:10703800EB5C002B00F07A8141F22C13EB5C002B07
:1070480000F0D38104238AF81430FFF762BBDFF81D
:10705800A491DFF8A4815F4DA3460BAA4946DAF84C
:1070680004001EF0FDFF012841464FF0030240F0E6
:107078005A810B9C2046002C3FF420AF2378002B2C
:107088003FF41CAF27F03AFB032229460028E4D13D
:1070980004F1080027F032FB03460028DDD154F83C
:1070A800030F0C9022798DF834200CA88DF8353018
:1070B80025F00AF8DAF81030984203D90CA825F020
:1070C80003F80346CAF81030C7E73E4D6B78032B28
:1070D8007FF41FAB41F2A4020123AA5C8AF81430A2
:1070E800002A00F0D48141F2E802AA5C002A00F0EC
:1070F800BF8141F22C13EB5C002B00F0B881002318
:107108008AF81430FFF705BBB278FFF707BB17F012
:10711800EDFB00283FF4FDAA2F4BB2784FF48051C5
:1071280019800A233B70FFF7CAB8402017F082FB8A
:1071380000287FF4EEAA2B68DFF8C080DFF8C0A033
:107148004FF040090DE017F011FCDAF800202B6829
:10715800013A0133B9F10109CAF800202B6000F0A7
:10716800468118F803301846002BECD100234FF065
:10717800FF322B6004236A603B70B278FFF79FB838
:10718800DFED167AFFF7ADB89FED157AF4EEC76A12
:10719800F1EE10FA44BF9FED137A77EE666A3BE68C
:1071A80000F0B480042385F82430FEF74CBB00219E
:1071B800DAF800001FF08EF800287FF468A8FFF7BF
:1071C800A8BA00BF3C3700201C4900208C150308D2
:1071D8005917B7D1C4100308802E00200000000002
:1071E800DB0FC9BFDB0F49C0CDCCCCCCD34D62106F
:1071F8001F85EB51284D0020C010030804EA02083F
:10720800BC4D0020137C022B7FF4C9AB92F8FE31F1
:10721800552B7FF4C4AB92F8FF31AA2B7FF4BFAB98
:10722800D189AF59B74B0F441F60567B41F21020EC
:10723800731E7F2B2E503FF6B2AB734236EA030320
:107248007FF4ADAB41F218207302013B2B50D08A7A
:1072580000B9506ADFF860E341F20423E850B2F85D
:1072680011305B0103F2FF135B12CEF80030B2F865
:1072780013C0BCF1000F01D1D2F820C0400019445E
:107288000144ACEB010141F2082E40F6F47CB1FB5D
:10729800F6F1614545F80E1040F2BD804FF6F476E0
:1072A800B14240F2BF8003212970D26A96493B441B
:1072B800184441F20C2641F21C230978A851EA50DF
:1072C80009B91FF045FFAB780133AB70FEF75ABA26
:1072D80002283C467EF456AA41F2B4120123AB546C
:1072E8006B70FEF74FBA1EF005FE2B69FFF774BAF4
:1072F800864D28680CF0A6FA854B1B780022022BD5
:107308002A6000F09380B278FEF7D7BF11F0AAFB8D
:1073180002287EF49AAAFEF796BAF0EE476A6FE55D
:10732800B0EE667A56E55C46FFF7F3B90B4603EB19
:10733800031305EB830000F58550764B0093414617
:107348003C23202204301FF00BFBFFF7E2B9F0EEDC
:10735800477AFFF7FABBB0EE677AFFF7E0BB6E4BF0
:107368006E491A8A6E4812F0B1FB2B68B278013365
:107378002B60FEF7A4BF1FFA89F31FFA88F2694948
:10738800694812F0A3FBF0E74FF07E52674968485E
:1073980012F09CFBE9E7674B6749DA8A674812F005
:1073A80095FBE2E7634B64499A8A654812F08EFBC5
:1073B800DBE7737832786349634812F087FBD4E7D8
:1073C800624A6349634812F081FBCEE7624B634A25
:1073D8006349644812F07AFBC7E7802014F002FE84
:1073E80000287EF4D7A9FFF7E3BB02239FE718F82C
:1073F8000330002B7FF48DA9B8E6452017F0B6FAC4
:10740800FF2017F0B3FA584817F084FA304617F0FF
:10741800ADFAFEF7F5BF01232B70FFF7C0BAF0EE07
:10742800676A57E402222A7000223FE70BF008FD42
:1074380069E7F0EE667A37E40222FEF743BF4B4A6B
:107448004B4B019200934B4A4B4B4C494C4812F022
:107458003DFB8AE7474A3E494A4812F037FB84E732
:107468001FF076FE00287FF46BADFFF752B90223B8
:10747800442202FB035303F58550434B009310222B
:107488001323424904301FF06BFAFFF742B9134641
:10749800EEE73F4A2349D3893E48528912F016FB4A
:1074A80063E73B4B24495A793B4812F00FFB5CE7F2
:1074B800374B21491A79394812F008FB55E7344B04
:1074C8001D49DA78364812F001FB4EE762791A490D
:1074D800344812F0FBFA48E722791749324812F08B
:1074E800F5FA42E7314B14491B6831489A8D12F07E
:1074F800EDFA3AE72D4B10491B682E485A8D12F0C9
:10750800E5FA32E73C4900201C490020C04D002024
:1075180039300020D5DD0108D85E00209C11030811
:10752800A0110308881103089011030874110308B7
:107538007C110308FC310020581103086811030866
:107548005C110308441103084C1103089C5E0020D9
:10755800D410030838110308D00E0308C40E03081A
:1075680020110308281103088015030814110308C3
:10757800DC0E0308C8100308E8100308F01003081D
:1075880000110308D810030819E80108B810030807
:10759800E06000204414030834140308201403088E
:1075A800141403080414030808140308B05E002028
:1075B800F0130308E01303085C490020A84BA9490D
:1075C8001B68A948DA8F12F081FACEE6A44BA549C8
:1075D8001B68A6489A8F12F079FAC6E6A04BA14913
:1075E8001B68A34893F83B2012F070FABDE69C4B49
:1075F8009C491B689F4893F83A2012F067FAB4E652
:10760800974B98491B689C481A8F12F05FFAACE6B2
:10761800934B94491B689948DA8E12F057FAA4E6FE
:107628008F4B90491B68964893F8302012F04EFA19
:107638009BE68B4B8B491B68924893F82F2012F0DE
:1076480045FA92E6864B87491B688F4893F82820AD
:1076580012F03CFA89E6824B82491B688B48DA8C27
:1076680012F034FA81E67E4B7E491B6888489A8C72
:1076780012F02CFA79E67A4B7A491B6885485A8CBD
:1076880012F024FA71E6764B76491B6882481A8C08
:1076980012F01CFA69E6724B72491B687F489A7FA0
:1076A80012F014FA61E66E4B7D49D3F800E07D488C
:1076B8009EF81C309EF81B209EF81DE0CDF800E0D7
:1076C80012F004FA51E6664B66491B6876481A7E42
:1076D80012F0FCF949E6624B7149D3F800E07348AF
:1076E8009EF816309EF815209EF817E0CDF800E0B9
:1076F80012F0ECF939E65A4B6949D3F800E06C48C6
:107708009EF813309EF812209EF814E0CDF800E0A1
:1077180012F0DCF929E6524B6149D3F800E06548DC
:107728009EF810309EF80F209EF811E0CDF800E08A
:1077380012F0CCF919E64A4B5949D3F800E05E48F3
:107748009EF80D309EF80C209EF80EE0CDF800E073
:1077580012F0BCF909E6424B5149D3F800E057480A
:107768009EF80A309EF809209EF80BE0CDF800E05C
:1077780012F0ACF9F9E53A4B4949D3F800E0504822
:107788009EF807309EF806209EF808E0CDF800E045
:1077980012F09CF9E9E5324B4149D3F800E0494839
:1077A8009EF804309EF803209EF805E0CDF800E02E
:1077B80012F08CF9D9E52A4B3949D3F800E0424850
:1077C8009EF801309EF800209EF802E0CDF800E017
:1077D80012F07CF9C9E53D4B22491A683C4812F081
:1077E80075F9C2E592781F493A4812F06FF9BCE57D
:1077F800394B1C495A8A394812F068F9B5E5364BB5
:1078080018491A88364812F061F9AEE5324B154925
:107818009A78344812F05AF9A7E52F4B11491A798A
:10782800314812F053F9A0E59BF808200D492F487C
:1078380012F04CF999E5BBF824200A492C4812F0BB
:1078480045F992E59BF8202006492A4812F03EF9AE
:107858008BE59BF81E200349274812F037F984E589
:10786800B05E002058110308D4130308C41303089A
:10787800AC130308901303087C130308641303086C
:107888005013030840130308301303081C1303089C
:107898000C13030800130308F0120308DC12030892
:1078A80070120308D4120308CC120308C01203088C
:1078B800B8120308B0120308A8120308A01203089C
:1078C800981203088C12030884120308442C002021
:1078D8007415030868150308FC31002054150308C3
:1078E80044150308301503081C1503080815030878
:1078F800EC140308D0140308BC14030894F8982067
:107908006F49704812F0E2F82FE56F4B6C49DA784E
:107918006E4812F0DBF828E56D4B69491A786D4816
:1079280012F0D4F821E56C4B6549DA786B4812F00F
:10793800CDF81AE5684B9FED6A7A1B88604969485B
:1079480007EE903AF8EEE77A67EE877AFDEEE77A87
:1079580017EE902A12F0BAF807E5634A6349138ACA
:107968006348928912F0B2F8FFE4624B62496348B7
:107978000C2202FB0E3E9EF806309EF805209EF86B
:1079880007E0CDF800E012F0A1F8EEE4594A4C49BE
:107998005B480C2303FB0E2EBEF80A2012F096F863
:1079A800E3E4544A464957480C2303FB0E2E9EF83D
:1079B800082012F08BF8D8E44E4A414952480C236B
:1079C80003FB0E2E9EF8042012F080F8CDE4494AFD
:1079D8003B494E480C2303FB0E2E9EF8032012F061
:1079E80075F8C2E4434A364949480C2303FB0E2E76
:1079F8009EF8092012F06AF8B7E43E4A3049454833
:107A08000C2303FB0E2E9EF8012012F05FF8ACE465
:107A1800384A2B4940480C2303FB0E2E9EF80220BF
:107A280012F054F8A1E40C2303FB0EFE314B244959
:107A380013F80E20394812F049F896E4384B2049DB
:107A48001A78384812F042F88FE4274B1C499A7884
:107A5800354812F03BF888E4344B19491A68344821
:107A680012F034F881E4334B5B79012B7FF47DAC61
:107A7800B4F99430B4F996201C492F4812F026F82E
:107A880073E42E4B2E491A882E4812F01FF86CE426
:107A980028482D4983784278007800902B4812F0C6
:107AA80015F862E42A4B1B68D80402D40C232B6017
:107AB8005BE4284B22491A78274812F007F854E467
:107AC80058110308A4140308C030002094140308B4
:107AD800D030002084140308344C002074140308A8
:107AE8000000C84268140308E060002088110308F9
:107AF80054140308B45E0020701203087C120308B3
:107B080060120308541203084812030840120308BD
:107B18003412030828120308201203081812030855
:107B28005856002004120308F411030818690020AD
:107B3800E81103087C600020D8110308A02E00205B
:107B48009C110308D0110308B4110308C0110308DD
:107B58009C2E0020CF740020A81103082DE9F04FB7
:107B68002DED028B8FB006461BF000FB9C4B1F7857
:107B780027B10FB0BDEC028BBDE8F08FDFF8C0B2C3
:107B8800DBF800305905F4D5964B974D1B78002B40
:107B980040F05C81954B1B78002B6BD0944C954A38
:107BA800D4F86C31F31A934201F2478094F8748147
:107BB800B8F1000F31D1904F3868FBF7EBFAC0B23B
:107BC80001280ED9022841F0E6838C4B1A78002A46
:107BD80041F0ED85D4F87821B21AB2F57A6F81F0C8
:107BE8004C87D4F87C31002B44D094F87431BBB95D
:107BF800834B1B689B7801211E3B00228B4284F833
:107C0800741184F8882141F23786386802210430DB
:107C18001AF095FE94F880310FE0D4F87C314BB31C
:107C2800D4F8843140F6B732F31A934222D994F843
:107C38008031002B01F0E0826F4F013BDBB284F80A
:107C48008031002B01F06B80D4F87C1194F88821E6
:107C580011F801EB94F88931C4F87C1172440133AE
:107C6800386884F88821714684F88931FBF796FAD8
:107C7800C4F88461634B2F681B7853B1DFF8C48163
:107C8800D8F8000028B1604B1B78013B012B41F26A
:107C980055805E4B1B7863B15D4F3B684BB1544CCC
:107CA800D5F80090D4F8C032A9EB0303632B00F297
:107CB8002587584C2378022B01F07F82DFF88881D2
:107CC80098F80030032B01F01680534B1B7873B1E2
:107CD800524F3B685BB1464C03F0D8FBD4F8C8322E
:107CE800009044F61F62C31A934200F27F814C4B06
:107CF8001B78002B4BD14B4B1B7843B13C4CD4F831
:107D0800183403F5C333A0339E4280F05787464B9F
:107D18001B78002B3FF42DAF354E444C444D06F2F2
:107D280039472068FBF736FA00283FF422AF20686D
:107D3800FBF72CFA2B7880465A1E33B120682A703C
:107D4800FBF728FA0028F2D113E703223946781EF8
:107D580026F048FC96F8383496F8392486F83B849F
:107D680083F47F4383F0FF039B1A1FFA88F89BB2C2
:107D7800B8EB132FD5D196F83A24DBB29A42D0D17A
:107D8800781E1AF0EBFC2B7818442870C9E7294CA8
:107D98002278002A40F0F286154CD4F8103403F506
:107DA800C333A0339E42A6D3234A94F81434C4F8AC
:107DB8001064D55CE90701F1EC83AA0701F1A883F7
:107DC8006B0701F1B4821D4A94F814341178013319
:107DD80093FBF1F201FB123384F814348BE700BFF4
:107DE800755E0020945F0020047300209E5F0020D1
:107DF800501D00203F0D0300545E002004000020A9
:107E0800585E0020A05F0020A85F0020B05F00201F
:107E1800E4770020844E0020B85F0020BC5F00207B
:107E28002460002032600020C25F0020C85F00206C
:107E3800CC5F00208C5F00202C6000203160002087
:107E480020370020FC5D00203D0F00205D4C2A6893
:107E5800D4F85C31D31A7C2B7FF69CAE94F8603151
:107E6800DFF880919FED588AC4F85C21013384F8CB
:107E780060314FF0240840461AF014FE534BF9ECD9
:107E8800016A1B8A07EE103AF8EEE66AB8EEC77A7E
:107E980008F10108C6EE877A5FFA88F867EE887AF3
:107EA800FDEEE77ACDED007ABDF900A05FFA8AF021
:107EB8001AF0CEFDCAF307201AF0CAFDB8F1270F51
:107EC800D9D130201AF0EEFDD4F86491DFF818818A
:107ED8005FFA89F01AF0BCFDC9F307201AF0B8FD63
:107EE800D8F800005E21FBF759F994F860319A0739
:107EF8002DD1D4F85C2141F288339A4201F28E8563
:107F080014201AF0CFFD324B324AB3F9043082FB09
:107F180003124FEAE379C9EBA2090FFA89F95FFA6C
:107F280089F01AF095FDC9F307201AF091FD1C207D
:107F38001AF0B8FD00201AF08BFD00201AF088FD19
:107F48005E21D8F80000FBF729F994F8603158074A
:107F580001F09A83282B7FF41DAE00271720D5F84F
:107F6800009084F860711AF09DFD38461AF070FD93
:107F7800194B1A4CA3FB09239B0BA4FB03125209B0
:107F8800C2EB0212A3EB8203D8B21AF061FD1820EB
:107F98001AF088FD124BA3FB09239B09A4FB0312CB
:107FA8005209C2EB0212A3EB8203D8B21AF050FDB9
:107FB80038461AF04DFDD8F800005E21FBF7EEF8C0
:107FC800E8E500BF501D002000007A44D85E00207C
:107FD8002C5F00206766666673B2E74589888888E3
:107FE800D34D62100C5F00205C5E002094F8CE3206
:107FF800002B41F07981E34B1A6802F00803002B4B
:1080080048F603414AF60B404BF60F4349F607483A
:1080180004BF0346884612F0040F4FF0190118BF39
:108028009846920684F8CE1203D548F4804848F062
:108038002008D54B1A79C8F309010191002A41F0AB
:108048005A855B79002B41F0D9869A4664204FF017
:10805800FF330A464FF00009CDF81880CDF81C8090
:108068000892ADF826A0ADF828308DF83600ADF8A6
:108078002490CDF82A90CDF82E90CDF832900DF1BD
:10808800180CBCE80F00DFF810E384F85190AEE854
:108098000F009CE80F00AEE807002EF8023B71467F
:1080A8004FF0010C1B0C4FF0FE0E1F20C82201F8E8
:1080B8001E3984F84EE084F8522084F853C084F8BE
:1080C8004F0094F8DE0284F8500080F0F10383EA50
:1080D8000313DAB2130983F0E70343EA022383EABE
:1080E800C2031BB283EA0312D2B2C3F3072383EAA3
:1080F800121343EA022383EAC2031BB283F0C802C5
:1081080082EA0212D2B2C3F3072383EA121343EAC4
:10811800022383EAC2031BB283EA0C0E8EEA0E1E08
:108128005FFA8EFEC3F3072282EA1E1242EA0E228B
:10813800604482EACE0E84F8DE02A4F84CE001F135
:108148001F0011F8013B83EA0E0383EA0313DBB235
:108158001A0982EA1E2242EA032282EAC3031BB2F8
:108168001FFA83FE8142A4F84CE0EAD183F07C0335
:1081780083EA0313DBB21A0982EA1E2E8EEA032E63
:108188008EEAC30E0FFA8EFE1FFA8EF34FEA132AF9
:108198005FFA8EFEA4F84C30DFF8009284F874A0E1
:1081A80004F16E0384F873E004F14E0C0193DCF8DB
:1081B8000C30DCF80000DCF80410DCF80820C846B5
:1081C800A8E80F00019B0CF1100C9C45C146EED1AC
:1081D800DCF80000C8F80000DFF8C4819CF804301F
:1081E80089F8043008F1270984F82DE384F82EA3D0
:1081F80018F8011F3868FAF7D1FFC145F8D194F88B
:10820800CF22002A41F0758060492B6808780A213E
:1082180084F8CF12002801F07181DFF888C10128A5
:10822800BCF80010059141F2C185BCF8021002911A
:10823800022801F07C84BCF804100391032801F0A3
:10824800F485BCF806100191042801F0E88505289A
:10825800BCF8081001F0DE850628BCF80AA001F079
:10826800D5850728BCF80CE001F0B985BCF80E905C
:1082780094F8DE220693104680F0300383EA031355
:10828800DBB20490424A9DF810C0128884F850C0AE
:10829800180980F07A0040EA032080EAC3033D48C9
:1082A800C2EB022280FB02C01044D217C2EB60224C
:1082B80005988DF82D204FF0000860F30F080398FB
:1082C8004FF0000C60F30F0C00201BB261F30F009D
:1082D80000216EF30F0183EA031EC3F30723039300
:1082E800029B63F31F48019BCDF81C8063F31F4C6E
:1082F800039BCDF820C05FFA8EFE6AF31F4069F336
:108308001F4183EA1E134FF0000A09900A918DF865
:108318002CA043EA0E2C0DF11809B9E80F008CEADD
:10832800CE0E0FFA8EFE8EF0C808DFF86CC084F807
:1083380051A088EA08185FFA88F8CEF3072EACE84F
:108348000F008EEA181E4EEA082399E8030083EA14
:10835800C8080FFA88F383F023024CF8040B82EA6A
:108368000210C0B2C3F3072282EA1012049B2CF851
:10837800141942EA0022591C82EAC0004FF023086F
:10838800162211E0286900207C600020345F00205C
:108398003C2E002003082080A41D00205820002027
:1083A80057200020BC8300204FF0FE0EC82384F81D
:1083B800DE12A4F84C000CEB020184F8538084F818
:1083C8004EE084F84F2084F852301CF8013B4340BB
:1083D80083EA0313DBB21A0982EA102242EA032273
:1083E80082EAC3031BB298B28C45A4F84C00ECD1C6
:1083F80083F0F40383EA0313DBB24FEA131E8EEA19
:10840800102E8EEA032E8EEAC30EA0460FFA8EFEB9
:108418001FFA8EF958F84E0FDFF818C4A4F84C90DC
:108428004FEA192A5FFA8EFE84F86AE084F86BA096
:10843800D8F80410D8F80820D8F80C30ACE80F00A9
:10844800D8F81000D8F81410D8F8182004F22539F4
:10845800ACE8070004F2073884F825A384F824E37D
:1084680018F8011F3868FAF799FEC145F8D194F851
:10847800D6E2BEF1000F40F04687E64B94F8DEC224
:10848800B3F90010B3F90220B3F904309FEDE26AA2
:1084980084F851E007EE103A2B6806938CF06A03D3
:1084A80083EA031306EE901AD9B20B0983F0D503B9
:1084B80043EA012383EAC1031BB283EA0311524250
:1084C800C9B207EE902AC3F3072383EA111343EADC
:1084D8000123F8EEE77AF8EEE66AB8EEC77A83EA9F
:1084E800C1031BB267EE867A66EE866A27EE067AC5
:1084F800002083F0C805CDED087ACDED076A8DED33
:10850800097A0A900B900C9085EA05150DF1180967
:10851800EDB2C3F30728B9E80F0088EA151848EA4E
:10852800052888EAC505DFF810832DB2A8E80F00F2
:1085380085F01E0E99E807008EEA0E13DBB2C5F32C
:10854800072E8EEA131E4EEA032E88E807008EEAED
:10855800C30EA8F110051C20C8214FF005091E23E1
:108568004FF0FE080CF1010284F8521084F8D692FC
:1085780084F8533084F84E8084F84F00291884F822
:1085880050C0A4F84CE084F8DE2215F8013B83EAD9
:108598000E0383EA0313DBB21A0982EA1E2242EAB7
:1085A800032282EAC3031BB21FFA83FE8D42A4F89A
:1085B8004CE0EAD183F0270383EA0313DBB21A09FC
:1085C80082EA1E2E8EEA032E8EEAC30E0FFA8EFE64
:1085D8001FFA8EF34FEA13295FFA8EFEDFF85482F2
:1085E800A4F84C3084F8719084F870E004F14E0CD3
:1085F80004F16E0ADCF80000DCF80410DCF808204E
:10860800DCF80C3045460FC50CF1100CD445A846D3
:10861800F0D1824DBCF80030A8F8003005F12408EC
:1086280084F82AE384F82B9315F8011F3868FAF7C1
:10863800B5FD4545F8D194F8D7320293002B40F0A8
:108648005D86774B1B68052213F0140F84F8D72238
:1086580040F0B286DFED737A94F8DE826D4B724A91
:10866800B3F90410B2F90620704D7148CDED087ABF
:1086780088F0220383EA03135FFA83FE4FEA1E138E
:1086880083F05903B2F5FA6F43EA0E2383EACE0367
:10869800A8BF4FF4FA621BB2B2F57A7F83EA031ED1
:1086A800B8BF4FF47A725FFA8EFE4FF0640CA2F5F1
:1086B8007A72C3F307230CFB02F283EA1E1385FBCD
:1086C800025980FB0150D21743EA0E25C9174FF013
:1086D800000AC2EBA912C1EBA00185EACE050DF193
:1086E800180CADF82A20ADF82810CDF818A0CDF850
:1086F8001CA0CDF824A02DB285F0C80ECDF804C07A
:10870800BCE80F008EEA0E1E5FFA8EFEC5F3072541
:1087180085EA1E15DFF82091DCF800C084F8508047
:1087280045EA0E25A9E80F0085EACE0212B282F0CA
:108738004A0383EA0313DBB2C2F3072282EA131265
:1087480049F810C942EA03224A2082EAC3034FF0DB
:10875800140E002508F101084FF0FE0C84F85300B0
:10876800C82084F8515084F8DE82A4F84C304A4678
:1087780009EB0E0184F84EC084F84FE084F85200EB
:108788001D4612F8010B684080EA0010C0B20309C8
:1087980083EA152343EA002383EAC00000B285B2C6
:1087A8008A42A4F84C50ECD180F0140080EA001002
:1087B800C0B24FEA101E8EEA152E8EEA002E8EEAFF
:1087C800C00E25460FFA8EFE1FFA8EF855F84E0F8A
:1087D800DFF860C0A4F84C804FEA182A5FFA8EFED2
:1087E80084F869A084F868E06968EB68AA68ACE86E
:1087F8000F00286969692B8BACE8030004F2073580
:10880800ACF80030A84684F823A384F822E304F2E5
:10881800233A13E02C5F002088C3E43A5720002055
:108828002869002000000000BC830020D34D62109E
:108838006766666658200020A41D002018F8011FEE
:108848003868FAF7ABFCC245F8D1D14BD14A1B784E
:108858001278013B12F00100DBB214BFC0224022A3
:10886800172B04D8CC490B4493F824300293CB4BF4
:1088780019888B071ABF002342F01002012311F454
:10888800027F18BF022311F0100F18BF062311F042
:10889800200F18BF1023002841F07C80032194F892
:1088A800DEE206938EF0460383EA0313D8B2030987
:1088B80083F0920343EA002383EAC0031BB283EAEE
:1088C8000310C0B2C3F3072888EA101848EA002842
:1088D80088EAC0080FFA88F888F0C80C9DF80800E4
:1088E8008DF81C008CEA0C1C00235FFA8CFC8DF8B8
:1088F8001E200320019A8DF81D30C8F307288DF833
:108908001F108DF8200088EA1C1807CA48EA0C28AE
:1089180088EACC0C0FFA8CFC8CEA0C18A9E8030046
:108928005FFA88F8CCF3072181EA181141EA082197
:1089380081EAC80894F854C089F800200FFA88F230
:108948008CEA020C8CEA0C1C5FFA8CFCC2F307223E
:1089580082EA1C1242EA0C2294F8550094F8561048
:1089680094F8579094F8588084F8533082EACC02EF
:1089780012B2504080EA0010C0B2C2F3072282EA65
:10898800101242EA002282EAC00212B2514081EA81
:108998000111C9B2C2F3072282EA111242EA012286
:1089A80082EAC10212B289EA020989EA09195FFA60
:1089B80089F9C2F3072282EA191242EA092282EAF5
:1089C800C90212B288EA020888EA08185FFA88F829
:1089D800C2F3072282EA181242EA082294F859C020
:1089E80094F85A0094F85B1094F85C9084F851302D
:1089F80082EAC80212B28CEA020C8CEA0C1C5FFAFA
:108A08008CFCC2F3072282EA1C1242EA0C2282EA98
:108A1800CC0212B2504080EA0010C0B2C2F3072262
:108A280082EA101242EA002282EAC00212B25140DF
:108A380081EA0111C9B2C2F3072282EA111242EA9D
:108A4800012282EAC10213B289EA030282EA02120F
:108A5800D2B2C3F3072383EA121343EA022383EA59
:108A6800C2031BB283F0320282EA0212D2B2C3F30B
:108A7800072383EA121343EA022383EAC2031BB2E1
:108A88009AB24FF0FE0CDFF8288184F850E00920F4
:108A9800C8210EF1010EDBB284F84EC04FEA122C49
:108AA80084F84F0084F8521084F8DEE2A4F84C20D1
:108AB80084F85EC084F85D30D8F80000D8F8041057
:108AC800D8F80820B8F80CA008F2BA2EAEE80700CB
:108AD80008F2CA288EF80290AEF800A084F818C3ED
:108AE80084F8173315F8011F3868FAF757FBA845BB
:108AF800F8D1009BC4F8C832FFF7F9B8DFF8B4A082
:108B0800DFF8B480412019F0CDFEBAF9023088FBB5
:108B18000320DB17C3EBA00080B219F0A9FEBAF955
:108B2800003088FB0320DB17C3EBA00080B219F0EC
:108B38009FFEBAF9043088FB0320DB17C3EBA000C3
:108B480080B219F095FE164B38681978FAF726FBAB
:108B580094F8C43213F0010800F03C84114AC4F8B8
:108B6800C0920133DBB2A2FB0312D20802EB8202ED
:108B7800A3EB420384F8C432FFF79BB80A4B0B49B6
:108B88001868FAF7DFFA00232370FFF705B900BF6A
:108B9800543000203585002078EC0208D0230020CE
:108BA800D8840020CDCCCCCC28600020685F002081
:108BB8009E1D00202C5F00206766666694F81C34B2
:108BC800C74AC4F8186402EB8302D26B42B30EADF5
:108BD80004F22343C34E45F8203D002104F23543F7
:108BE8003180079380211523A52784F8223428464D
:108BF80084F8211484F82074904728463188FBF7BC
:108C0800F7FB069DB84804F584616D1A152DA8BFB9
:108C180015252A4625F0DBFCB44A94F81C34157057
:108C2800B34A013382FB0312A2EBE37202EB420266
:108C38009B1A84F81C34FFF76AB8AE4BAE4AD4F8D6
:108C480070112868128893F80BE0AC4B401A4FF467
:108C58007A71D7B201FB0EF1120A9F771F7588420D
:108C68004FF00007DA775A759F701F7180F05183B3
:108C7800A34AA449DFF89CC212680F688868DFF825
:108C880098E2C4F86C618CFB0281D217C2EB6112C6
:108C9800D4F864118CFB018C8EFB07988EFB009E28
:108CA800C017C0EBAE0002F5FA724FEAE17E92B24D
:108CB800CEEB6C1CFF1701F5EA4EC7EBA8070EF1C7
:108CC800300E9A76120A0CF1780C4FEA2E2E3031BB
:108CD800DA764FEA272802121F7783F81D8083F877
:108CE800200083F8212083F824C083F823E083F848
:108CF8002210FEF75BBF844F386803685B699847AA
:108D080000283EF4E2AF3868036801219B69984760
:108D18000222002388F800202370FEF7D6BF94F8BB
:108D2800881194F8893138684A1C013384F88821FD
:108D380084F88931FAF732FAFEF79ABF734CDFF8F4
:108D4800DC914FF0000A0BE01B2B00F049820D2B41
:108D580000F012824FF0010389F80130D8F80000C2
:108D6800FAF718FA002837D0D8F80000FAF70EFA00
:108D780083B27E2B2A6828D099F80120002AEDD1E9
:108D880094F88A110029DFD07D2B00F0098294F82D
:108D98008EE1BEF1000F04D080F02003DBB284F82E
:108DA8008E214A1CD2B2092A635484F88A2100F021
:108DB800EB81082AD2D8B4F88C21134403EB13238F
:108DC80003F0FF03A4F88C31C8E784F88AA184F87B
:108DD8008BA189F801A0C1E794F88F312BB1637892
:108DE80084F88F01302B00F0658594F88B213C4B7B
:108DF800DFF82C91DFF82CC1DFF82CA14FF0010E21
:108E0800002A3EF446AF2968C91B012900F2AF8148
:108E180094F8A482B8F1000F40F0F98194F8BC12DC
:108E280033F8110010B984F8BCE2E9E70131B0F574
:108E3800826F84F8BC1200F0E0801ED9B0F5E26FB2
:108E480000F0C18034D9B0F5046F00F0CA80B0F5E5
:108E5800116F00F02581B0F5E46FD1D12C4AD76BA2
:108E6800118A642303FB07F393FBF1F119F04DFD1D
:108E7800002384F88B31FEF70CBFB0F5007F00F0BB
:108E8800298153D8B0F5807F00F04781B0F5887FFD
:108E9800B6D1D9F800104907B2D5D4F864114FF407
:108EA800887019F032FD002384F88B31FEF7F1BE8B
:108EB800B0F5C06F00F02181B0F5E06FA0D1144A81
:108EC800506B118A642303FB00F34FF4E06093FBBB
:108ED800F1F119F01AFD002384F88B31FEF7D9BEA1
:108EE80078EC0208405F0020984A0020AD4A002034
:108EF80056555555345E0020005E0020D05F002096
:108F0800BC1C0020045E0020984C0020501D00204E
:108F1800D85E00201F85EB51676666660400002056
:108F2800286900207C600020425E0020B0F5047FA4
:108F380000F00381B0F5806F7FF462AF94F8BD3222
:108F48000133DBB2032B00F2328142F2107184F854
:108F5800BD3201FB03F1BE4B1B88002B40F025817D
:108F68000131BC4B1B78D807BB4B1B8848BF043169
:108F7800DA0748BF0A31980748BF14311A0648BFB4
:108F88002831D80548BF28315A0748BF6431180727
:108F980048BFC8319A0548BF01F5C871980648BF4F
:108FA80001F57A71DA0648BF01F5FA61580648BF3B
:108FB80001F57A614FF4806019F0A7FC002384F86A
:108FC8008B31FEF766BEA54A976B118A642303FBB3
:108FD80007F393FBF1F119F098FC84F88B81FEF705
:108FE80058BE9F4BB3F9041001EB8101490019F0F9
:108FF8008CFC84F88B81FEF74CBED9F8001011F078
:1090080020087FF4FDAEDBF80010090600F13C846F
:109018009449097B00293FF4F3AE94F8BE12032962
:1090280000F24486DFE801F0322819028E4B1B68F3
:1090380059799A79DB7901F1407101EB022101EB51
:109048000341002384F8BE324FF4826019F05DFCBE
:10905800002384F88B31FEF71CBE844B1A68137A00
:10906800507992781B0403EB002313444A1C84F8BC
:10907800BE2203EB0161E7E77C4B1A68D3791079CC
:1090880052781B0403EB00231344EFE7774B1A686D
:109098009379D07812781B0403EB00231344E5E797
:1090A8009CF8041000293FF4ABAE9AF80010002990
:1090B8003FF4A6AE6E4B1B8803EB83035B004FF4B3
:1090C800116093FBF1F119F020FC002384F88B3137
:1090D800FEF7DFBD9CF8051000293FF491AE654B03
:1090E80065491B6881FB0321DB17C3EBA10119F05C
:1090F8000CFC84F88B81FEF7CCBD9CF80510002988
:109108003FF47EAE5B4B4FF4C060996819F0FDFBED
:10911800002384F88B31FEF7BCBDD9F8001048074E
:109128007FF56EAE554B4FF48070196819F0EDFB62
:10913800002384F88B31FEF7ACBD9CF8041000299D
:109148003FF45EAE9AF8000000283FF459AE454B54
:109158005B7B002B00F01A84454B198891FBF0F1DA
:1091680001EB810149004FF4047019F0CEFB002394
:1091780084F88B31FEF78DBD4FF0010284F88A2107
:109188002370A4F88C11E9E5B4F88C21C2F1FF0230
:1091980093427FF4DFAD4FF0010384F88F31D9E5B6
:1091A8004FF0010384F88E31D8E50231D9E6012366
:1091B80084F8BD3242F21071CDE602F067F9304B07
:1091C8001A6840F6B833801A984200F2EB802D4FA7
:1091D8003B793A2B00F0F18200232370FEF775BD2E
:1091E800D8F80000F9F7D6FF00287FF4B3AD4FF0A8
:1091F800010384F88B31B1E5C4F87C3184F874310B
:10920800214F19F0CFFB94F88031FEF716BDD4F842
:109218009432DFF8789094F8BA224B4500F04A84EB
:10922800511C94F8BBE2D4F898C284F8BA1202F040
:109238000F028DF818200DF11902ACEB030100297B
:1092480040F3458506A901910DF11E0723E000BFF3
:109258003A4D002035850020D0230020D85E00201C
:109268002C5F0020345E0020FC860020B05E0020C9
:10927800005E0020045E002067666666BC1C002055
:109288008C4E0020744E0020545E0020E41E002006
:10929800002840F39C800133C4F8943213F8011C71
:1092A80002F8011BBA42ACEB030081EA0E0EEFD3C1
:1092B80084F8BBE200F00585501CB84282F800E053
:1092C80005D20EAB9A1A1B3A002125F0A5F901998F
:1092D800322019F0FFFA4FF00008002384F8A48226
:1092E80084F88B31FEF7D5BC013B84F8CE32FEF70B
:1092F80086BF013A84F8CF22FFF7B9B8013B84F85A
:10930800D732FFF7F6BB0EF1FF3E84F8D6E2FFF73F
:1093180092B9C64A29681278C4F87011013A012A2C
:109328003FF6A6AC1021022299701A71A0E4C04A37
:10933800C04B12680793A3F1240800202121D5000F
:1093480003F8240C88F8021040F11483BA49032763
:10935800BA4B1B88580500F10A83DA0700F1E48349
:1093680003F00203B64A002B1CBF03271146B54D74
:109378003A46284625F02BF97B190EA80133A91E79
:1093880040F8203D00225B1A7A5588F8013019F020
:10939800ABFEFEF718BD19F0F5FAAB4B01221A70B7
:1093A800FEF71FBCA94AB2F8C63200210133A2F861
:1093B800C6322170FEF789BCA54B9FEDA67AD3ED86
:1093C800007AF8EEE77A67EE877AFFF745B984F80E
:1093D800BBE271E7994B1B88DA0515D4D80600F172
:1093E800AE83990600F15E845A0600F19E84180740
:1093F80000F1BD84D90700F19C8413F0020F0CBF63
:109408004FF004084FF00C08934B944A1B78D2781D
:1094180003F001030AB143F002035320009319F04B
:1094280041FA8F4A128802EB820202EB8202900014
:1094380080B219F01DFA002019F01AFA894A8A49EF
:1094480012883868C2EBC212520081FB0231114403
:109458004FEAE27ACAEB612A5FFA8AFA5146F9F7CB
:109468009DFE824B38681A78009B48EA03087F4BB8
:109478008AEA020A002183F800A0F9F78FFE414624
:109488003868F9F78BFE794B784A1B78386888EA90
:109498000303DBB219461370F9F780FE94F8C4325F
:1094A800002B7FF45BAB4F2019F0FCF91FF008FC90
:1094B8001FF006FC1FF004FC01213868F9F76EFE66
:1094C8006B4A6A4B92F800801B78684A386808F043
:1094D8000108414683F001031370F9F75FFE634BFF
:1094E80038681B7888EA0308604B414683F8008097
:1094F800F9F754FE94F8C432FFF730BB864682462B
:10950800014601900390029005908146FEF7B0BE97
:10951800484B534907930EAFA3F1210047F8200D9C
:109528004FF0080E4FF000080A2003F822EC03F869
:10953800230C03F8248C38460988FAF733FF4D4B7F
:109548004D491B6881FB0321DB17C3EBA10138469A
:1095580089B2FAF727FF494BB3F8069009F0CCF91E
:10956800069B5A1C069283F80080069B4FEA192234
:10957800591C06911A70069B5A1C069283F8009093
:10958800069B5A1C06921870384619F0ADFDFEF776
:1095980017BCDFF8F0809FED3A8AB8F90230254A07
:1095A800079207EE903AF8EEE77A0EAF67EE887A00
:1095B800A2F12403FDEEE77AA2F12101002047F889
:1095C800201D02F8240C0822CDED007A5A701E22C4
:1095D8009A70BDF800103846FAF7E4FEB8F9003082
:1095E80007EE903AF8EEE77A384667EE887AFDEEAD
:1095F800E77ACDED007ABDF80010FAF7D3FEB8F996
:10960800043007EE903AF8EEE77A384667EE887A43
:10961800FDEEE77ACDED007ABDF80010FAF7C2FE4C
:10962800384619F061FDFEF7C8BB00BFC42B002007
:109638008C2E0020685F002088160308D0230020A5
:1096480098160308475F002004000020501D0020E2
:10965800BC1C00200AD7233C35850020546000201C
:10966800005E00203C2E002003082080D8840020C3
:10967800942E0020045E0020676666667C600020E9
:1096880058A08B412C5F0020022019F00BFACD4B1B
:10969800CD4ADB69323382FB0329DB17C3EB691937
:1096A8005FFA89F019F0D4F9C9F3072019F0D0F955
:1096B800032019F0F7F9C54B1B78D90740F17281DF
:1096C80021F058FCC24B9FEDC37AD3ED037A67EEC5
:1096D800877AFCEEE77ACDED007ABDF800300028F5
:1096E80000F0D982DFB24FEA1329384619F0B0F9F1
:1096F800484619F0ADF9DFF8109399F80430002BBB
:1097080040F020820DF118094946B34819F064F970
:10971800132019F0C7F9BDF91870F8B219F098F9C3
:10972800C7F3072019F094F91B2019F0BBF9BDF90C
:109738001A70F8B219F08CF9C7F3072019F088F9F4
:10974800232019F0AFF94E2019F082F9002019F002
:109758007FF94946A04819F03FF9122019F0A2F9FB
:10976800BDF91870F8B219F073F9C7F3072019F0AA
:109778006FF91A2019F096F9BDF91A70F8B219F0B4
:1097880067F9C7F3072019F063F9222019F08AF95D
:10979800452019F05DF9002019F05AF95E21D8F832
:1097A8000000F9F7FBFC94F86031FEF7D3BBC4F86E
:1097B800786183F80080FEF714BABB78DBB103F157
:1097C800FF3C5FFA8CFC0CF1010CBC44BE46002245
:1097D8001EF8013B534083EA0313DBB2120AD90097
:1097E80042EA0322F44581EA131382EA0302EFD125
:1097F800002A7FF4F1AC794BDFF810C2D3F800E00F
:10980800774B78491B68DEF83080774ACCF83830D7
:10981800764B0988CCF81810CCF868001168B3F8B2
:10982800C6029268CCF82810CCF84820CCF858002A
:10983800B8F1000F00F08F82D8F80430DEF840103D
:109848008B423BBFDEF80C205B1A5B1A9B18002B7F
:109858007EF434AADEF80030DFF8B4819B697046E4
:10986800022198470423F87888F8003015F08AFD1B
:1098780003232370FEF724BA02213868F9F782FC23
:1098880094F88031FEF7D9B910230422184606A9A6
:109898008DF81A808DF81B808DF81C808DF81D803E
:1098A8008DF818308DF8192019F014F884F88B8188
:1098B800FEF7EFB9A3785A09012A40F0CA8103F0EC
:1098C8000F0C13F0100300F0D681DFF84881E3781D
:1098D80094F804E0A4F8B20208EB03018EEA03004E
:1098E80084F890214346C4F8A882C4F8AC12A8F1C1
:1098F800070284F8B802A4F8B0E294F8B802DFF8D6
:10990800188186460CE012F8011BC4F8A8024245EB
:1099180081EA0E0E197007D2D4F8AC12D4F8A83226
:10992800994203F10100EED1424584F8B8E200F013
:109938006182127894F8B8329A4200F0CE812C4BAA
:10994800C4F8943200220133B4F8B012C4F8983243
:1099580084F8902101234FF6F672A4F89C1284F83B
:10996800943184F8A432A4F89E22FFF73EBA032764
:109978002049FCE4DBF800301F4A204903F4800347
:10998800834216BF114604270327E1E4154B1988C3
:10999800FFF7E6BB1A49C97800290CBF0421052145
:1099A800FEF77DBFDFF86090164BB9F80670A3FB91
:1099B8000737BF08F8B219F04BF8380A19F048F819
:1099C8009BE600BF1C2E00201F85EB51358500202B
:1099D800445E0020CDCC4C3E80969800984C0020E8
:1099E800BC1C0020005E0020045E0020501D0020EA
:1099F800E41E00208C160308881603088016030846
:109A080054600020CDCCCCCC7C600020CC0E002053
:109A18003D0F00205C1D0020581D0020DFF884A3A6
:109A2800102019F03FF8D54ADAF8003082FB0329F4
:109A3800DB17C3EB69195FFA89F019F009F8C9F364
:109A4800072019F005F8212019F02CF8DAF8002081
:109A5800CA4B83FB023AD3176421C3EB6A1301FB99
:109A68001323002BD8BF5B421BB2D8B218F0F0FF0B
:109A7800002018F0EDFFFEF743BA012238681A708B
:109A8800F9F784FB80463868F9F780FB18F07F0FF8
:109A98007EF4A7A88E287EF4A4A894F87431002B2D
:109AA8007EF4BBA8B64BC4F87C312D2384F88031F2
:109AB800FEF79EB8B4F99E12D4F898C294F89CE2C6
:109AC800501C02F00F0242F010020029B8BF42F009
:109AD80020028DF81820ACEB090282EA0E0E5FFA1C
:109AE8008EFE8DF8192084F8BA0284F8BBE20DF1D5
:109AF8001A02FFF7A2BBA3495A790B8803EB830329
:109B080003EB83034FEA830A1FFA8AFA002A00F05C
:109B180032819D4B1B681BB2029308F0EDFE029B3D
:109B2800019A40B2FEF796BA984904271FE4964670
:109B380092461146019203929146FEF799BB4FF067
:109B4800340861E4DFF860A29AF80020002A3FF4A4
:109B5800D9ADB4F868718B4B00921B883F01642122
:109B6800BFB201FB03235100B3FBF1F347EA03271C
:109B7800BFB2C3F303231F43062018F093FFF8B2C4
:109B880018F066FF380A18F063FFB4F868317D4AA8
:109B98007F491788009A01339BB293FBF2F002FBCE
:109BA8001033487AA4F86831012800F00E814B7B05
:109BB8006E2202FB07F7152297FBF2F7002B40F005
:109BC800FE803A2018F06EFFBFB24FF0640AB7FB70
:109BD800FAF293B2D8B20192009318F039FF009BC1
:109BE800180A18F035FF3B2018F05CFF019A0AFBB1
:109BF800127080B20A23053090FBF3F0C0B218F05F
:109C080027FF002018F024FFDFF87CA1282018F097
:109C180049FF0A23DAF8007097FBF3F7F8B218F057
:109C280017FFC7F3072018F013FF042018F03AFFB6
:109C3800B9F80630002B40F08680DAF8087087F310
:109C48001007F8B218F004FFC7F3072018F000FF58
:109C580058E5504B504AC4F89432591C012384F8F3
:109C6800900184F89401C4F89812C4F89C2284F8EE
:109C7800A432FFF7BAB894F89021002A3FF4B5A8A7
:109C880094F8B922013202F00F02624555D084F8E7
:109C98009031FFF7AAB8DBF80020D2067FF522AD95
:109CA800814622E54FF02408FFF7AEBB4B1CDBB220
:109CB800042B84F8BE324FEA01617FF4C5A9FFF78F
:109CC800C0B90199322018F005FEFFF706BB06ABB4
:109CD80001930DF11E07FFF7EFBA304BD4F8A82215
:109CE800C4F8AC224FF0000E03F52272114603F5BA
:109CF800C479C4F8982203F527707246C4F8A832CC
:109D0800C4F89CE2C4F8949284F890E1F6F738FA23
:109D1800013067D0D4F89432C4F898320123C4F8DB
:109D2800949284F8A432FFF760B84FF01008FFF758
:109D38006BBB4FF00808FFF767BBD4F8AC12D4F838
:109D4800A832174AD9E508F0D7FD18F081FE00209F
:109D580018F07EFED6E4DEF81C10DEF820309942BA
:109D68003BBFDEF80C205218CB1AD31A6FE54FF020
:109D78002008FFF749BB4FF0FF33CCE61F85EB51B6
:109D8800D05F0020005E0020045E002090160308CB
:109D9800345E0020E41E00200000F6FF5C1D002059
:109DA800531D0020BC1C0020425E002096469246AF
:109DB80011460192039202929146FEF759BABFB238
:109DC8009AF8003097FBF3F7FBE6392018F06AFEA3
:109DD800F8B218F03DFE380A18F03AFE14E791463A
:109DE800FEF746BAD4F894320222591CC4F89412E9
:109DF8001A708FE784F8B9C2FEF7F7BF0E4B924688
:109E0800B3F9003064200A46FEF724B99646914615
:109E1800FEF72EBA964692469146FEF729BA96461E
:109E2800924611469146FEF723BA96469246114647
:109E380001929146FEF71CBA045E002003680A7A74
:109E4800591C01601A70704738B50B4C23688BB1E8
:109E58005A68821A002A054604DA0CE05A68AA1AD7
:109E6800002A07DB9A68226018461A689047236818
:109E7800002BF3D138BD38BDF44B00200B4B00222A
:109E880010B4027203F5AA74042102E0072A09DC5F
:109E98009979890702D51979815401329C4203F1D5
:109EA8001403F3D15DF8044B704700BF9005030815
:109EB80010B40D4C04232146002200E08B7913F0E6
:109EC800010301F1140106D10132122AF6D10370FF
:109ED8005DF8044B704702EB820204EB82025DF8E6
:109EE800044B1379037070479005030830B40123BD
:109EF80030253324312132224570C4714171C2703A
:109F0800037083710371837030BC704770B54E68FD
:109F18000546304621F04EFB314604460246286885
:109F280024F055FB2A68131901333B212B60115586
:109F380070BD00BF08B516F0B5F8024B024ADA60EA
:109F4800FEE700BF00ED00E00400FA052DE9F04748
:109F58000569C3681D4028D00F4606464FF00048E3
:109F68004FF00009B5FA85F328FA03F2D2431B3BF8
:109F780032611540042B16D8DFE803F03129211986
:109F880003007B6A002B32D003F1FF3A1FFA8AFAEA
:109F9800C7F824903C6A34B1236820465146984754
:109FA8006468002CF8D1002DDCD1BDE8F087386852
:109FB800716B036889B29847002DD3D1F5E77868AB
:109FC800B16B036889B29847002DCBD1EDE7B8682B
:109FD800F16B036889B29847002DC3D1E5E7F868AB
:109FE800316C036889B29847002DBBD1DDE7F36A6D
:109FF8001FFA83FACEE700BFF0B5464B1A6883B064
:10A00800012351024449009358BF03F18053096862
:10A0180058BF0093D7005CBF43F0100300938E072E
:10A0280044BF43F0C60300934C0744BF43F0080302
:10A038000093080744BF43F020030093D105374934
:10A04800097848BF43F0006301F0EF0048BF009370
:10A0580008286D4651D00E294FD03148009B007812
:10A06800D70454BF43F0884343F0C843002843F45F
:10A0780000530CBF07200F20960648BF43F4807397
:10A08800540748BF43F4003343F4002452050094B6
:10A0980002D5244A1279A2BB182936D0019000278C
:10A0A800012639462846FCB2FAF7E6FB60B11E4B9A
:10A0B800002203F5D87103E08B420FD013F80C2C63
:10A0C800944203F10C03F7D10137242FE9D195E825
:10A0D8000300164B83E8030003B0F0BD7A0904F0CF
:10A0E8001F0455F8223006FA04F4013723EA040461
:10A0F800242F45F82240D4D1E9E743F48053009354
:10A10800ABE743F4C0130093C6E7009B43F06073CA
:10A118000093C3E72037002028690020543000202E
:10A1280024320020345E0020D0E702084C1C0020B6
:10A138002DE9F84F4E014FF0000B174D8146904620
:10A1480006F120075C46594628465FFA8BFAFAF76B
:10A1580093FBC0B1A64215D8A74213D900200F4AD5
:10A16800014604E00131242914D012F80C0C5045A2
:10A1780002F10C02F6D10A4B01EB410103EB81011C
:10A188004846C04701340BF1010BBBF1240FDAD16B
:10A19800BDE8F88F0021F3E74C1C0020D0E7020847
:10A1A800C4E7020800210A4A0B4604E00133242BC5
:10A1B8000BD012F80C1C884202F10C02F6D10548AB
:10A1C80003EB430300EB830070470020704700BF98
:10A1D800D8E70208C4E7020800210A4A0B4604E04F
:10A1E8000133242B0BD012F80C1C884202F10C020C
:10A1F800F6D1054803EB430300EB830070470020CA
:10A20800704700BFD0E70208C4E7020808B501217B
:10A218000220F9F775FC094B1B7803F00503052BA1
:10A2280008D000210120F9F76BFC00210846F9F756
:10A2380067FCFEE715F0E6FFF3E700BF042A0020FD
:10A24800022828BF022010B4084C094B207000EBEC
:10A25800C00200EB820207495DF8044B013003EBB2
:10A268004203C0B20B6017F093BA00BF985E00209B
:10A27800DE740020B05E002008B513F0D1F9F9F7BC
:10A288006DFEBDE8084013F0B3B900BF38B5434BC5
:10A298005A899989914224BF00225A81198ADA89F8
:10A2A800914224BF0022DA81DA7892B1072A10D0CD
:10A2B8003B4C3C48A27801210025062A0170997080
:10A2C800DD719D7152D92379DFED376A002B3CD1BE
:10A2D80038BDDA79002A4ED09A783248DFED326AF2
:10A2E8000178042A38BF042207EE902AB8EEE77AEC
:10A2F80007EE901A27EE267AF8EEE77A9A7067EE5C
:10A30800877A274CA2780025062A9D712BD8274BDF
:10A3180003EB8203D3ED006AF4EEE76AF1EE10FA7C
:10A3280010DDC6EE877AFDEEE77A17EE903A102B2D
:10A33800A8BF1023012BB8BF0123DBB28B4228BF73
:10A348000B4603702379002BC2D0013A032ABFD8E9
:10A35800B7EE000A80EE260A22F046F823889842D3
:10A3680038BF208038BDDFED106AD5E7DFED107A01
:10A37800B0EE677ACBE79A780A48DFED0E6A017883
:10A3880007EE102A07EE901AB8EEC77AF8EEE77AC9
:10A3980027EE267A67EE877AB3E700BFE0600020F1
:10A3A800FC310020585600206F120338C0EC020818
:10A3B8006F12833A6F12033938B50C4C0C4DAC420E
:10A3C80006D2616820461434F9F74CFDAC42F8D344
:10A3D800084B094C094818600025257015F0E6FC63
:10A3E800074B084A65701A6038BD00BF503F030824
:10A3F80060430308B05E0020985E0020DE740020F1
:10A40800FC860020B45E002008B5FFF7D5FF13F0E6
:10A4180007F9F9F7A3FDBDE8084013F0E9B800BF54
:10A42800F0B50C292BD8DFE801F06F2A2A2A4C2A2C
:10A438002A2A2B2A2A2A0700046AB2F80CE09788ED
:10A448001668674D24F480540462036A4468C1693D
:10A4580023F4005343EA0E3321F4E641A84243EAC9
:10A46800073341EA062100F0B58005F50065A842EA
:10A4780000F0B08092684460C16102640362F0BD7C
:10A48800046A96899588D2F800E0554F24F48074C0
:10A498000462036A4468C16923F4007343EA06232B
:10A4A80021F07301B84243EA052341EA0E017ED048
:10A4B8004C4DA8427BD092684460C161C26303627C
:10A4C800F0BD046A96899588D2F800E0444F24F0DC
:10A4D80010040462036A4468816923F0200321F0B0
:10A4E800807143EA061321F4E641B84243EA0513B2
:10A4F80041EA0E2148D03B4DA84245D092684460BD
:10A50800816182630362F0BD046A9389B2F804E052
:10A518001768334E24F001040462056A44688169AF
:10A5280043EA0E0321F4803125F002059BB221F0A5
:10A538007301B04243EA050341EA070114D0294DEB
:10A54800A84211D005F54065A8420DD005F58065F3
:10A55800A84209D005F58065A84205D092684460F4
:10A56800816142630362F0BDD689158A578A23F058
:10A57800080333433D43D68824F4407423F004038E
:10A58800ADB233432C43E9E7D589178AD68823F03F
:10A59800800343EA051324F44064558A23F04003FA
:10A5A80044EA870443EA061344EA8504A6E7D58902
:10A5B800178AD68823F4006343EA052324F4405419
:10A5C800558A23F4806344EA071443EA062344EADD
:10A5D800051470E7158A24F4804444EA851449E791
:10A5E800002C0140003401402DE9F84F4FF4A072CF
:10A5F80000218548854C864D864E874FDFF834828A
:10A60800DFF8349224F008F884488549DFF82CE212
:10A61800DFF82CC2002213588B4200F0D580B3F12A
:10A62800804F00F0D880AB4200F0DC80B34200F0ED
:10A63800DC80BB4200F0DC80734500F0DC806345C1
:10A6480000F0AD80434500F0D9804B4500F0D9803B
:10A65800DFF8F0A1534508BF4FF4802A00F0A1802D
:10A668001432B2F5B47FD6D1DFF8B0816D4F6E4D9C
:10A6780008F5B4764FF0030A4FF0020998F8043051
:10A688001C09013C052C03F00F0300F2818037F808
:10A69800140040FA03F2D2077AD54FF0010B0BFAF7
:10A6A80003F3013B184021F02FFC604B1B5D18445D
:10A6B80015EBC0046CD055F830305D4898F8081098
:10A6C80003F13842920A825C02F01F005209022A02
:10A6D8000BFA00FB71D0032A68D0012A05D14B4A36
:10A6E8004A4852694BEA02024261B4F804E0BEFAF1
:10A6F8008EF2C2F11F0292B2D00803EB800002F082
:10A708000702046A92004FF00F0C0CFA02FC24EACC
:10A718000C040462046A01FA02F222430024026271
:10A728004FF0010C224603E0102A04F102042FD056
:10A738000CFA02F030EA0E0102F10102F4D1D3F86A
:10A7480008B00AFA04F1C9430BEA010BC3F808B0D0
:10A75800D3F808B0C3F808B0B3F804B01FFA8BFBFD
:10A768002BEA00009880988880B298801868084082
:10A778001860D3F800B009FA04F040EA0B0018603A
:10A78800D868102A01EA0001D96004F10204CFD187
:10A7980008F1140846457FF471AFBDE8F88F4FF40F
:10A7A800005AA36943EA0A03A36159E7174A1748FD
:10A7B800D2694BEA0202C26197E7144A13489269C8
:10A7C8004BEA0202826190E7A3694FF4006A43EA08
:10A7D8000A03A36144E74FF0010AE36943EA0A0365
:10A7E800E3613DE74FF0020AF7E74FF0040AF4E7A8
:10A7F8004FF0100AF1E74FF0200AEEE74FF4803AE5
:10A80800CFE74FF4003ACCE7147300200010024061
:10A8180000040040000800400010004090050308B4
:10A82800002C014070050308A46F00207C05030874
:10A838008405030800400140004401400014004022
:10A84800003401400048014001490248FFF77EBB3F
:10A858002C7400200048014001490248FFF776BBEC
:10A86800DC7300200040014001490248FFF76EBB3D
:10A87800B47300200034014001490248FFF766BB69
:10A88800B47300200034014001490248FFF75EBB61
:10A898008C7300200008004001490248FFF756BBAE
:10A8A800647300200004004002494FF08040FFF725
:10A8B8004DBB00BF3C73002010B5064C064821462E
:10A8C800FFF744FB04F1F0010448BDE81040FFF72E
:10A8D8003DBB00BF14730020002C01400044014020
:10A8E80001490248FFF732BB14730020002C0140D5
:10A8F8002DE9F0410468574DA30AAB4200F085806A
:10A908005CD9554DAB426CD078D9544DAB4264D02C
:10A918000135AB4240F09A804FF49C7E0726477978
:10A928004FEA970C00297CD0B000634685190227AE
:10A93800D4F80C809F400CEB4503BFB2484D03F19F
:10A94800040C47EA080745F8231045F82C20E7606F
:10A95800EFF31181502282F31288821905EBC202AB
:10A968001369002B41D013620433821905EBC2022C
:10A97800576917B11F6053690433821905EBC20286
:10A98800976917B11F6093690433821905EBC202F6
:10A99800D76917B11F60D36904330027CAB21F6093
:10A9A80082F31188304405EBC000036A03BBE368F7
:10A9B8004FF6FE721340E360BDE8F0814A3DAB42BA
:10A9C8002BD00135AB4204D0B3F5801F21D0BDE8B0
:10A9D800F0814FF0980E0326A1E74FF4887E0626F3
:10A9E8009DE74FF0E80E052699E705EB0E03BCE757
:10A9F800E36843F00103E360BDE8F081033DAB4247
:10AA080026D14FF0C00E042689E74FF0200E00260D
:10AA180085E74FF0480E012681E74FF0700E0226B9
:10AA28007DE7BF08022306FA03F0BB40DB43E76873
:10AA38000B4D9BB23B4087190CEB470CE3600CF1C4
:10AA4800040345F82C1045F8232081E7BDE8F08180
:10AA5800BDE8F0814B0010005000100051001000BC
:10AA68001473002030B503685C4D18885C4CB4FB47
:10AA7800F2F20139013AAB4294B283B089B282B2A0
:10AA880066D05848834263D0B3F1804F60D0A0F5B8
:10AA9800983083425CD000F58060834258D0524899
:10AAA80083425BD000F5806083427DD022F44072FF
:10AAB80000F58C3092B283421A80D9621C850ED080
:10AAC800484A93420BD002F54062934207D002F500
:10AAD8008062934203D002F58062934201D1002242
:10AAE8001A8601225A611A883C4992B242F0010240
:10AAF8008B421A8062D0B3F1804F61D03B4A9342B7
:10AB080060D002F5806293425ED002F50062934203
:10AB18005CD002F5806293425AD002F5903293429B
:10AB280058D002F54062934256D002F580629342B3
:10AB38001ED002F58062934208BF092219D002A8EC
:10AB48004FF0012340F8043D1AF0A0F803B030BDDF
:10AB5800254822F07002834292B2A3D101201A80C4
:10AB6800D9621C8558611A8892B202431A80C5E7D7
:10AB780008221F4B03EBC20301A893F821408DF86C
:10AB88000440012300228DF805308DF807308DF838
:10AB980006201AF07BF81B2CD8D1164B019301A87C
:10ABA8001AF074F803B030BD01201A80D9621C85F0
:10ABB80058611A8892B202431A809CE70022D8E7AB
:10ABC8000122D6E70222D4E70322D2E70422D0E703
:10ABD8000522CEE70622CCE70722CAE7002C01406F
:10ABE80000A24A0400340140001000400004004064
:10ABF800C0EC020819010001204B98422DD0B0F199
:10AC0800804F2CD0A3F5943398422AD003F5806363
:10AC1800984228D003F50063984226D003F5806354
:10AC2800984224D003F59033984222D003F540632C
:10AC3800984220D003F58063984207D003F58063DB
:10AC4800984208BF092202D00020704708220C4B06
:10AC580003EBC20393F8200070470022F7E70122B4
:10AC6800F5E70222F3E70322F1E70422EFE70522E2
:10AC7800EDE70622EBE70722E9E700BF002C0140D9
:10AC8800C0EC02082DE9F04F013085B0C3B2039340
:10AC98008C4D8D4F8D4C8E4E0A230293DFF83492E3
:10ACA8001AF00AFA4FF4FA7A4FF0100C4FF47A704F
:10ACB800D9F80430C3F30803002B40F0C580EFF344
:10ACC8001183002B40F0C0802968A26800BF2B6860
:10ACD8009942F9D1D7F800E000FB0EF39B1AB3FBB9
:10ACE800FEF300FB01314FF0010E0191D9F8043059
:10ACF800C3F30803002B40F08B80EFF31183002B84
:10AD080040F086802B68A16800BF2A689342F9D179
:10AD1800D7F800B000FB0BF2521AB2FBFBF200FBB3
:10AD28000323019A9B1AB3F57A7FDFD3BAF1010A9C
:10AD3800BED1039B002B40F0C1804FF47A7ADFF834
:10AD4800949150464FF0100CD9F80430C3F308031F
:10AD5800002B40F09680EFF31183002B40F0918098
:10AD68002968A26800BF2B689942F9D1D7F800E09A
:10AD780000FB0EF39B1AB3FBFEF300FB01314FF00F
:10AD8800010E0191D9F80430C3F3080323BBEFF394
:10AD980011830BBB2B68A16800BF2A689342F9D1C5
:10ADA800D7F800B000FB0BF2521AB2FBFBF200FB23
:10ADB8000323019A9B1AB3F57A7FE3D3BAF1010A08
:10ADC800C2D1029B013B02937FF468AF414B424AD8
:10ADD800DA6005B0BDE8F08FEFF311888CF31288C4
:10ADE800A1682368DB0344BFC6F800E0A1682B68AC
:10ADF80032685FFA88F888F31188D7F800801A4417
:10AE080000FB08F35B1AB3FBF8F300FB0233D0E74F
:10AE1800EFF311888CF31288A1682368DB0344BF21
:10AE2800C6F800E0A1682B6832685FFA88F888F3F2
:10AE38001188D7F800801A4400FB08F35B1AB3FBAB
:10AE4800F8F300FB02336CE7EFF311828CF31288FE
:10AE5800D4F808E02368D90303D501233360D4F874
:10AE680008E02B683168D2B282F311883A68194435
:10AE780000FB02F3A3EB0E03B3FBF2F300FB01317B
:10AE880031E7EFF311828CF31288D4F808E02368D5
:10AE9800D90303D501233360D4F808E02B6831685F
:10AEA800D2B282F311883A68194400FB02F3A3EB8B
:10AEB8000E03B3FBF2F300FB013160E7184619F00B
:10AEC8005FFF3AE7047300200873002010E000E0F9
:10AED8000073002000ED00E00400FA052DE9F047BA
:10AEE800A84FA94E12F09CFBBE421ED2DFF8208369
:10AEF800DFF820934446258862197DB14A450DD272
:10AF0800052D0BD933886188C3F30B03994200F0F0
:10AF1800D880144625886219002DEFD17168304613
:10AF28001436F8F79FFFBE42E4D3984A5378022BB1
:10AF380040F2EC8000239649537013789548022B11
:10AF4800016000F2DF8003EBC301934A03EB810346
:10AF580002EB4303914C1846236014F027FF904AF4
:10AF68001378A3F1170102290FD98E4911F833007C
:10AF7800002840F0D180D8000144497829B18A4995
:10AF880011F83330002B00F0F580884B9A78042AAA
:10AF980000F0E78032B91A88B2F5F07F84BF4FF429
:10AFA800F0721A80824D834A2B681A40002A00F0FA
:10AFB800E480DE0700F1D080580400F1C88019074A
:10AFC80000F1C0809A0100F1B7809B0400F1AD80C8
:10AFD80023689A8CD98C914224BF00229A84FFF767
:10AFE80055F910F0EDF910B9734815F075FD20F01A
:10AFF8000DF800213022714823F00EFB704B2668B3
:10B0080003F1500102E00433994279D01A78002AFA
:10B01800F9D19C78D8788442F5D26A496A4B91F87C
:10B0280000E06A486A4D1C6B6A4B2860C827642197
:10B0380011FB0E71DFF8E0E15960674F30F8041C2E
:10B04800664DAEF8001000219960D9601961596108
:10B058009961D96183F8201083F821103A702E6025
:10B068000CB10FF06FFC5E4B9FED5E5A1B885E4A79
:10B078009FED5E6A55795E4C5E495F48086006EE52
:10B08800903AF8EEE66A1388C5EE265A07EE103AAB
:10B0980053881279C4ED005A07EE903AB8EEC77A91
:10B0A800564BF8EEE77A1D725A7227EE067A67EE6B
:10B0B800867ABDE8F04783ED017AC3ED007A12F095
:10B0C80097BA63799B077FF424AF716894F804A05A
:10B0D8003046F8F7C7FE3388BAEB133F0BD17388B5
:10B0E8007068AA1FC3F30B039A4204F10601A8BFB4
:10B0F8001A4623F06CFA1436BE42FFF4FBAE14E78E
:10B1080001228AE700231370234B23E7204903EB2E
:10B11800430301EB830110E7D8000D186D68002D7B
:10B128007FF42AAF1725157026E73548F8F7D0FEC3
:10B138004020F8F7CDFE4BE746F20900F8F7C8FEC5
:10B148002B6842E72F48F8F7C3FE2B683AE72E48EA
:10B15800F8F7BEFE2B6832E72C48F8F7B9FE2B68E3
:10B168002AE71A8BB2F57A7FBFF41CAF4FF47A72D4
:10B178001A8317E71823137007E743F400532B606B
:10B1880017E700BF60430308503F0308985E00209C
:10B19800B45E0020FC860020DE740020B05E002033
:10B1A80054300020F809030888010308FC31002006
:10B1B800442C002009600002587400204C22002012
:10B1C80058300020802D0020D85E0020384C002008
:10B1D800BC8500205460002044000020802200200C
:10B1E800C81C0020C0C9FB488C21002017B7D138E3
:10B1F800CC1C0020242C00203661023D002C0020AD
:10B2080009400002016000020920000208600002F3
:10B2180007F00308000004080C31002008B512F0FC
:10B22800FFF9F8F79BFE12F0E3F9FFF757FE01204C
:10B23800BDE8084016F0ACBA2DE9F04F013085B0F2
:10B24800C3B203930B4602918B4C8C4E002B00F03B
:10B2580099808B4D8B4FDFF8309219F02DFF4FF40A
:10B26800FA7A4FF0100C4FF47A70D9F80430C3F31F
:10B278000803002B40F0DE80EFF31183002B40F031
:10B28800D9802968A26800BF2B689942F9D1D7F8FC
:10B2980000E000FB0EF39B1AB3FBFEF300FB013149
:10B2A8004FF0010E0191D9F80430C3F30803002BC5
:10B2B80040F08780EFF31183002B40F082802B68E9
:10B2C800A16800BF2A689342F9D1D7F800B000FB03
:10B2D8000BF2521AB2FBFBF200FB0323019A9B1AF2
:10B2E800B3F57A7FDFD3BAF1010ABED1039B002BF5
:10B2F80040F0BD804FF47A7ADFF88C9150464FF0D9
:10B30800100CD9F80430C3F30803002B75D1EFF300
:10B318001183002B71D12968A26800BF2B6899425C
:10B32800F9D1D7F800E000FB0EF39B1AB3FBFEF34C
:10B3380000FB01314FF0010E0191D9F80430C3F33D
:10B34800080313BBEFF31183FBB92B68A16800BF97
:10B358002A689342F9D1D7F800B000FB0BF2521AD1
:10B36800B2FBFBF200FB0323019A9B1AB3F57A7F29
:10B37800E3D3BAF1010AC4D1029B013B0293002B2B
:10B388007FF467AF05B0BDE8F08FEFF311888CF359
:10B398001288A1682368DB0344BFC6F800E0A168EF
:10B3A8002B6832685FFA88F888F31188D7F800802C
:10B3B8001A4400FB08F35B1AB3FBF8F300FB0233F3
:10B3C800D2E7EFF311888CF31288A1682368DB03B6
:10B3D80044BFC6F800E0A1682B6832685FFA88F8B5
:10B3E80088F31188D7F800801A4400FB08F35B1A29
:10B3F800B3FBF8F300FB023370E7EFF311828CF331
:10B408001288D4F808E02368D90303D501233360F0
:10B41800D4F808E02B683168D2B282F311883A6810
:10B42800194400FB02F3A3EB0E03B3FBF2F300FB9A
:10B4380001317FE7EFF311828CF31288D4F808E02A
:10B448002368D90303D501233360D4F808E02B68B7
:10B458003168D2B282F311883A68194400FB02F3CA
:10B46800A3EB0E03B3FBF2F300FB013118E7184618
:10B4780019F086FC3EE700BF10E000E000730020F2
:10B48800047300200873002000ED00E0204B5B6887
:10B49800C3F3080330B4BBB9EFF31183A3B91D4B51
:10B4A8001D4C1868A16800BF1A689042F9D11B4B5F
:10B4B8001C684FF47A7202FB04F3591AB1FBF4F1D9
:10B4C80030BC02FB00107047EFF31182102383F3A6
:10B4D800128811498C680B6813F4803F104B02D016
:10B4E800012018608C680B49D2B20D68186882F385
:10B4F80011880A4B19684FF47A72284402FB01F349
:10B508001B1B30BCB3FBF1F302FB0030704700BFDC
:10B5180000ED00E00473002010E000E00873002054
:10B52800007300202DE9F84F8046FFF7AFFF254E46
:10B538002549DFF8A0E0254A254D844610274FF419
:10B548007A740120DEF80430C3F30803D3B9EFF3AB
:10B558001183BBB90B68D2F808A000BFD1F80090DE
:10B568004B45F7D1D6F800B004FB0BF9A9EB0A0953
:10B57800B9FBFBF904FB0393A3EB0C034345E1D3AD
:10B58800BDE8F88FEFF3118A87F31288D2F808B074
:10B598001368DB0344BF2860D2F808B00B68D5F8FD
:10B5A80000905FFA8AFA8AF31188D6F800A09944C5
:10B5B80004FB0AF3A3EB0B03B3FBFAF304FB093315
:10B5C800DAE700BF087300200473002010E000E0F1
:10B5D8000073002000ED00E02DE9F04FDFF830C1E6
:10B5E800474A4849484E494D8046102718F1FF38C8
:10B5F800C0F08480DCF80430C3F30803002B5CD16E
:10B60800EFF31183002B58D10B68946800BF0868CA
:10B618008342F9D1D6F800904FF47A7000FB09FE06
:10B62800AEEB040EBEFBF9FE00FB03EEDCF80430C3
:10B63800C3F308034FF47A740120FBB9EFF31183C5
:10B64800E3B90B68D2F808A000BFD1F800904B45C9
:10B65800F7D1D6F800B004FB0BF9A9EB0A09B9FB3E
:10B66800FBF904FB0393A3EB0E03B3F57A7FBDD27A
:10B67800DCF80430C3F30803002BDFD0EFF3118AA2
:10B6880087F31288D2F808B01368DB0344BF286038
:10B69800D2F808B00B68D5F800905FFA8AFA8AF3F6
:10B6A8001188D6F800A0994404FB0AF3A3EB0B0316
:10B6B800B3FBFAF304FB0933D5E7EFF3118487F3FF
:10B6C8001288D2F808901368D80303D501232B6099
:10B6D800D2F808900B682868E4B284F31188D6F889
:10B6E80000A04FF47A7400EB030E04FB0AF3A3EBFB
:10B6F8000903B3FBFAF304FB0E3E97E7BDE8F08FAE
:10B7080010E000E00473002008730020007300209C
:10B7180000ED00E030B4EFF31183102282F31288B9
:10B728000649074C0A680748013200250A60256067
:10B73800DBB2026883F3118830BC704704730020C1
:10B748000073002010E000E00F4B1B88014643B94E
:10B758000E4B0F4A1B7810680BB981F00101F8F7FE
:10B76800C5B90C4B5A691AB118B91A6810605874DF
:10B778007047094A18681188084A92FBF1F20121BA
:10B7880002605974704700BFDC720020DE7200202E
:10B79800E0720020E4720020FC72002020A1070063
:10B7A8001D4B70B55C68236D226BDD69C2B1636B9C
:10B7B8002BB12B0702D5236D08221A6270BD2A0609
:10B7C800F7D5A26A616A8A421FD0511CA069A1629A
:10B7D800825C2069266D81423285EAD3A362E8E75C
:10B7E800A906E4D5E26A1AB1988C80B29047DEE7E0
:10B7F800E1699B8C6069DBB24E1CE6614354E169E8
:10B80800E368994228BFE261D1E7226D136823F00B
:10B8180080031360CDE700BF082A00201D4B70B5D8
:10B828001C68236D226BDD69C2B1636B2BB12B07DA
:10B8380002D5236D08221A6270BD2A06F7D5A26ABE
:10B84800616A8A421FD0511CA069A162825C20698A
:10B85800266D81423285EAD3A362E8E7A906E4D5DA
:10B86800E26A1AB1988C80B29047DEE7E1699B8C56
:10B878006069DBB24E1CE6614354E169E3689942B2
:10B8880028BFE261D1E7226D136823F080031360BB
:10B89800CDE700BF082A00202DE9F04F9A4A9B49BE
:10B8A800137895B00446099000F59C4020300C9020
:10B8B8000860002B00F07C84954909688C4240F2AE
:10B8C80096809449059109689348944CDFF888B2AA
:10B8D8000391013B137001F4805302900893002BED
:10B8E80040F09480029B5B7D002B40F06283039BB9
:10B8F8001E0400F11186039BDD050BD5099A884BC0
:10B90800DFF858A29A429AF8022000F2D287002A59
:10B9180040F0D387834B0493834D039B13F48057E4
:10B9280040F06783029BBBF906605B8B9E42B4BF05
:10B93800002601267D4B1B6813F0805373D0049AB0
:10B94800127812F0010275D002987949808C91ED35
:10B95800037A07EE900AF8EEE77AB4EEE77AF1EEAA
:10B9680010FA80F2B286002E69D194F8A41000294A
:10B9780065D170487049006890F830004FF0000EAB
:10B98800C1F800E0C1F804E0C1F808E06B490028FC
:10B9980056D10870002A57D0039AD10654D5684A60
:10B9A8001278D20650D4002F4ED1002B4CD1039BD5
:10B9B8005B0249D495F800C0BCF1000F01F0638523
:10B9C800604B9B78002E41F08E853BB15E4A5F4B01
:10B9D80012681B689B1A002BC1F2A885102015F06D
:10B9E800F5FD012384F8A53095F800C02EE0494BF9
:10B9F80005931B680393484A484C029203F480530A
:10BA0800DFF854B10893002B3FF46CAF002147488E
:10BA1800F8F732FF00287FF465AF08F047FC059B74
:10BA28001B6803935EE7039A500288D4049A12783D
:10BA380002F00102002184F8A410002E99D03F4999
:10BA480001200870002AA7D195F800C0029ABBF916
:10BA580000E0508B918BBBF902208645CCBF802734
:10BA6800002747F040038E45A8BF3B469B0843F09C
:10BA780080078242C8BF3B4643F040078A42B4BFB2
:10BA88003A461A469208BBF904E0BBF9067042F040
:10BA980080038645C8BF1A4642F040038E45A8BFBA
:10BAA80013469B0843F080028742D4BF18461046CD
:10BAB80040F0400294F8A6308F42ACBF01461146D0
:10BAC8008B4200F01884002384F8A61084F8A7306D
:10BAD800BCF1000F00F0A685059B1D4A1B68039268
:10BAE80003F00403002B40F00B830DF14808194DB7
:10BAF8000023C8F8043005F15009129340F6330AC0
:10BB0800192740F283362EE0484C0020D84B0020FD
:10BB1800444C002020370020F03600209C210020D3
:10BB2800404B4C0035850020440000208C2E00201E
:10BB3800445E0020B05E0020002E0020FC23002080
:10BB4800942E0020301D0020047300209C2A002021
:10BB58002869002058300020BC8300205460002051
:10BB680004354D4520D0AA78EB789A4217FB02603D
:10BB7800F6D26978043117FB03623BF9113053455B
:10BB8800A8BF5346B3F5617FB8BF4FF461739842BD
:10BB9800E6DA9A42E4DB29782329E1D840460435DD
:10BBA800F8F75AFE4D45DED1AB4B98E803001E78F6
:10BBB800AA4B83E80300002E00F032820121A74837
:10BBC800F8F75AFE002840F00C81059B1B68DC053D
:10BBD80000F10281A24C23881DB225F00105AFB205
:10BBE800BB42278000F0FB839E4D02260F204FF0BA
:10BBF80014094FF0FF082E7085F8019085F802802F
:10BC080015F0E4FC314695482788F8F735FE0028FA
:10BC180040F09B8727F002039BB2BB4223800AD0E7
:10BC2800904B1421FF2202250F201D7059709A7025
:10BC380015F0CCFC2788DFF858A28B4B9AF8001037
:10BC480002935868BB0708BF81F00201C1F34001A5
:10BC5800F7F74CFF039B1B6813F00A0F24D005214C
:10BC68007E48F8F709FE002800F0C78425886F078A
:10BC780040F1ED8679480621F8F7FEFD002800F02E
:10BC8800A9846E0640F1008707217448F8F7F4FD8F
:10BC980050B1764B764AB3F90430764982FB0302F9
:10BCA800DB17C3EBA2030B800C216C48F8F7E4FD0B
:10BCB8002288002800F0B18042F480739A422380E1
:10BCC80009D0684B02251421FF220F201D705970DE
:10BCD8009A7015F07BFC684B1B78082B00F0A98044
:10BCE8000E2B00F0A680059B1B685D0542D5634BB3
:10BCF8001B79002B58D014215848F8F7BDFD0028AF
:10BD080056D117F033FA012015F0B6FB90B3DFF8DF
:10BD1800848100254FF0CC0902E0DDB2022D29D83C
:10BD280009FB05F76B1C58F80760002EF5D1C3789E
:10BD3800534A90F9020052F82330019603220092E8
:10BD48000121324614F0EEFE034605EB450000EBF8
:10BD58000010059353B1314608EB8000CC2222F045
:10BD68005BFC059B48F807300135EDB21AF054F832
:10BD78000028D3D1049B1B78D80740F18D80414916
:10BD8800414A01230B701370029B9AF8001018683F
:10BD980001F00101F7F7AAFE039B1B685B0700F19E
:10BDA800EB8015B0BDE8F08F049B1B78D907A8D5A8
:10BDB8003C2010F017F90028DCD007F069FD3C2082
:10BDC80010F0BCF80028D5D007F062FD3C2010F038
:10BDD800B5F80028F1D1CDE72C4BDB78002B3FF4E8
:10BDE800F9AE039B1B6898077FF5F4AE1C4C2788B7
:10BDF800F9073FF50FAF47F001039F4223803FF457
:10BE080009AF184B1421FF2202250F201D7059700D
:10BE18009A7015F0DBFB2788FCE622F480739BB24E
:10BE28009A4223807FF44DAF134B1B78082B7FF485
:10BE380057AF228822F040039BB29A4223803FF4F6
:10BE480052AF084B02251421FF220F201D70597094
:10BE58009A7015F0BBFB46E7755E00208C2E00201B
:10BE6800D02300208C2D0020D07200202C5F0020D1
:10BE780067666666A21C002054300020345E0020ED
:10BE88007803030836850020D01C00205460002069
:10BE9800CC720020E8770020AA4B93F80090B9F103
:10BEA800000F5FD1DFF80083A74F18F8030C3E7826
:10BEB8004146A8F103050AF0C3F8002800F0D4822F
:10BEC800002E40F0268305F1080168790AF0B8F8D9
:10BED800002841F0DB819D49A87A0AF0B1F80028D2
:10BEE80000F0D582022E41F0D5819949E87B0AF00D
:10BEF800A7F8002841F0B1819649287D0AF0A0F8FA
:10BF0800002800F0D582042E41F0AB819249687E6A
:10BF18000AF096F8002841F0B1819049A87F0AF00C
:10BF28008FF8002800F0D582062E41F0AB818C49AD
:10BF380095F823000AF084F8002840F0EE86894935
:10BF480095F828000AF07CF8002800F0D582082E21
:10BF580040F0F986844995F82D000AF071F8002818
:10BF680040F0D582814B01221A701FF031FA039BF1
:10BF78001B685B077FF515AF03200AF08BF80028D4
:10BF880000F0F785238813F008047FF40AAF08202F
:10BF980015F02EFC7648774D7749784A784BBBF8F0
:10BFA800066000682E80086014601C6015B0BDE84B
:10BFB800F08F029A013BD27D3BF91330002A40F002
:10BFC8004A83A3F57A73B3F57A7FA8BF4FF47A73DF
:10BFD80023EAE37307EE903A9FED6A7AF8EEE77A80
:10BFE80067EE877A684AFCEEE77A17EE903A138094
:10BFF80081E41D216548F8F73FFC00287FF492ACE6
:10C00800634A029BD2881B8BBBF90660991A8E4241
:10C0180040F3358613449E42B4BF0026012689E4C6
:10C02800DFF888915B4F09F15A054FF0010849463E
:10C0380019F8010C0AF004F8F8B199F8040099F815
:10C04800023099F803E000EB400104EB8101013B69
:10C05800D1F8B42003EB43033B4493420DD094F84A
:10C06800E02081F8B0E008FA00F022EA0000C1F808
:10C07800B430C1F8B86084F8E00009F10609A945B0
:10C08800D5D14549454A464B0968D2F8009093F8FE
:10C0980000A0444D069100266B685BB31F784FB330
:10C0A800AA68A9EB0202002A0ADB94F8E020012121
:10C0B800B14022EA010209F5FA7184F8E020A9608A
:10C0C800BAF1000F16D02A7859780432D2B2002972
:10C0D80040F0008302993BF91220098B01F1C80056
:10C0E800824240F3A08594F8E0209B783241D10742
:10C0F80040F102860136042E05F10C05CCD15DE530
:10C1080094F8AB3053B1049B1B78D80706D5029B33
:10C11800BBF906205B8B9A4200F3E08511211B488E
:10C12800F8F7AAFB002800F0B78294F8AE302BB9D4
:10C1380094F8A93013B93223A4F8AC30012384F859
:10C14800AE30D2E436850020060000204B2D0020BA
:10C15800502D0020552D00205A2D00205F2D002045
:10C16800642D0020692D00206E2D0020D01C002099
:10C17800BC1C0020AC1C0020B81C0020B01C0020F7
:10C18800A81C0020AAF1823F3C2E00208C2E002003
:10C19800645700202CED0208FC8600200473002060
:10C1A800786000204C220020412D0020592C0020CE
:10C1B800994C9A4B26780293994F002E00F0618291
:10C1C800B6B1DFF89492DFF894B2DFF85482CA4629
:10C1D8000025072D4046E9B27B6841F3E780984780
:10C1E80000B20135AE422BF8020F0AF1040AF0D171
:10C1F8008C4B05931A4609998B4B12680392A3FB43
:10C20800013E42F2010313404FEA9E1E079300F0DD
:10C2180034828648864A874B007887490690127888
:10C228001A70069B08702BB1824B93F800B08BF004
:10C2380001030693814A0299127838781090B1F870
:10C248002680088D91F822C00B92098B0B9A1191C8
:10C2580094F829107A4B0E9008461146A3FB011357
:10C268005B0803EB4303D31ADBB20D93039B2578DA
:10C27800744EDFF8ECB1DFF8EC91CDF810800F22A6
:10C288000CF1040C03F4805384F828200A945FFA14
:10C298008CFC109C0F92AA460893002180461097A8
:10C2A8002DB9A44599BFE2466546A2462546A9424E
:10C2B80080F29082069B002B00F04882624B049823
:10C2C80033F9112097B287424FEA410303D30E98FE
:10C2D800874240F2138259F82120964580F0408227
:10C2E8003BF90320079F002F40F010822BF8032012
:10C2F80001310636D4E794F8A790B9F1F90F00F2A6
:10C30800DD8109F101095FFA89F984F8A79084F8B9
:10C31800A610BCF1000F00F08681B9F1140F7FF46C
:10C32800DBAB5F2940F09281049E337813F0010360
:10C3380000F04F8707F0BAFF337803F00103002BB2
:10C348007FF4CAAB94F8A620572A00F0CD86059B47
:10C358001B6813F0040302D05A2A00F0F8845D2AFF
:10C3680000F028875B2A00F030875E2A00F0CA8434
:10C37800562A00F093872B782BB16F2A00F09D87FF
:10C38800324B00211960972A00F09B87A72A00F0FA
:10C3980098840021BB2A129100F0D787B72A00F0B1
:10C3A800B487BE2A00F0D487BD2A00F0D387792A43
:10C3B80000F0E9877A2A00F0DF879E2A00F0D58707
:10C3C8009D2A00F0CA87AE2A01F05580AD2A7FF475
:10C3D80083ABFF2100201DF0D6FAFFF77DBB0221B9
:10C3E8001B48F8F749FA00283FF414AC2580BA072F
:10C3F8003FF521AC47F00203BB4223803FF41BAC5E
:10C40800144B02201421FF2218700F2059709A70C3
:10C4180015F0DCF827880EE49C210020F036002077
:10C42800345F002020370020D34D6210B44B002029
:10C43800A0010020A101002078600020494C0020C4
:10C44800ABAAAAAAC8210020A0210020A02A002067
:10C458008C2E00208C2D0020B04C00209E21002026
:10C46800BC8300204C4C002008F10501687909F0D4
:10C47800E7FD00283FF42FAD012E40F0078705F1B6
:10C488000D01A87A09F0DCFD002840F00387C049B7
:10C49800E87B09F0D5FD00283FF42EAD032E40F0CF
:10C4A800DC86BC49287D09F0CBFD002840F0D98600
:10C4B800B949687E09F0C4FD00283FF42EAD052E69
:10C4C80040F0DC86B549A87F09F0BAFD002840F0A5
:10C4D800D986B34995F8230009F0B2FD00283FF446
:10C4E8002EAD072E40F01984AE4995F8280009F0C2
:10C4F800A7FD002840F02784AB4995F82D0009F0E6
:10C508009FFD00283FF42EAD092E3FF42BAD4FF0D0
:10C5180009094B4600F004BCD4F88C30099AD31AA8
:10C52800002BFFF6E8A9A14A94F89030517CA04A64
:10C53800029D32F811200C98A97DC4F88C000133B3
:10C5480003F00F0384F89030234492B292FBF1F287
:10C5580083F8942094F8940094F8951094F8962011
:10C5680094F8973001440A4494F8980094F8991084
:10C578001344184494F89A2094F89B3001440A44D0
:10C5880094F89C0094F89D101344184494F89E2045
:10C5980094F89F3001440A4494F8A00094F8A1103C
:10C5A8001344184494F8A23094F8A32001440B448F
:10C5B8001A4442F30B12642AE97DA8BF642213B21D
:10C5C80009B1C2F1640307EE903A9FED7A7AF8EE6A
:10C5D800E77A05E525F040039BB2AB4223803FF4A0
:10C5E80053AB754B02251421FF220F201D70597083
:10C5F8009A7014F0EBFFFFF747BB238823F004057C
:10C60800ADB2AB4225803FF435AB6B4B022514210C
:10C61800FF220F201D7059709A7014F0D7FF2588DB
:10C62800FFF728BBE14600216448F8F725F9B8B1BF
:10C63800002384F8A83007F0B5FC94F8A730142B31
:10C648007FF44AAA2B78002B40F07C87049B1B7848
:10C6580003F0010373E6C3F53B6308331BB2B0E490
:10C66800049B574A1B781060DF0700F11885B9F161
:10C67800140F3FF467AEFFF72FBA524B1B7806939F
:10C68800D1E593F822303E780433DBB2B3428EBF53
:10C69800267023701E4693E594F8A930002B3FF4CA
:10C6A80024AA049B1B7813F001037FF41EAA01221D
:10C6B80084F8A93084F8AA20FFF717BA84F8A630BE
:10C6C800BCF1000FAFD0FFF707BA012184F8A4101E
:10C6D800FFF7B5B9012900F0228594F8E02001237D
:10C6E800B34001361343042E84F8E03005F10C05FD
:10C6F8007FF4D2ACFFF762BA1A464B000EF5967774
:10C7080049F82170079F002F3FF4F0AD0D985F188E
:10C7180007440A9800EB4707BA85B8F1000F03D120
:10C728000B9802287FF6E2ADB6F802803288B78807
:10C7380042441744244A3FB282FB07022348A2EB33
:10C74800E772C75212B24FF00108CFE5049B002BE5
:10C75800D2D059F8212096454FEA4103FFF4C0ADE5
:10C768001B4A1B48D25CC718002A00F09581022A90
:10C7780040F05E817A7802EB820202EB820202F2DA
:10C78800EE2292B2032940F38B8012B2AAE500BFD1
:10C79800502D0020552D00205A2D00205F2D0020FF
:10C7A800642D0020692D00206E2D00204872002085
:10C7B8006472002014AE23418C2D00208C2E0020A2
:10C7C800A02A0020786000205655555510220020D8
:10C7D800E44C00200F990A9CB64B109F84F800A0E7
:10C7E8000F2942460CBF0122002284F8298084F8D0
:10C7F80028101A7006D11B21AF48F8F73DF8002819
:10C8080000F0CA84AD48AE4B82681968AD4BC16070
:10C818008A1A012119704368AB4E9A42029A317004
:10C8280088BF002392F8226088BF80F82130089BD7
:10C838003878B2F826C0B2F818E00436F6B2002B01
:10C8480000F05A818642A14A40F2CB81A04E174699
:10C8580000210DB982460546A94218DA12F81130AE
:10C8680083B1022B0CD17B7803EB830303EB8303A7
:10C8780003F2EE239BB226F8023B01310237E8E7C8
:10C888003388F8E7CBB2032BFAD87346F3E784F87A
:10C8980000A00B9B8F4A01331370089BFFF71FB84A
:10C8A800012000FA01F70F9820EA070012B20F9052
:10C8B80018E512B901228AF80220874B04931D78E3
:10C8C8009AF8218005F001031B20039309F0E2FB8D
:10C8D800B8F1010F079000F0D58105F00203069327
:10C8E8009AF820207D4DDFF80C927D4E744F052A72
:10C8F80000F29580DFE802F08579032F3E51B8F108
:10C90800010F04BF05238AF82030039B002B00F099
:10C918009C80029B3868B3F91810B9F802300022DD
:10C9280061F30F0263F31F42002361F30F0361F306
:10C938001F43DAF81410CBF804208842CBF80030F3
:10C9480040F222810323069347F230520323CAF8A8
:10C958001C208AF82030338843F00203338007F024
:10C96800A5FC3A68DAF81C3013440422CAF81830D7
:10C978008AF82020B8F1010F40F020843B68DAF8EB
:10C9880018209A424BD2287818B909F083FB00285E
:10C9980045D1338823F0020333803A68B9F806306A
:10C9A800642101FB03234FF4806000228AF82020D1
:10C9B8008AF80320CAF8103014F002FF9AF82020F1
:10C9C80095E71EF0D7FA012800F03D84079B002B5D
:10C9D80040F05B81B8F1010F21D03B68DAF81020F4
:10C9E8009A4228D301238AF82030B8F1010FD4D015
:10C9F80099F80830012B1ED00BF024FE9AF820205D
:10CA080075E7039B002BDCD1079B4FF48060002B5C
:10CA180000F0AC8014F0ECFE0022CAF81020069B4F
:10CA2800002B40F0AD80059B1B680393FEF776BF93
:10CA38003BF80320A6E60BF005FE032240F6B833C8
:10CA48008AF82020CAF81C3085E73B687CE745F067
:10CA580004039D4223800AD0224B02251421FF2281
:10CA68000F201D7059709A7014F0B0FD25881E4B68
:10CA78001E4AB3F904301E4982FB0302DB17C3EBDD
:10CA8800A2030B80FFF7F6B845F04003AB422380C2
:10CA98007FF4A7ADFFF7F8B8CAB2022A40F2FC82C9
:10CAA800032AC5D1119A0898049F002808BF3A465E
:10CAB80068E600BF796000208C2E002054600020BA
:10CAC80004730020A0010020A1010020E44C0020F4
:10CAD800BC830020494C00203585002044000020FC
:10CAE8003A4D00208C2D00202C5F0020676666667A
:10CAF800981C0020802D002086421946B04A4BD849
:10CB0800B04817460DB9B24635468D427FF7BFAEDD
:10CB180012F8113083B1022B0CD17B7803EB83031D
:10CB280003EB830303F2EE239BB220F8023B0131AF
:10CB38000237E7E70388F8E7CBB2022B03D9032BC8
:10CB4800F8D16346F1E77346EFE727F001039BB29C
:10CB5800BB4223803FF44BAC0F202E7085F8019028
:10CB680085F8028014F032FD278840E414F028FE8E
:10CB780052E7082014F024FEFFF713B903230693A5
:10CB8800069814F023FD4EE7B8F1010FF6D1032300
:10CB98009AF820200693AAE68A4E17460DB98246CF
:10CBA8000546A942BFF673AE12F8113083B1022BC5
:10CBB8000CD17B7803EB830303EB830303F2EE23AF
:10CBC8009BB226F8023B01310237E7E73388F8E7E2
:10CBD800CBB2022B03D9032BF8D16346F1E7734696
:10CBE800EFE77848174600210DB9B24635468D4221
:10CBF8007FF74DAE12F8113083B1022B0CD17B7840
:10CC080003EB830303EB830303F2EE239BB220F8C9
:10CC1800023B01310237E7E70388F8E7CBB2032B81
:10CC2800FAD87346F3E7C8398A423DDA94F8E02027
:10CC38009B783241D2073FF55DAAC3F10008012075
:10CC480014F0A6FD7A1E162A00F2E780DFE812F03B
:10CC5800D801EC01C101390100021102AE019B01AA
:10CC6800860171015C01E500390149011102AE013B
:10CC78009B0125011101FD00E800A300D200012657
:10CC8800FEF758BE002306932AE699F80430002BD5
:10CC98003FF4A0AE0BF0D6FC03224FF47A738AF867
:10CCA8002020CAF81C3056E694F8E0300122B24041
:10CCB80023EA020309F5FA7284F8E030AA60FFF764
:10CCC80019BA4149059B0A781B6842F004020A70A8
:10CCD80003F004033D4A0392FEF704BF00213C48D9
:10CCE800F7F7CAFD00287FF419AA322384F8AB00AD
:10CCF800A4F8AC30FFF712BA9846002B0CBF0120FD
:10CD080002209DE7334B02220320334D33492A701A
:10CD18000B6014F03DFDFEF7DFBE4FF007094B46F0
:10CD280003EB83031D4487F80090A97868781BF00B
:10CD38006DFA049B2A4A1B7801211170DA077FF5E6
:10CD480014A9FFF721B84FF008094B46E8E794F813
:10CD5800A920002A40F0AD8394F8AB2082F00102AC
:10CD680084F8AB20002A40F09F831E49096811F41B
:10CD7800003104D01C490979002940F0DE830A46B5
:10CD88001A48855C0D2D02F10C0200F05B8301311D
:10CD98001529F6D19EE7D4F8E400154B90F83B101E
:10CDA8009A784144FE29A8BFFE2121EAE17180F862
:10CDB8003B10002A40F0B48312F02AFD8DE400BF36
:10CDC800E44C0020BC830020942E00202869002019
:10CDD8008C2E002072750020985E0020B05E002026
:10CDE800D01C0020502C00207C60002074F2020827
:10CDF800F1750020D4F8E400B74B90F83A109A780F
:10CE080041446429A8BF642121EAE17180F83A10FD
:10CE1800002AD1D017201EF0DFF8D4F8E400CBE7C1
:10CE2800069AAD4B51784144B1F5967FA8BF4FF4AF
:10CE3800967121EAE17151709B78002BEDD0152095
:10CE48001EF0CAF8D4F8E400B6E7D4F8E400817814
:10CE5800A14B4144C829A8BFC82121EAE1718170CA
:10CE68009B78002BA8D014201EF0B6F8D4F8E40064
:10CE7800A2E7D4F8E4004178974B4144C829A8BFF9
:10CE8800C82121EAE17141709B78002B94D01320CE
:10CE98001EF0A2F8D4F8E4008EE7D4F8E400017894
:10CEA8008D4B4144C829A8BFC82121EAE17101700E
:10CEB8009B78002B80D012201EF08EF8D4F8E40066
:10CEC8007AE70698844B81799A7841446429A8BF07
:10CED800642121EAE1718171002A40F0FA820D2F64
:10CEE8009BD006987C4B41799A7841446429A8BF25
:10CEF800642121EAE1714171002A8ED00E201EF0D2
:10CF08006BF8D4F8E40057E7D4F8E400724B017AE0
:10CF18009A784144C829A8BFC82121EAE171017261
:10CF2800002A3FF449AF0B201EF056F8D4F8E4006D
:10CF380042E7D4F8E400684BC1799A784144C8299B
:10CF4800A8BFC82121EAE171C171002A3FF434AFBA
:10CF58000A201EF041F8D4F8E4002DE7D4F8E400E4
:10CF68005D4B81799A784144C829A8BFC82121EA34
:10CF7800E1718171002A3FF41FAF09201EF02CF8DF
:10CF8800D4F8E40018E7D4F8E400534B41799A78D0
:10CF98004144C829A8BFC82121EAE1714171002A8A
:10CFA80040F09182112F7FF452AF05E7D4F8E400E6
:10CFB800494B01799A784144C829A8BFC82121EA78
:10CFC800E1710171002A40F0A582102F7FF453AF60
:10CFD800F2E6069A17794744642FA8BF642727EA20
:10CFE800E77717711EF012F83B4B9B78002B3FF444
:10CFF80014AF032039461DF0EFFFD4F8E400DBE658
:10D00800069A354B11784144FA29A8BFFA2121EA3A
:10D01800E17111709B78002B3FF4FFAE01201DF0E9
:10D02800DBFFD4F8E400C7E6069A2B4B917841441D
:10D038006429A8BF642121EAE17191709B78002BD3
:10D048003FF4EBAE02201DF0C7FFD4F8E400B3E6CE
:10D058000698214BC1799A78414481F30801C1713E
:10D06800002A3FF4DAAE05201DF0B6FFD4F8E4003C
:10D07800A2E6D4F8E400184BC1789A784144C8294C
:10D08800A8BFC82121EAE171C170002A40F02582B9
:10D098000F2F7FF404AF8FE6119AFFF773BB0F4B86
:10D0A8001B78002B3EF418AD0D4BDB78002B7EF47B
:10D0B80013AD94F8A8300133DBB2032B84F8A83001
:10D0C8007EF60AAD074B5B7813B9002E7EF404ADEB
:10D0D80007F0ECF8FFF7B1BAF1750020786000208E
:10D0E80054600020301D0020C24AC34B03921046F2
:10D0F8001A68C2494FF47A73B3FBF2F3C3EB4312D5
:10D1080003EB82030268DB005507A1F8A83000F1A1
:10D11800AC80059B1B6803F00403FEF7E3BC3BF9F6
:10D1280012209978B2F5617F4FF4966393FBF1F37F
:10D13800C0F2818040F633019142A8BF11460C2FFE
:10D14800A1F5617191FBF3F800F0C780182F7FF407
:10D15800C4AA5FFA88F1C8290B46A8BFC823D4F827
:10D16800E400C27DDFB297423FF4B7AA9B1AA44AF3
:10D17800C77548BF0733DB1092785F1CFFB23AB916
:10D18800002F3FF4AAAA384614F002FBFFF7A5BA0D
:10D1980018201DF021FFF3E79A499B4BCA681B68CA
:10D1A8008B609B1AC82B7FF674AB012381F8213062
:10D1B800FFF76FBB954B00220120A6E53968DAF826
:10D1C8001C200A44CAF8182029E4914B01220220A5
:10D1D8009BE5904A1268960304D58F4A1279002A73
:10D1E80040F0D8808D4819461A46465C0B2E01F14E
:10D1F8000C0107D00132152AF7D1002284F8A720A4
:10D20800FFF79DB8864ED6F800E05100BEF1000F3A
:10D2180007D08F1800EB87079EF801E07F787745E5
:10D22800EBD20A447F4F804900EB82020020326033
:10D2380038800860E1E70C2F64D0182F7FF44DAADE
:10D2480000210B468BE73A68B9F80630642101FBE8
:10D258000323CAF81030FFF7B9BB4FF003094B4658
:10D268005EE54FF004094B465AE5059B6F4A1B687B
:10D278000A21118003F00403FEF734BC4FF00509BE
:10D288004B464DE54FF006094B4649E54FF001097D
:10D298004B4645E54FF002094B4641E510F0C0F911
:10D2A800F6F75CFE10F0A4F9FDF718FE012014F063
:10D2B8006FFA94F8A620FFF75EB806F073FEFEF743
:10D2C8000BBC059B5A4A1B684FF4C8711180494A28
:10D2D800039203F00403FEF705BC5FFA88F7554B89
:10D2E8005B78BB423FF4F9A9384605F0F1FA444BA4
:10D2F8009B7823B15FFA88F10C201DF06DFE013791
:10D30800FFB23DE70027B846E9E70B464FF6FE7146
:10D31800494A38485589039090892B4401445381E0
:10D32800918110F07DF9F6F719FE10F061F9FDF71B
:10D33800D5FD012014F02CFA059B1B68002203F090
:10D34800040384F8A720FEF7CDBB0B460221DFE7D4
:10D358000223DDE74FF6FE73DAE70021FF201CF019
:10D3680012FB94F8A620FFF72EB801201CF00BFB47
:10D3780094F8A620FFF724B8304A137A43F0010343
:10D388001372FEF7A9BB2D4A137A23F00103137217
:10D39800FEF7A2BB2A4A1278002A7FF423AF14F0C2
:10D3A800F7F8049B1B7803F0010326E7029A515D06
:10D3B8009847032D1BDC40F2EE2240F6CA0C0028E9
:10D3C8003EF40FAF39F825E0BAF802104FF47A733B
:10D3D800A0EB0E0003FB00F0A1EB0E0190FBF1F0B7
:10D3E80018449042B8BF10466045A8BF604600B2D6
:10D3F800FEF7F7BE2869002018690020F4600020B5
:10D40800F17500205460002004730020DE740020B1
:10D4180028750020502C00207C60002074F202083F
:10D42800A82300204224002044240020188700203C
:10D438001A870020985E0020344C002038600020B5
:10D44800425E0020434E37684A003FB1551800EB52
:10D4580085057F786D78BD42BFF43CAC0A4400EB8B
:10D4680082023D4F3D4D326000213D4A398029609E
:10D478000392FEF737BB012100201CF084FA94F8D0
:10D48800A620FEF7A3BF002E3EF4A8AA94F8A5C0D4
:10D49800BCF1000F3EF4DAAA14F07AF895F800C04F
:10D4A80084F8A570FEF7D2BA0C2014F08FF8FEF7B6
:10D4B80013BB0122002184F8AA20294A84F8A91064
:10D4C8000392FEF70FBB11201DF086FDD4F8E4008F
:10D4D80068E50D201DF080FD01E50F201DF07CFDA5
:10D4E800D4F8E400D4E53BB11E491F4A09684FF45B
:10D4F8007A7000FB0313136094F8A530002B3EF4F8
:10D50800A5AA14F045F8002384F8A53095F800C0C2
:10D51800FEF79CBA10201DF05FFDD4F8E40054E536
:10D5280016201DF059FDD4F8E40045E406F0BEFECF
:10D53800002384F8A530FEF787BA0C49097829B189
:10D5480011461DE494F8A610FEF7EBBE14F020F87F
:10D55800FEF7C2BAA8230020422400204424002059
:10D5680028690020047300209C2A0020425E0020C5
:10D578002DE9F04FDFF808B12DED0C8B9BF800304A
:10D5880099B0012B039001F02882DFF8F8A09AF8EF
:10D598000021002A41F03082072B01F037824FF03A
:10D5A8000009344C63682046984700286ED0B4F8C8
:10D5B800A860002284F84920002E40F08E82B4F939
:10D5C8002450E16AB4F92600226BB4F92830691AAC
:10D5D800A16329490091821A606BE2630D461B1A08
:10D5E80094F84A10236404F138000DF02DF92B68E3
:10D5F80013F0005302F0C281D4ED0F5AD4ED0E7A25
:10D608001E4A9AED416ADAED426A9AED437ADAF8EF
:10D6180010311268B8EEE58AD4ED105AF8EEE77AC0
:10D62800F8EEE58A013377EE867A38EE268A78EEC8
:10D63800878A9342CAED417A8AED428ACAED438AC3
:10D64800CAF8103101F0A0869BF80060142E02F091
:10D65800A6870023DAF818510193062D02F25082AA
:10D66800DFE815F0D714C314EE111E171616AD1601
:10D678009A1500BFF4600020203700202C69002094
:10D688005630002084220020DDF804909BF80080AA
:10D69800B8F1070F00F0D8829AF828310593002BCB
:10D6A80040F0DE82CD4B5B79002B40F011820123E4
:10D6B8009BF800208AF82831072A02F07B82002391
:10D6C8000793C74BDAED4C9A93ED007AC54AC64BDF
:10D6D8001268C64FDAED4B8ADFF89093DFEDC4AAE3
:10D6E8009FEDC49A9FEDC4BADFEDC4CA9FEDC4AAEA
:10D6F800DFEDC4BADFF87883C34E0493F7EE007AFF
:10D7080037EEE98A002428EE078A0292B4EEE78A07
:10D71800F1EE10FA88BFB0EE678A019325460097AC
:10D72800BA4B2344D3ED007AB94BF5EE407A234443
:10D73800F1EE10FA93ED00CA17D0B64B234493EDDF
:10D74800007A7CEE476AB0EEE66AF4EEC67AF1EE4D
:10D7580010FA08D5F5EEC06AF1EE10FACCBF37EE34
:10D7680087CA37EE67CA83ED00CABAF84C71BB079F
:10D7780000F07E82022D04F022850299A64B91F8D2
:10D78800322007EE102A91F831202344D3ED006AA5
:10D798005342B8EEC77A07EE903A27EE267AF8EEAB
:10D7A800E77AB4EEE77AF1EE10FA0AD407EE902A97
:10D7B800F8EE677AF4EEC77AF1EE10FA88BFF0EE69
:10D7C800477A964B0693964A03EB450332F91510B0
:10D7D800B3F90A30C81A07EE100AB8EEC77AF80784
:10D7E800E7EE497A40F195828E4F97ED00CA27EE11
:10D7F8008CCA9AF86871E7B18A4FDAF86C0197ED2C
:10D80800007A894F5B1A07EE903A039B396827EE36
:10D81800097AF8EEE77A1F1A8F4227EE87CA01F3D2
:10D82800AB81F7EE007AF4EEE79AF1EE10FA01F127
:10D838006F817E4B2344D3ED007A019BD3ED01DA4F
:10D84800009B68EEA77A3CEE6DDA67EE8D7AC3ED41
:10D85800007A774BD9ED006A93ED007A754BD6EDD7
:10D86800007A26EE877A234467EE086A93ED007AF9
:10D8780026EE877AF0EE676AE7EE0D6AB0EE667A12
:10D888009AED4C6AF7EE006AB4EEE66AF1EE10FA29
:10D89800ACBF0123002343B1F0EEE77AF0EEC76A8C
:10D8A800F4EEE76AF1EE10FA01D586ED007A022D62
:10D8B80004F07E84604A614B52F825001B68B0EE84
:10D8C8006D0A98475E4A5F4B52F825001B689847D7
:10D8D800029B93F83A30632B04D8BAF84C31002BEA
:10D8E80001F05C81F0EE6C7A574B99ED007A37EED7
:10D8F800C00A2344D3ED007A83ED000A029B30EE80
:10D90800670A93F8482080EE07CADAB1F7EE007A82
:10D91800F4EEE79AF1EE10FA14DB4C4BD3ED007AF3
:10D92800B0EECC7AB4EEE77AF1EE10FA0ADD484BA5
:10D93800D3ED007AB0EECDDAB4EEE7DAF1EE10FA14
:10D9480001F38A81434B9AF878212344D3ED007A76
:10D9580068EEA77A27EE8CCA88ED00CA32B9009B18
:10D96800C6ED00CAC3ED00CAC8ED00CA009B043367
:10D978000093019B043404330C2C05F1010508F1D4
:10D98800040806F1040601937FF4CAAE9BF8003040
:10D99800072B02F0C980012B02F0FC8000230493BE
:10D9A8002D4B00931A460F4B12681B6801921146C3
:10D9B80093F82F2011F48053069300F04D82274BE3
:10D9C80002931B782648079013F0010F254B039309
:10D9D800198B254B90ED037ADB884BE0E060002043
:10D9E80060510020B05E002018690020F42D00204E
:10D9F80000009642CDCCCC3DAE47813F00000000F0
:10DA08000000C84200003443002E0020545100207A
:10DA1800B8230020C4230020D4230020344C002045
:10DA28002C5F002038510020645100200C51002048
:10DA380008000020185100207C5100207851002057
:10DA4800E0510020DC510020F42300207451002014
:10DA580070510020245100202037002035850020F7
:10DA6800445E0020F036002064570020505100200A
:10DA78000C2E002008BFAAF88011C81A07EE900AD9
:10DA8800F8EEE77AB4EEE77AF1EE10FA42F2668041
:10DA9800CC1806EE904AF8EEE66AB4EEE67AF1EEB5
:10DAA80010FA81F23A84BAF88031984283F24581BB
:10DAB800D44BD54993ED004AD1ED004AD34BCAED7A
:10DAC800614A8AED624AD3ED006ADFEDD17ADFE17F
:10DAD800D04B1B78013BDBB2EAE5CF49CF4B497805
:10DAE800049300911B68CE4F9BF80080B7F906009D
:10DAF8004FF47A71B1FBF3F3C3EB431503EB8503E2
:10DB0800DD00ADB2AE4202F02E86E16FB4F924E03A
:10DB1800236E4A1C07EE90EA7344012AE2672366E3
:10DB2800F8EEE77A02F02986D4ED1B5AD4ED1D6A87
:10DB380007EE102A37EEE56AB8EEC75A012E86EED0
:10DB4800057A37EE257A77EEC77A84ED1C7AE6EE09
:10DB5800276A84ED1B7AF0EE667AC4ED1E6AC4ED7E
:10DB68001D6A03F04981D4F89010B4F926E0636E79
:10DB78004A1C07EE90EA7344012AC4F890206366B1
:10DB8800F8EEE77A02F01186D4ED205AD4ED226A35
:10DB980007EE102A37EEE56AB8EEC75A012E86EE70
:10DBA800057A37EE257A77EEC77A84ED217AE6EEA4
:10DBB800276A84ED207AF0EE667AC4ED236AC4ED14
:10DBC800226A03F03B81D4F8A410B4F928E0A36ECC
:10DBD8004A1C07EE90EA7344012AC4F8A420A366FD
:10DBE800F8EEE77A02F0FA85D4ED255AD4ED276AE3
:10DBF80007EE102A37EEE56AB8EEC75A012E86EE10
:10DC0800057A37EE257A77EEC77A84ED267AE6EE3E
:10DC1800276A84ED257AF0EE667AC4ED286AC4EDA9
:10DC2800276A03F02D81F880B4F8A8309BF80080AB
:10DC3800013BA4F8A83004990023B8F1070F4B6002
:10DC48008B60CB607FF428ADFDF720FC744F9AF809
:10DC580028310593A0EB09003880002B3FF422AD52
:10DC6800013B8AF8283119B0BDEC0C8BBDE8F08F68
:10DC78009AF8683163B1022D04F0A482694B0693C7
:10DC8800694A03EB450332F91510B3F90A30B3E5D5
:10DC9800664B234493ED000A019BD3ED01DA009B08
:10DCA80028EE800A3CEE6DDA022D20EE0D0A83ED97
:10DCB800000A7FF4CEAD5E4A5E4B10681B68984739
:10DCC8005D4BD9ED006A93ED007A5C4BD6ED007A96
:10DCD8001A785B4B83ED020A5A4B26EE877A234467
:10DCE80027EE087A93ED006A27EE067AF0EE676A67
:10DCF800E7EE0D6A012AB0EE667A02D0192A7FF49F
:10DD0800BFADB4EEEADAF1EE10FACCBF012300237E
:10DD1800C1E5DAED576A9AED587AB2F900E0B2F93E
:10DD28000270B4EEE67AF1EE10FA8EEAEE7087EA47
:10DD3800E77C4CBFB7EE007AF7EE006AA0EBEE7016
:10DD4800ACEBE77C4CBF77EE665A76EEC75A604577
:10DD580040F34487BEF1000FD6BFCEF1000007EEB6
:10DD680010EA07EE100A384FB8EEC77A3F7827EE68
:10DD7800097A002F00F04287344F97ED005AB5EE2C
:10DD8800C05AF1EE10FA41F35786314FD7ED004AE9
:10DD9800F5EEC04AF1EE10FA41F34E8634EEC77A3A
:10DDA800B7EE006AC7EE246A75EEC65AF4EEC66A84
:10DDB80065EE8A5AF1EE10FA85EE857A88BFF0EEA4
:10DDC800466AF5EEC06AF1EE10FA37EE067AB8BF89
:10DDD800F0EE6C6A66EE876AF4EEC66AF1EE10FA47
:10DDE80088BFF0EE466AF5EEC06AF1EE10FAB8BFE9
:10DDF800F0EE6C6A174F97ED007A67EE877AA7EE18
:10DE0800A6CAF6E45C570020585700207457002033
:10DE18000000000058560020E0600020186900202B
:10DE2800765E0020344C00202C5F00200C5100202E
:10DE380040560020545600200800002008510020B9
:10DE4800F42D00201851002044510020405100209A
:10DE5800485100203C510020E24B03935B8BE24980
:10DE6800079107EE903AE14B91ED037AE04993ED83
:10DE7800004AE04BD1ED004AD3ED006ADE4B8AED53
:10DE8800624AF8EEE77A029377EE677ACAED614A5A
:10DE9800C7EEA62AD949DA4B91ED008AD949DFEDB8
:10DEA800DA6A91ED005AD9499FEDD96AD1ED005A45
:10DEB80093ED007AF7EE007AF4EEE72A38EE058A59
:10DEC800F1EE10FA88BFF0EE672A38EE258AF4EEF4
:10DED800E62AF1EE10FA28EE066AB8BFF0EE662AD6
:10DEE800F1EE476A34EEC43AB4EEE66AF1EE10FA9F
:10DEF800CAED632A8AED653A00F16B85B4EEC76A0C
:10DF0800F1EE10FA88BFB0EE476ABC4BDFEDC07A7D
:10DF1800D3ED018ABB4B93ED015ABC4B78EE858A51
:10DF2800D3ED015A78EEA58A68EEA77AF4EEE76A8F
:10DF3800F1EE10FA08DCB4EEE77AF1EE10FA8CBFD5
:10DF4800F0EE676AF0EE476AAC4BDFEDB17A93ED1D
:10DF5800029AAC4BD3ED025AAE4B39EE259A93EDAB
:10DF6800007A69EE277AF1EE475AF4EEE57AF1EE97
:10DF780010FA08D4F4EEC77AF1EE10FA8CBFF0EE7E
:10DF8800475AF0EE675A002A41F08982F7EE007A84
:10DF9800A14B5A789AF89831002AA04AFFEE003A25
:10DFA800B7EE007A127814BFB0EE472AB0EE632AB3
:10DFB800002B14BFB0EE635AB0EE475A002A02F0A5
:10DFC8005B84F4EEC77AF1EE10FA65EE825A944B50
:10DFD80041F3128393ED027A93ED011AD3ED031AFC
:10DFE8009FED892A26EE877A67EE853AA6EE017AB2
:10DFF800A5EEA17A27EE237AB4EEC27AF1EE10FAF2
:10E00800B4BFF0EE427AF0EE477A8DED0C7A88BF15
:10E01800B0EE427A012A00F0BE8193ED065AD3EDA4
:10E02800051A93ED072A26EE855AA6EE215AA5EE83
:10E03800825A25EE235AB4EEC57AF1EE10FAF4EEC0
:10E04800C57A8CBFB0EE452AB0EE472AF1EE10FA39
:10E0580058BFB0EE427AB8BFF0EE457A022A8DED8D
:10E068000D5A00F0988193ED0A5AD3ED091A93EDF1
:10E078000B2A26EE855AA6EE215AA5EE825A25EEDF
:10E08800235AB4EEC57AF1EE10FAF4EEC57A8CBFD5
:10E09800B0EE452AB0EE472AF1EE10FA58BFB0EEBE
:10E0A800427AB8BFF0EE457A032A8DED0E5A00F099
:10E0B800728193ED0E5AD3ED0D1A93ED0F2A26EEC9
:10E0C800855AA6EE215AA5EE825A25EE235AB4EEB9
:10E0D800C57AF1EE10FAF4EEC57A8CBFB0EE452A97
:10E0E800B0EE472AF1EE10FA58BFB0EE427AB8BF48
:10E0F800F0EE457A042A8DED0F5A00F04C8193ED2D
:10E10800125AD3ED111A93ED132A26EE855AA6EE6C
:10E11800215AA5EE825A25EE235AB4EEC57AF1EEBD
:10E1280010FAF4EEC57A8CBFB0EE452AB0EE472A55
:10E13800F1EE10FA58BFB0EE427AB8BFF0EE457A69
:10E14800052A8DED105A00F0268193ED165AD3ED6D
:10E15800151A93ED172A26EE855AA6EE215AA5EE32
:10E16800825A25EE235AB4EEC57AF1EE10FAF4EE8F
:10E17800C57A8CBFB0EE452AB0EE472AF1EE10FA08
:10E1880058BFB0EE427AB8BFF0EE457A062A8DED58
:10E19800115A00F0008193ED1A5AD3ED191A93ED34
:10E1A8001B2A26EE855AA6EE215AA5EE825A25EE9E
:10E1B800235AB4EEC57AF1EE10FAF4EEC57A8CBFA4
:10E1C800B0EE452AB0EE472AF1EE10FA58BFB0EE8D
:10E1D800427AB8BFF0EE457A072A8DED125A00F060
:10E1E800DA801FE0F0360020445E0020A42E0020D4
:10E1F800585700206C57002035850020F42D00204A
:10E208005C560020002E0020000000000C2E00208C
:10E218006F12833A6056002054300020182E0020D8
:10E228009856002093ED1E5AD3ED1D1A93ED1F2A20
:10E2380026EE855AA6EE215AA5EE825A25EE235AD5
:10E24800B4EEC57AF1EE10FAF4EEC57A8CBFB0EEF2
:10E25800452AB0EE472AF1EE10FA58BFB0EE427ADE
:10E26800B8BFF0EE457A082A8DED135A00F0938076
:10E2780093ED225AD3ED211A93ED232A26EE855ADF
:10E28800A6EE215AA5EE825A25EE235AB4EEC57A97
:10E29800F1EE10FAF4EEC57A8CBFB0EE452AB0EE76
:10E2A800472AF1EE10FA58BFB0EE427AB8BFF0EE46
:10E2B800457A092A8DED145A6DD093ED265AD3ED7F
:10E2C800251A93ED272A26EE855AA6EE215AA5EEA1
:10E2D800825A25EE235AB4EEC57AF1EE10FAF4EE1E
:10E2E800C57A8CBFB0EE452AB0EE472AF1EE10FA97
:10E2F80058BFB0EE427AB8BFF0EE457A0A2A8DEDE3
:10E30800155A48D093ED2A5AD3ED291A93ED2B2AA2
:10E3180026EE855AA6EE215AA5EE825A25EE235AF4
:10E32800B4EEC57AF1EE10FAF4EEC57A8CBFB0EE11
:10E33800452AB0EE472AF1EE10FA8DED165A58BF6D
:10E34800B0EE427AA8BFB0EE675A0B2A02F0F18409
:10E35800D3ED2E7AD3ED2D1A93ED2F2A66EEA77AF8
:10E36800E1EE867AE2EE257A67EEA37AF4EEC77AD2
:10E37800F1EE10FAF4EEC57A8CBFF0EE476AF0EED3
:10E38800676AF1EE10FACDED177A98BFB0EE667AAB
:10E39800B8BFF0EE457A77EEC77AF7EE006AF4EE8A
:10E3A800E67AF1EE10FACAED4C7A42F3B28486EEC0
:10E3B800A77A012ADDED0C7A67EE877ACDED0C7A23
:10E3C80055D0DDED0D7A67EE877A022ACDED0D7A0C
:10E3D8004DD0DDED0E7A67EE877A032ACDED0E7A01
:10E3E80045D0DDED0F7A67EE877A042ACDED0F7AF6
:10E3F8003DD0DDED107A67EE877A052ACDED107AEB
:10E4080035D0DDED117A67EE877A062ACDED117ADF
:10E418002DD0DDED127A67EE877A072ACDED127AD4
:10E4280025D0DDED137A67EE877A082ACDED137AC9
:10E438001DD0DDED147A67EE877A092ACDED147ABE
:10E4480015D0DDED157A67EE877A0A2ACDED157AB3
:10E458000DD0DDED167A67EE877A0B2ACDED167AA8
:10E4680005D0DDED177A27EE877A8DED177AE14B27
:10E47800196811F0805100F0AC834FF07C53CAF852
:10E488008C31002A02F0F281029BDB4E1F78DB4CB4
:10E49800DB48DC4DD6ED005A9AF89031039EE478BB
:10E4A8000078B5F90650DAED636A768B07F0010C4F
:10E4B800019F07F0100E07F48007002B40F0AB8295
:10E4C800BEF1000F00F0AE85BCF1000F42F07E8374
:10E4D800002C42F05A84CC4BDDED0C7A93ED007A97
:10E4E800CA48E7EE267ABDEEE47A17EE101AB0EEC7
:10E4F800447AA3EE277A0D46F0EE477AFDEEE77AE6
:10E50800BDEEC47A17EE906A17EE104AB142A8BF62
:10E518003546B442C8BF254607EE905AF8EEE77A6A
:10E52800012AC0ED007A00F04D8193ED047ADDED0B
:10E538000D7AE7EE267AB0EE447AA3EE277AFDEE5E
:10E54800C77A17EE906A17EE905A8E42A8BF0D460A
:10E55800A642B8BF254607EE905AF8EEE77A022A97
:10E56800C0ED017A00F02E8193ED087ADDED0E7A88
:10E57800E7EE267AB0EE447AA3EE277AFDEEC77A64
:10E5880017EE906A17EE905A8E42A8BF0D46A64223
:10E59800B8BF254607EE905AF8EEE77A032AC0ED91
:10E5A800027A00F00F8193ED0C7ADDED0F7AE7EE39
:10E5B800267AB0EE447AA3EE277AFDEEC77A17EEF4
:10E5C800906A17EE905A8E42A8BF0D46A642B8BF71
:10E5D800254607EE905AF8EEE77A042AC0ED037A4A
:10E5E80000F0F08093ED107ADDED107AE7EE267AF0
:10E5F800B0EE447AA3EE277AFDEEC77A17EE906A5A
:10E6080017EE905A8E42A8BF0D46A642B8BF2546BF
:10E6180007EE905AF8EEE77A052AC0ED047A00F082
:10E62800D18093ED147ADDED117AE7EE267AB0EE1B
:10E63800447AA3EE277AFDEEC77A17EE906A17EEB2
:10E64800905A8E42A8BF0D46A642B8BF254607EE8F
:10E65800905AF8EEE77A062AC0ED057A00F0B28003
:10E6680093ED187ADDED127AE7EE267AB0EE447A69
:10E67800A3EE277AFDEEC77A17EE906A17EE905A46
:10E688008E42A8BF0D46A642B8BF254607EE905A4F
:10E69800F8EEE77A072AC0ED067A00F0938093ED4A
:10E6A8001C7ADDED137AE7EE267AB0EE447AA3EE13
:10E6B800277AFDEEC77A17EE906A17EE905A8E42C7
:10E6C800A8BF0D46A642B8BF254607EE905AF8EEF9
:10E6D800E77A082AC0ED077A74D093ED207ADDED49
:10E6E800147AE7EE267AB0EE447AA3EE277AFDEEA6
:10E6F800C77A17EE906A17EE905A8E42A8BF0D4659
:10E70800A642B8BF254607EE905AF8EEE77A092ADE
:10E71800C0ED087A56D093ED247ADDED157AE7EE50
:10E72800267AB0EE447AA3EE277AFDEEC77A17EE82
:10E73800906A17EE905A8E42A8BF0D46A642B8BFFF
:10E74800254607EE905AF8EEE77A0A2AC0ED097ACC
:10E7580038D093ED287ADDED167AE7EE267AB0EE1A
:10E76800447AA3EE277AFDEEC77A17EE906A17EE81
:10E77800905A8E42A8BF0D46A642B8BF254607EE5E
:10E78800905AF8EEE77A0B2AC0ED0A7A1AD093ED80
:10E798002C7ADDED177AE6EE877AA3EE274AFDEEAE
:10E7A800C47A17EE903A9942A8BF19469C42D8BF3E
:10E7B8000C4607EE904AF8EEE77AC0ED0B7A002A8D
:10E7C80000F0F9839200124910481FF000FF114B26
:10E7D8001B68002B00F0F4830F4B1B78192B22D8F1
:10E7E80001220E4902FA03F31940002942F054832A
:10E7F80016E000BF8C2E00206456002054600020D4
:10E8080024320020BC83002098560020502E00207F
:10E81800685600200451002008510020324130037E
:10E828001E0301F1AE86AD4DAD4E019B9C061BD576
:10E83800F37AFF2B04D0AB4A12789A4201F29C86F5
:10E84800B6F90870F37D2F80FF2B04D0A54A127803
:10E858009A4201F28C86B6F914406C80082007F0C1
:10E8680019FC002841F0A083B6F90600B5F900E0CC
:10E87800B5F90270B6F91210B6F91E20B5F90440C0
:10E88800B6F90430B5F906C07045A8BF7046B9425C
:10E89800A8BF3946A242A8BF22469E45A8BF034644
:10E8A8002B80B6F91030B5F90800BB42C8BF19462D
:10E8B800B6F92A306980B6F91C10B6F93470634588
:10E8C800A8BF6346A142CCBF0C461446B6F9362011
:10E8D800AC80B6F92840B5F90A108242A8BF0246B2
:10E8E800A445ACBF9C46A446B6F94230B5F90C40E5
:10E8F800A5F806C08B42A8BF0B468742CCBF384656
:10E908001046B6F94E202881B6F94000B5F90E70C8
:10E91800A242A8BF22468842C8BF0346B6F95A0099
:10E92800B6F94C106B81B842B6F958306E4EA8BF94
:10E9380038469F42A8BF0346A142D8BF1146A981C5
:10E94800EB81B38923B3694FDFF8B891DFF8908181
:10E9580007F11004B7F9023000EE103A4846B8EE55
:10E96800C00AF3F761FF1DF03FFDB8F90430B8F9AC
:10E97800062000B2984209F12C0908F10C0803DBC3
:10E9880082421346A8BF034627F8023FA742E1D1B7
:10E99800574B1B78013B182B00F2C485DFE813F0B6
:10E9A800B005C205C205F00AC205C205C2051F0EA0
:10E9B800C205C205C205C205C2055F0EC205C20571
:10E9C800C205C2050E0EF00A500EC205C2055F0E42
:10E9D800B005B0EE666AFFF798BA464BDFF828A193
:10E9E8001968454A454F9AF80031C9691288398033
:10E9F8007A80002B3EF4D3ADF6F786FA00238AF826
:10EA080000319BF80030072B7EF4C9ADFCF73EFDC2
:10EA18008146FEF7C6BDBEF1000F00F04B81BCF188
:10EA2800000F42F02181002841F03A82FDEEC47ABD
:10EA38000DF1300E17EE906AFDEEE47A0EEB8203CC
:10EA480017EE907AFDEEE57A2D48DFF8C090CDF804
:10EA580024A017EE905AB1EE436A84F001084FFAE9
:10EA680084FC08929A46034693ED007AFEEC017AFC
:10EA7800E7EE267A3A461030B0EE647AA6EE277AA8
:10EA8800FDEEC77A17EE903A9F42A8BF1A469D42FC
:10EA9800CCBF002104F00101002914BF114629460A
:10EAA8009E42CCBF002308F0010307EE901A002B0A
:10EAB80014BF13463346B8EEE77A07EE903AF8EEFD
:10EAC800E77ABCF1000F18BFF0EE477AD645E9ECBB
:10EAD800017AC8D1089ADDF824A070E6402E0020FB
:10EAE800E4570020345F0020D46E00203E2E002022
:10EAF80008510020DC600020C82B0020765E002032
:10EB080098560020C04E002084220020502E00205D
:10EB1800069BB2F90070B3F90A305A49F81A096825
:10EB280080EAE073A3EBE0738B42BEF682AEB2F9E3
:10EB38000230069AB2F90C209A1A82EAE273A3EB21
:10EB4800E27399427EF775AE04994F4BD1ED017A85
:10EB580093ED007AF0EEE77AF4EEC77AF1EE10FA68
:10EB68007EF567AED1ED027AF0EEE77AB4EEE77A99
:10EB7800F1EE10FA7EF75DAE444B1A8800238AF84E
:10EB88006831002A40F0EA83414A424B11781868FC
:10EB980081F00101F4F7AAFFFEF74BBE3E4B3F4A56
:10EBA8002344D3ED006A92ED007A3D4B26EE877A36
:10EBB800F7EE006AB4EEE67AD3ED007AF1EE10FAD9
:10EBC80088BFB0EE667A27EE277A67EE0C7AFEF7F2
:10EBD8008BBE019B5F023FF550AC52E4002FD6BFBD
:10EBE800784207EE107A07EE100A2E4FB8EEC77A71
:10EBF8003F7827EE097A002F7FF4BEA82A4FD7ED79
:10EC0800006AF4EECB6AF1EE10FA40F1BE87B7EE77
:10EC1800005A35EE665A9FED256A254F3BEEC77AB6
:10EC280025EE065A97ED006AE7EE056A26EE867A23
:10EC3800B5EEC07AF1EE10FA40F2FE86CAEE076A27
:10EC4800B7EE006A35EEC67AF0EE465AE7EE265A77
:10EC5800F0EE656AFFF7C0B801230399CAF86C1192
:10EC6800022A8AF868317EF46DAE084A1288002AB2
:10EC780043F0DF81064A074B11781868F4F736FF2E
:10EC8800FEF760BE685100206C510020DC72002045
:10EC9800DE720020E0720020E023002034510020C2
:10ECA80030510020445100204C510020610BB63BEC
:10ECB80040510020D44BDDED0C7A93ED007A00280A
:10ECC80040F09887E7EE267AD048B1EE436AB0EE76
:10ECD800647AA6EE277AF0EE477ABDEEE47A002C45
:10ECE80042F0F082FDEEE77A17EE104A17EE906ACE
:10ECF800FDEEC47AB44217EE901A17EE105AA8BF68
:10ED08003546B142C8BF0D4607EE905AF8EEE77A8D
:10ED1800012AC0ED007A00F04A8193ED047ADDED16
:10ED28000D7AE7EE267AB0EE647AA6EE277AFDEE43
:10ED3800C77A17EE906A17EE905AA642A8BF2546E2
:10ED48008E42B8BF0D4607EE905AF8EEE77A022ACF
:10ED5800C0ED017A00F02B8193ED087ADDED0E7A93
:10ED6800E7EE267AB0EE647AA6EE277AFDEEC77A49
:10ED780017EE906A17EE905AA642A8BF25468E4213
:10ED8800B8BF0D4607EE905AF8EEE77A032AC0EDB1
:10ED9800027A00F00C8193ED0C7ADDED0F7AE7EE44
:10EDA800267AB0EE647AA6EE277AFDEEC77A17EED9
:10EDB800906A17EE905AA642A8BF25468E42B8BF61
:10EDC8000D4607EE905AF8EEE77A042AC0ED037A6A
:10EDD80000F0ED8093ED107ADDED107AE7EE267AFB
:10EDE800B0EE647AA6EE277AFDEEC77A17EE906A3F
:10EDF80017EE905AA642A8BF25468E42B8BF0D46C8
:10EE080007EE905AF8EEE77A052AC0ED047A00F08A
:10EE1800CE8093ED147ADDED117AE7EE267AB0EE26
:10EE2800647AA6EE277AFDEEC77A17EE906A17EE97
:10EE3800905AA642A8BF25468E42B8BF0D4607EE97
:10EE4800905AF8EEE77A062AC0ED057A00F0AF800E
:10EE580093ED187ADDED127AE7EE267AB0EE647A51
:10EE6800A6EE277AFDEEC77A17EE906A17EE905A4B
:10EE7800A642A8BF25468E42B8BF0D4607EE905A57
:10EE8800F8EEE77A072AC0ED067A00F0908093ED55
:10EE98001C7ADDED137AE7EE267AB0EE647AA6EEF8
:10EEA800277AFDEEC77A17EE906A17EE905AA642B7
:10EEB800A8BF25468E42B8BF0D4607EE905AF8EE19
:10EEC800E77A082AC0ED077A71D093ED207ADDED54
:10EED800147AE7EE267AB0EE647AA6EE277AFDEE8B
:10EEE800C77A17EE906A17EE905AA642A8BF254631
:10EEF8008E42B8BF0D4607EE905AF8EEE77A092A17
:10EF0800C0ED087A53D093ED247ADDED157AE7EE5B
:10EF1800267AB0EE647AA6EE277AFDEEC77A17EE67
:10EF2800906A17EE905AA642A8BF25468E42B8BFEF
:10EF38000D4607EE905AF8EEE77A0A2AC0ED097AEC
:10EF480035D093ED287ADDED167AE7EE267AB0EE25
:10EF5800647AA6EE277AFDEEC77A17EE906A17EE66
:10EF6800905AA642A8BF25468E42B8BF0D4607EE66
:10EF7800905AF8EEE77A0B2AC0ED0A7A17D093ED8B
:10EF88002C7ADDED177AE6EE877AE6EE274AFDEE73
:10EF9800E47A17EE903A9C42A8BF1C469942D8BF23
:10EFA800214607EE901AF8EEE77AC0ED0B7ABCF12D
:10EFB800000F3FF404AC164B1B68002B7FF40CAC1D
:10EFC800144B1B7893B1144B187860B10F4D134E46
:10EFD8000024E0B23368B5EC010A98470E4B187864
:10EFE80001348442F5DB0E4B1B6898479BF80030D0
:10EFF800072B00F0AB8501238AF8003119B0BDEC6E
:10F008000C8BBDE8F08F00BF98560020502E0020D2
:10F01800045100208C360020182E002018320020C1
:10F0280020320020D24BDDED0C7A93ED007A002CD3
:10F0380041F05484E7EE267ACE48BDEEE47A17EE26
:10F04800101AB0EE447AA3EE277A0D46F0EE477A0E
:10F05800FDEEE77ABDEEC47A17EE906A17EE104A15
:10F06800B142A8BF3546B442C8BF254607EE905AFC
:10F07800F8EEE77A012AC0ED007A98D093ED047A89
:10F08800DDED0D7AE7EE267AB0EE447AA3EE277A24
:10F09800FDEEC77A17EE906A17EE905A8E42A8BF17
:10F0A8000D46A642B8BF254607EE905AF8EEE77A15
:10F0B800022AC0ED017A3FF47AAF93ED087ADDEDCC
:10F0C8000E7AE7EE267AB0EE447AA3EE277AFDEEC2
:10F0D800C77A17EE906A17EE905A8E42A8BF0D466F
:10F0E800A642B8BF254607EE905AF8EEE77A032AFB
:10F0F800C0ED027A3FF45BAF93ED0C7ADDED0F7A49
:10F10800E7EE267AB0EE447AA3EE277AFDEEC77AC8
:10F1180017EE906A17EE905A8E42A8BF0D46A64287
:10F12800B8BF254607EE905AF8EEE77A042AC0EDF4
:10F13800037A3FF43CAF93ED107ADDED107AE7EEF9
:10F14800267AB0EE447AA3EE277AFDEEC77A17EE58
:10F15800906A17EE905A8E42A8BF0D46A642B8BFD5
:10F16800254607EE905AF8EEE77A052AC0ED047AAC
:10F178003FF41DAF93ED147ADDED117AE7EE267AB0
:10F18800B0EE447AA3EE277AFDEEC77A17EE906ABE
:10F1980017EE905A8E42A8BF0D46A642B8BF254624
:10F1A80007EE905AF8EEE77A062AC0ED057A3FF4A2
:10F1B800FEAE93ED187ADDED127AE7EE267AB0EE20
:10F1C800447AA3EE277AFDEEC77A17EE906A17EE17
:10F1D800905A8E42A8BF0D46A642B8BF254607EEF4
:10F1E800905AF8EEE77A072AC0ED067A3FF4DFAEC8
:10F1F80093ED1C7ADDED137AE7EE267AB0EE447AC9
:10F20800A3EE277AFDEEC77A17EE906A17EE905AAA
:10F218008E42A8BF0D46A642B8BF254607EE905AB3
:10F22800F8EEE77A082AC0ED077A3FF4C0AE93ED0E
:10F23800207ADDED147AE7EE267AB0EE447AA3EE72
:10F24800277AFDEEC77A17EE906A17EE905A8E422B
:10F25800A8BF0D46A642B8BF254607EE905AF8EE5D
:10F26800E77A092AC0ED087A3FF4A1AE93ED247A33
:10F27800DDED157AE7EE267AB0EE447AA3EE277A2A
:10F28800FDEEC77A17EE906A17EE905A8E42A8BF25
:10F298000D46A642B8BF254607EE905AF8EEE77A23
:10F2A8000A2AC0ED097A3FF482AE93ED287ADDEDA3
:10F2B800167AE7EE267AB0EE447AA3EE277AFDEEC8
:10F2C800C77A17EE906A17EE905A8E42A8BF0D467D
:10F2D800A642B8BF254607EE905AF8EEE77A0B2A01
:10F2E800C0ED0A7A3FF463AE93ED2C7ADDED177A20
:10F2F800E6EE877AA3EE274AFDEEC47A17EE903A37
:10F308009942A8BF19469C42D8BF0C4607EE904ABE
:10F31800F8EEE77AC0ED0B7A49E607EE901AF8EEB8
:10F32800E77A1548154C90ED004AD4ED004A144888
:10F33800CAED614A06EE903A77EE677ABCEEC77A74
:10F34800F8EEE66A17EE103A77EEE67A8AED624A48
:10F35800AAF88031D0ED006AFEF79ABD09494A69DA
:10F36800002A3EF466AA0A6813604B74FEF761BA75
:10F3780098560020502E00205C5700205857002037
:10F3880074570020E472002007EE103A9BF8003012
:10F398008E4FCAF81061B8EEC77AF7EE006A132BE1
:10F3A80086EE879AB7F90400BAF8145194ED080A62
:10F3B80001F06481864B874A93ED001A93ED093A70
:10F3C80093ED162A93ED1F6AD3ED0B1A93ED144AA9
:10F3D800D3ED015AD3ED0A3A93ED0C7A93ED155A11
:10F3E800D3ED172AD3ED206AD3ED044AD3ED030AEF
:10F3F80069EE277A69EE288A29EE088AA7EE813A0B
:10F4080002EB85060021A2EE286ACAF80411CAF8A0
:10F418000811A8EE214AE7EEA53AA8EE075A93ED9F
:10F428001A7AD3ED0F5A93ED021AD3ED0E1A86ED20
:10F43800003AE2EEA86A64EEC34A27EE467A93EDF4
:10F448000D2AD3ED192A86ED204AE3EE603A65EEDF
:10F45800C45A93ED183AC3ED093AE7EE814AF0EE43
:10F46800477AA4EE615AE8EE025AE2EEC66AE3EE83
:10F47800287AC3ED0A4A83ED145AC3ED155A86ED6E
:10F48800406AC3ED1F6AC3ED207ACAF80C116B1CE1
:10F4980003F01F03AAF81431B880FEF7D5B84E4B15
:10F4A8001A79002A3EF472AD4C4A1278002A3EF4CA
:10F4B8006DAD1B789FED4A2A07EE103A494B07EECF
:10F4C800902A1B88F8EEE77A05EE103AB8EE477AEC
:10F4D800B8EE455A27EE277AF7EE003AC7EE057AD6
:10F4E800F4EEC27AF1EE10FA88BFF0EE427AF4EE4A
:10F4F800E37AF1EE10FAB8BFF0EE637AFEF748BD92
:10F50800B37B002B42F06984029B1B7813F0010344
:10F5180042F06384344A1268002A02F01F8613609E
:10F5280001230593009B1B68980633D42F4A127851
:10F53800052A2FD0D9027FF543ADF57B112D3FF673
:10F548003FAD2B4BDDF814801C4633F9153000EE27
:10F55800103A4046B8EEC00A6F1C05F10E0605F0D9
:10F5680003FB4346FFB25D1BF6B2A04600E0274608
:10F578007C1C7819122FE4B2C0B23FF421AD38F9DF
:10F58800173000EE103AB8EEC00A05F0EDFAB442B2
:10F59800EDD115E5059A13460233541CDBB210462B
:10F5A800E4B20593B5F9003000EE103AB8EEC00A9F
:10F5B80005F0DAFAB5F9023000EE103A2046B8EE56
:10F5C800C00A05F0D1FA009B1B68B3E7765E0020FD
:10F5D800EC6B0020506900207C600020425E002017
:10F5E800713DAA3F005E0020E46E00200851002013
:10F5F800BC8300200000000093ED027A93ED012AFD
:10F60800D3ED037A5FED053A26EE877AA6EE027A05
:10F61800A5EEA77A27EE057AB4EEE37AF1EE10FAB2
:10F62800B4BFF0EE637AF0EE477A8DED0C7A88BFBE
:10F63800B0EE637A012A3EF4AEAED3ED063AD3EDCE
:10F64800051A93ED072A66EEA33AE6EE213AE5EEAF
:10F65800823A63EE853AB4EEE37AF1EE10FAF4EE0C
:10F66800E37A8CBFB0EE632AB0EE472AF1EE10FAC7
:10F6780058BFB0EE427AB8BFF0EE637A022ACDEDF9
:10F688000D3A3EF488AED3ED0A3AD3ED091A93ED5C
:10F698000B2A66EEA33AE6EE213AE5EE823A63EEED
:10F6A800853AB4EEE37AF1EE10FAF4EEE37A8CBF21
:10F6B800B0EE632AB0EE472AF1EE10FA58BFB0EE6A
:10F6C800427AB8BFF0EE637A032ACDED0E3A3EF4E3
:10F6D80062AED3ED0E3AD3ED0D1A93ED0F2A66EE16
:10F6E800A33AE6EE213AE5EE823A63EE853AB4EEC5
:10F6F800E37AF1EE10FAF4EEE37A8CBFB0EE632A07
:10F70800B0EE472AF1EE10FA58BFB0EE427AB8BF11
:10F71800F0EE637A042ACDED0F3A3EF43CAED3ED19
:10F72800123AD3ED111A93ED132A66EEA33AE6EED8
:10F73800213AE5EE823A63EE853AB4EEE37AF1EEE9
:10F7480010FAF4EEE37A8CBFB0EE632AB0EE472AE3
:10F75800F1EE10FA58BFB0EE427AB8BFF0EE637A15
:10F76800052ACDED103A3EF416AED3ED163AD3ED98
:10F77800151A93ED172A66EEA33AE6EE213AE5EE5E
:10F78800823A63EE853AB4EEE37AF1EE10FAF4EEDB
:10F79800E37A8CBFB0EE632AB0EE472AF1EE10FA96
:10F7A80058BFB0EE427AB8BFF0EE637A062ACDEDC4
:10F7B800113A3EF4F0ADD3ED1A3AD3ED191A93EDA0
:10F7C8001B2A66EEA33AE6EE213AE5EE823A63EEAC
:10F7D800853AB4EEE37AF1EE10FAF4EEE37A8CBFF0
:10F7E800B0EE632AB0EE472AF1EE10FA58BFB0EE39
:10F7F800427AB8BFF0EE637A072ACDED123A3EF4AA
:10F80800CAADD3ED1E3AD3ED1D1A93ED1F2A66EE4D
:10F81800A33AE6EE213AE5EE823A63EE853AB4EE93
:10F82800E37AF1EE10FAF4EEE37A8CBFB0EE632AD5
:10F83800B0EE472AF1EE10FA58BFB0EE427AB8BFE0
:10F84800F0EE637A082ACDED133A3EF4A4ADD3ED79
:10F85800223AD3ED211A93ED232A66EEA33AE6EE77
:10F86800213AE5EE823A63EE853AB4EEE37AF1EEB8
:10F8780010FAF4EEE37A8CBFB0EE632AB0EE472AB2
:10F88800F1EE10FA58BFB0EE427AB8BFF0EE637AE4
:10F89800092ACDED143A3EF47EADD3ED263AD3EDE8
:10F8A800251A93ED272A66EEA33AE6EE213AE5EE0D
:10F8B800823A63EE853AB4EEE37AF1EE10FAF4EEAA
:10F8C800E37A8CBFB0EE632AB0EE472AF1EE10FA65
:10F8D80058BFB0EE427AB8BFF0EE637A0A2ACDED8F
:10F8E800153A3EF458AD93ED2A2AD3ED291AD3EDF3
:10F8F8002B3A26EE822AA6EE212AA5EEA32A22EE8C
:10F90800052AB4EEC27AF1EE10FAF4EEC27A8CBF90
:10F91800F0EE423AF0EE473AF1EE10FA8DED162A83
:10F9280058BFB0EE637AA8BFB0EE672A0B2A02F080
:10F938003883D3ED2E7AD3ED2D1AD3ED2F3A66EE18
:10F94800A77AE6EE217AE3EEA57A67EE857AF4EEF9
:10F95800C77AF1EE10FAF4EEC27A8CBFF0EE476A7D
:10F96800F0EE676AF1EE10FACDED177A98BFB0EEB7
:10F97800667AB8BFF0EE427AFEF70DBD904A04925F
:10F988000025904E904FDDF81080CDF80490A946E0
:10F99800B6EC018AD4ED087AB8EEC88A28EE278A30
:10F9A800B9F1000F02F0E9837BBB9BF80030082B0C
:10F9B8003BD005F5D260B0EE480A2044D4F88C3626
:10F9C800984705F5E360D4F81437204498479BF826
:10F9D8000030032BB0EE408A22D0D4F8AC30D6F8F1
:10F9E8004406B0EE480A984708EB890309F1010973
:10F9F800B9F1030F05F12C0583ED010A3DF444AE7E
:10FA0800009B1B6803F00053C2E705F5F460B0EEF5
:10FA1800480A2044D4F89C379847B0EE408AC4E797
:10FA28001CF0E2FC27F81900D7E7B0EE480A1CF0F2
:10FA3800DBFC27F81900BCE7DFED646AFEF7DAB9EA
:10FA4800DFF8A881DAED017A9AED006AB8F80000CB
:10FA5800D8F8143077EEA77AF0EE006AB0EE677A3D
:10FA6800A6EE267A01380AEBC002D6EE267A083AC4
:10FA78001033F6EE003A27EE237A67EEA37A8AED82
:10FA8800207ACAED217ADFF868A157460AF1800189
:10FA980092ED027A92ED036AD7ED036AD7ED027A06
:10FAA80053ED014A13ED025A37EE674A76EEC65A0D
:10FAB80077EE277AE4EE845A0138A2F10802E5EEDF
:10FAC800047A07F1080703F1080336EE267A01F1F4
:10FAD8000801E4EE877AE5EE475A67EEA37A25EE49
:10FAE800A37AC1ED007A81ED017AD1D1142E07D124
:10FAF800FBF7CCFC019B344FC01A7880DAF8185118
:10FB08002F4B0493324A009B013582FB0512511991
:10FB1800EA17C2EBA1021B68C2EBC202AD1ACAF80F
:10FB2800185103F000532BE7FBF7B0FC9BF80030AB
:10FB3800079A254F801A012B78802CD0072B7DF44B
:10FB48002DAFFBF7A3FC0490FDF72ABFFBF79EFC43
:10FB5800049A1D4B801AD880FFF74DBA1D491E48DC
:10FB68001E4B91ED004AD0ED004A1D491B78CAEDA5
:10FB7800614A8AED624AD1ED006A13B101238AF81D
:10FB88009031DAED637AFEF783B9164F97ED007A74
:10FB9800FFF74EB80C4FFBF779FC134ADAF87C31C3
:10FBA80012680490C31A9A1ACAF87C01BB80FA80BA
:10FBB800FDF7F6BEFBF76AFC0790FDF782BD00BFB4
:10FBC800186900202C610020765E002000000000EB
:10FBD80093244992A42E002060570020243200204C
:10FBE80070570020405100203C3000203869002028
:10FBF80084220020E7EE267ADF48B1EE436AB0EEB1
:10FC0800647AA6EE277AF0EE477ABDEEE47A002C05
:10FC180041F09486FDEEE77A17EE104A17EE906AE7
:10FC2800FDEEC47AB44217EE901A17EE105AA8BF28
:10FC38003546B142C8BF0D4607EE905AF8EEE77A4E
:10FC4800012AC0ED007A3FF4B2A993ED047ADDED04
:10FC58000D7AE7EE267AB0EE647AA6EE277AFDEE04
:10FC6800C77A17EE906A17EE905AA642A8BF2546A3
:10FC78008E42B8BF0D4607EE905AF8EEE77A022A90
:10FC8800C0ED017A3FF493A993ED087ADDED0E7A81
:10FC9800E7EE267AB0EE647AA6EE277AFDEEC77A0A
:10FCA80017EE906A17EE905AA642A8BF25468E42D4
:10FCB800B8BF0D4607EE905AF8EEE77A032AC0ED72
:10FCC800027A3FF474A993ED0C7ADDED0F7AE7EE32
:10FCD800267AB0EE647AA7EEC37AFDEEC77A17EEFD
:10FCE800906A17EE905AA642A8BF25468E42B8BF22
:10FCF8000D4607EE905AF8EEE77A042AC0ED037A2B
:10FD08003FF455A993ED107ADDED107AE7EE267AE7
:10FD1800B0EE647AA7EEC37AFDEEC77A17EE906A62
:10FD280017EE905AA642A8BF25468E42B8BF0D4688
:10FD380007EE905AF8EEE77A052AC0ED047A3FF408
:10FD480036A993ED147ADDED117AE7EE267AB0EE56
:10FD5800647AA7EEC37AFDEEC77A17EE906A17EEBB
:10FD6800905AA642A8BF25468E42B8BF0D4607EE58
:10FD7800905AF8EEE77A062AC0ED057A3FF417A9FB
:10FD880093ED187ADDED127AE7EE267AB0EE647A12
:10FD9800A7EEC37AFDEEC77A17EE906A17EE905A6F
:10FDA800A642A8BF25468E42B8BF0D4607EE905A18
:10FDB800F8EEE77A072AC0ED067A3FF4F8A893ED43
:10FDC8001C7ADDED137AE6EE877A2546B0EE647A82
:10FDD800A6EE277AFDEEC77A17EE906AB442A8BF5E
:10FDE8003546B142C8BF0D4607EE905AF8EEE77A9D
:10FDF800082AC0ED077A3FF4DAA893ED207ADDED02
:10FE0800147AE6EE877A2546B0EE647AA6EE277A6B
:10FE1800FDEEC77A17EE906AB442A8BF3546B142E4
:10FE2800C8BF0D4607EE905AF8EEE77A092AC0EDEA
:10FE3800087A3FF4BCA893ED247ADDED157AE6EE56
:10FE4800877A2546B0EE647AA6EE277AFDEEC77A61
:10FE580017EE906AB442A8BF3546B142C8BF0D46F6
:10FE680007EE905AF8EEE77A0A2AC0ED097A3FF4CD
:10FE78009EA893ED287ADDED167AE7EE267A2546D8
:10FE8800B0EE647AA7EEC37AFDEEC77A17EE906AF1
:10FE9800B442A8BF3546B142C8BF0D46FFF767B8A0
:10FEA800FDEEC47A0CA817EE906AFDEEE47A00EB3A
:10FEB800820317EE907AFDEEE57ADFF8C090DFF85E
:10FEC800B8E0089217EE905AB1EE436A84F0010840
:10FED8004FFA84FC1946CDF824A04B4693ED007ADE
:10FEE800F0EC017AE7EE267A04F0010309F1100933
:10FEF800B0EE647AA6EE277AB4EEC74AF1EE10FAAD
:10FF0800D8BF0023002BF0EE477A18BFB0EE657A11
:10FF1800BDEEC77AFDEEE77A17EE102A17EE90AA23
:10FF2800BA4217EE103AA8BF3B469542CCBF002212
:10FF380004F00102002A08BF2B46574507EE103A85
:10FF48003A46A8BF52465645CCBF002308F00103E5
:10FF5800002B08BF324607EE902AB8EEC77AF8EEB3
:10FF6800E77ABCF1000F18BFF0EE477A8842EEEC52
:10FF7800017AB2D1FEF7AEBD502E0020985600206F
:10FF8800B84BB5F908101A6802B111609B69B5F948
:10FF98000A2003B11A60009B1B689A0601F1A38628
:10FFA80002220592FFF7C6BA9AF8BC31012B01F07C
:10FFB8002087AD4B96F916005A8896F90AE01B88F7
:10FFC800AA4910FB03F31EFB02F281FB020C81FB22
:10FFD8000301D217DB17C2EB2C12C3EB21133A44EF
:10FFE8001C442A806C80FEF73FBCDFF8A082A04842
:08FFF800D8F80820B8F80C103D
:020000040801F1
:100000001BF072FA9BF80060142E02F05680DAF8AA
:1000100018510135CAF8185118E5DFF87882B8F898
:100020000060D8F804E04FEA560C4FEA8C020AEB65
:100030008607F6080AEB020300F09F8010320136B3
:100040008E4803EB06163A4410330EF1100507F103
:10005000100151ED032A51ED043A10ED043A10ED70
:10006000032A51ED026A11ED016A10ED020A10ED4A
:10007000018A12ED044A12ED035A53ED044A53ED7E
:10008000035A13ED027A53ED017A52ED020A12ED92
:10009000011A73EE238A72EE221A40ED048A40EDB3
:1000A000031A70EE268A78EE061A40ED028A40EDB9
:1000B000011A74EE848A75EE851A43ED048A43EDC5
:1000C000031A77EE208A77EE811A43ED028A43ED18
:1000D000011A73EE633A75EE655A15ED035A32EE66
:1000E000623A74EE644A65EE631A15ED044A23EE33
:1000F000052A64EE652AE3EE041A1033B34224EEB7
:10010000843AA3EE842A00F1100005F11005A5EE53
:10011000853A01F1100102F11002E4EE852A41ED69
:10012000071A01ED082A02ED073A42ED082A55EDBB
:10013000055A15ED065A70EE666A38EE466A30EEDC
:10014000C77A71EE677A26EE253A65EEE63A25EE35
:10015000674A67EE054AE6EE053AA6EE853AA7EE4F
:10016000254AE7EEA54A01ED063A41ED053A02EDD2
:10017000064A42ED054A7FF46CAF1FFA8CF57246D1
:1001800029463D4815F030F92946D8F8042038466C
:1001900015F02AF99BF80030142B7FF4B3ACABE4D4
:1001A000374BDAF81CC10493BAF81481C8F1200364
:1001B000D8B2344B08EB4C1703EB8707830801F0E8
:1001C000778701331B0130492C4A029307EB030E5A
:1001D00007F1100313ED024A13ED035A13ED016A00
:1001E00013ED047A51ED024A51ED035A51ED016AC3
:1001F00051ED047A64EE244A65EE255A66EE266ACD
:1002000067EE277A1033734542ED024A42ED035AF6
:1002100042ED016A42ED047A01F1100102F110028F
:10022000D8D1029B1949A3F11002174401EB020E29
:10023000524410F0030309D0B7EC017AFEEC017AC6
:1002400067EE277A013BE2EC017AF5D1B8F1000FB5
:1002500041F05385142E7FF459ACFBF71BF9019B39
:100260000B4FDAF81851C01A78804FE4E46E002082
:100270002C5F00201F85EB51842200209422002057
:100280001869002050690020E06A0020D06A002030
:10029000765E002038690020D94B1A78DAF81CE124
:1002A000D8489FEDD97A4FEACE07C31983ED007A7B
:1002B000002A7AD0D549B0EE476AF0EE476A0023AB
:1002C000F1EC017A013367EEA77A05EE903AB4EECD
:1002D000E77AF1EE10FAF8EEE55AB8BFB0EE677AB9
:1002E000934276EEA76AA7EEA56AE9D1F5EEC06A59
:1002F000C319F1EE10FA83ED007A56DDC6EE265AE8
:10030000C34BC44A1288F7EE007A75EEE75AD3ED74
:10031000007A65EEA77AFDEEE77A17EE903A812B28
:1003200041F307839342A8BF134607EE903AF8EED5
:10033000E77AB94B2C2101FB0E3393ED097AD3ED0B
:10034000003A93ED0A6A93ED014AD3ED046AD3EDC6
:10035000034A93ED025AA3EEA77AA4EE276A66EE4B
:10036000C76AA7EE646ABDEEC77AE5EE276A17EEA4
:10037000101A812983ED096AC3ED0A6A41F3D68216
:100380008A42A8BF0A4607EE902AF8EEE77AFCEE0A
:10039000E77ACDED027ABDF80830C2199380BEF13C
:1003A000000F02D1132E01F05786152E7FF4A2AB59
:1003B00038449A4F838827F81E30994BDAF8185141
:1003C0000493FFF7A3BBDAF81C81954A8D4B049286
:1003D00003EBC803126802929DED027A9B88DFED61
:1003E000917A914AF8EE478A09EE103A643BC82B9D
:1003F000A8BFC82368EEA78AF8EE497A782BB8BF61
:10040000782368EEA78A07EE903A2C27B0EE680AA8
:1004100007FB0827B8EEE78A1CF036F8B8EEC99A51
:10042000F0EE409AB0EE680A1BF090FF38EE097AC1
:1004300079EE487A28EE098A67EE877AB7EE006A85
:1004400088EE277A142EF8EE007A77EE076A60EECF
:10045000277A89EEA67A77EE065A36EE477AC6EE06
:10046000256A67EEA67A27EE267AC7ED006A87ED41
:10047000047AC7ED026AC7ED017AC7ED037A01F08D
:1004800034866A4B9BF8006008F1010883FB083C46
:10049000ACEBE87C0CEB4C0C0135A8EB0C0CCAF86F
:1004A0001851CAF81CC17FE6DFF8548198F8002083
:1004B000970801F03986DFF88CC1781C40010CEBFD
:1004C000000E0CF12003ACF1700113ED076A53ED3F
:1004D000056A13ED037A53ED017A53ED025A13EDD9
:1004E000084A53ED064A13ED045A26EE066A66EEF4
:1004F000A66A27EE077A67EEA77AA4EE046A20338D
:100500007345E4EEA46A01F11001A5EE057AE5EE6B
:10051000A57AF1EEC65AB1EEE66AF1EEC76AB1EE1F
:10052000E77A41ED085A01ED076A41ED066A01EDEF
:10053000057ACAD1203884440AEB071712F0030366
:1005400018BF0CF1080C0FD05CED017A1CED027A9B
:1005500067EEA77A013BE7EE077A0CF1080CB1EEE3
:10056000E77AA7EC017AEFD1142E01F0B0850135BE
:10057000CAF8185192E62E4A32F91340FEF771B9C3
:100580002B4A32F91370FEF761B9294B294D1A68CD
:1005900059682A609A68DB68EB606960264EAA6039
:1005A000019BFEF747B9FAF775FF9BF800600190D1
:1005B000142E05BF194FDAF81851DAF818513D809A
:1005C000FDF74FB81D4F002437F9023F00EE103AF7
:1005D000E0B2B8EEC00A013404F0CAFA082CF3D134
:1005E0000594FEF7A3BF164BB5F906101A6802B1C1
:1005F00011609B69B5F90820002B7FF4CFACCEE4E5
:1006000032690020506B002000000000842200208E
:100610003469002030690020686B0020765E00207D
:100620001869002027D4D2369468002056555555B5
:10063000BC830020402E0020E45700203E2E0020E6
:10064000E46E0020042300209A4F002437F9023B77
:1006500000EE103AE0B2B8EEC00A013404F088FAB5
:10066000042CF3D1BCE7944F002437F9023F00EE8D
:10067000103AE0B2B8EEC00A013404F079FA062C60
:10068000F3D1ADE78D4EDFF8588296ED004A96ED36
:10069000097AD6ED014A96ED0A6AD6ED046A96ED1E
:1006A000035AD6ED025A69EE277A08EB8503A7EEC6
:1006B000847AA7EEA46A66EEC76AA7EE456AE7EEFB
:1006C000A56A20EE070A86ED096AC6ED0A6A83ED7F
:1006D000007A29EE088A1BF08BFE69EE288AD6ED97
:1006E000145AD6ED1F6A96ED0B1AD6ED161A96ED32
:1006F000155A96ED207A96ED0C2AD6ED172A96ED2E
:100700000F6AD6ED1A7A96ED0E3AD6ED0D3A96EDC1
:10071000194AD6ED184AE8EE015A002208EB850383
:10072000E8EEA16A00B2CAF80421A8EE025ACAF89B
:100730000821CAF80C21A8EEA27A26EE656A67EEB7
:10074000E67AA5EEC35AA8EE236AA6EEC47AE8EECE
:10075000A47A86ED145AC3ED205A86ED156AC3EDCE
:10076000406A86ED1F7AC6ED207AFEF794BEB4F992
:100770002430E26207EE903A0122F8EEE77A23662F
:10078000E2670023012EC4ED1C7AC4ED1B7A636777
:1007900001F04F84AE427DF4EAA9B4F926306366D5
:1007A00007EE903A00220123F8EEE77A2263C4F8BC
:1007B00090300023012EC4ED217AC4ED207AC4F8D4
:1007C000883001F03284AE427DF401AAB4F92830B9
:1007D000A36607EE903A00220123F8EEE77A6263FF
:1007E000C4F8A4300023012EC4ED267AC4ED257A86
:1007F000C4F89C307DF41BAA9FED318AB8F1030F39
:1008000001F0E583009B4BB107EE903AF8EEE77AF2
:10081000F4EEC87AF1EE10FA01F18B84294AA36E46
:1008200012689AF82011F88003EB550393FBF5F555
:100830000023656393621363D36221B1224B1B884B
:10084000002B7DF4F5A9214B1B6813F4003304D071
:100850001F4B1B79002B41F061841E491A46C85C6E
:10086000012803F10C0301F02A820132152AF6D186
:10087000FDF7DEB9029B1F7807F0010CFEF79BBB6A
:10088000154BDFED167A1968CAED4C7A11F08051DC
:1008900000F07082B7EE007A77EE677AF4EEE27AD3
:1008A000F1EE10FA88BFF0EE627ACAED637AFDF7D6
:1008B000ECBD00BF462E0020422E0020EC6B002035
:1008C00000000000DC6000203A4D0020502C002089
:1008D0007C60002074F202088C2E00200000008052
:1008E00050690020002840F04E86E7EE267ADE4868
:1008F000BDEEE47A17EE105AB0EE447AA3EE277AF2
:100900002C46F0EE477AFDEEE77ABDEEE57A17EE7B
:10091000906A17EE101AB542A8BF3446B142C8BF5C
:100920000C4607EE904AF8EEE77A012AC0ED007A0D
:100930003EF441AB93ED047ADDED0D7AE7EE267AD5
:10094000B0EE447AA3EE277AFDEEC77A17EE906AEE
:1009500017EE904AAE42A8BF2C468E42B8BF0C4656
:1009600007EE904AF8EEE77A022AC0ED017A3EF4EB
:1009700022AB93ED087ADDED0E7AE7EE267AB0EE43
:10098000447AA3EE277AFDEEC77A17EE906A17EE47
:10099000904AAE42A8BF2C468E42B8BF0C4607EE26
:1009A000904AF8EEE77A032AC0ED027A3EF403ABF0
:1009B00093ED0C7ADDED0F7AE7EE267AB0EE447A0D
:1009C000A3EE277AFDEEC77A17EE906A17EE904AEB
:1009D000AE42A8BF2C468E42B8BF0C4607EE904AE6
:1009E000F8EEE77A042AC0ED037A3EF4E4AA93ED28
:1009F000107ADDED107AE7EE267AB0EE447AA3EEB7
:100A0000277AFDEEC77A17EE906A17EE904AAE424B
:100A1000A8BF2C468E42B8BF0C4607EE904AF8EEAF
:100A2000E77A052AC0ED047A3EF4C5AA93ED147A5C
:100A3000DDED117AE7EE267AB0EE447AA3EE277A5E
:100A4000FDEEC77A17EE906A17EE904AAE42A8BF45
:100A50002C468E42B8BF0C4607EE904AF8EEE77A75
:100A6000062AC0ED057A3EF4A6AA93ED187ADDEDCC
:100A7000127AE7EE267AB0EE447AA3EE277AFDEEFC
:100A8000C77A17EE906A17EE904AAE42A8BF2C467E
:100A90008E42B8BF0C4607EE904AF8EEE77A072A76
:100AA000C0ED067A3EF487AA93ED1C7ADDED137A49
:100AB000E7EE267AB0EE447AA3EE277AFDEEC77A07
:100AC00017EE906A17EE904AAE42A8BF2C468E42AF
:100AD000B8BF0C4607EE904AF8EEE77A082AC0ED58
:100AE000077A3EF468AA93ED207ADDED147AE7EEFA
:100AF000267AB0EE447AA3EE277AFDEEC77A17EE97
:100B0000906A17EE904AAE42A8BF2C468E42B8BFFC
:100B10000C4607EE904AF8EEE77A092AC0ED087A0B
:100B20003EF449AA93ED247ADDED157AE7EE267AB4
:100B3000B0EE447AA3EE277AFDEEC77A17EE906AFC
:100B400017EE904AAE42A8BF2C468E42B8BF0C4664
:100B500007EE904AF8EEE77A0A2AC0ED097A3EF4E9
:100B60002AAA93ED287ADDED167AE7EE267AB0EE22
:100B7000447AA3EE277AFDEEC77A17EE906A17EE55
:100B8000904AAE42A8BF2C468E42B8BF0C4607EE34
:100B9000904AF8EEE77A0B2AC0ED0A7A3EF40BAAE7
:100BA00093ED2C7ADDED177AE6EE877AA3EE274AED
:100BB000FDEEC47A17EE903A9D42A8BF1D469942B9
:100BC000D8BF294607EE901AF8EEE77AC0ED0B7A07
:100BD000FEF7F1B9069B002B01F03081FDEEE57ABE
:100BE0000CA917EE90EAFDEEE47A204D1E4E17EEAA
:100BF000903AFDEEC47A01EB820217EE907A14E08F
:100C0000FDEEC77A17EE908AB84503DB9845C446D7
:100C1000A8BF9C4607EE90CAF8EEE77A9142E6EC50
:100C2000017A05F110053EF4CAA995ED007AF1ECC0
:100C3000017AE7EE267ABC46B0EE447AA3EE277A34
:100C4000F0EE477A002CDBD030B1B4EE474AF1EE3B
:100C500010FAC8BFF0EE657AFDEEE77AF44617EEBB
:100C6000908AC645D2DDD5E7502E00209856002048
:100C7000069B002B01F03E81FDEEC47A0CAB17EE13
:100C8000906AFDEEE47ACF49CF4D17EE90EAFDEE83
:100C9000E57AB1EE436A17EE907A03EB820214E034
:100CA000FDEEC77A17EE90CAB44503DBF445A8BF42
:100CB000F446E04607EE908AF8EEE77A9342E5ECD8
:100CC000017A01F110013EF47AA991ED007AF3EC7A
:100CD000017AE7EE267AB046B0EE647AA6EE277A7D
:100CE000F0EE477A002CDBD0BC4630B1B4EE447A4B
:100CF000F1EE10FA48BFF0EE657AFDEEE77A17EEF6
:100D0000908AB84504DBF04517EE90CAA8BFF446B8
:100D100007EE90CAF8EEE77AD0E7AC4B196811F00D
:100D2000805127D0B6EE007A67EE877AF4EEE72A94
:100D3000F1EE10FA3FF5B9ADACE5F0EE457AFDF70E
:100D40002EBBA349A348A44B91ED004AD0ED004A25
:100D5000A2491B78CAED637ACAED614A8AED624AFC
:100D6000D1ED006A002B3DF497A801238AF8903159
:100D7000FDF792B8019B13F4800101D00021D1E767
:100D8000B6EE007AF4EEC72AF1EE10FACADCFDF7EF
:100D90007CBBFDEEE57A0CAB17EE905AFDEEE47AE3
:100DA0008849894C17EE90EA03EB8206D1ED007A70
:100DB000B3EC017AA6EEA77A1031B0EE446AA3EE46
:100DC000076A07EE905AB0EE467A30B1B4EE464A62
:100DD000F1EE10FAC8BFB0EE657ABDEEC77A17EE35
:100DE000107ABD4204DC7745A8BF774607EE907ABB
:100DF000F8EEE77AB342E4EC017AD7D1FDF7E3BC31
:100E0000012A41F3168107EE101AB8EEC77AC7EE31
:100E1000876AB1EEE68AB8F1030F01F0CA80009B41
:100E20004BB107EE903AF8EEE77AB4EEE78AF1EECE
:100E300010FA01F37E81236E03EB550393FBF5F368
:100E4000E362A7E4012A41F3F08007EE101AB8EE3E
:100E5000C77AC7EE876AB1EEE68AB8F1030F01F0F0
:100E6000AF80009B4BB107EE903AF8EEE77AB4EE14
:100E7000E78AF1EE10FA01F35C81636E03EB550330
:100E800093FBF5F323639EE4012A7FF7B5AC07EEED
:100E9000101AB8EEC77AC7EE876AB1EEE68AADE4FB
:100EA000BAF84C31DD0541F19980079A4C4B92ED2F
:100EB000017AD2ED006AD2ED027A0893BDEEC77ACC
:100EC000039AB3F90600118B17EE103AFDEEE66AAD
:100ED000FDEEE77A16EE902AADF8323017EE903A32
:100EE000ADF83020ADF834303E4A374CB2F902301C
:100EF000B2F900203C4DD4ED007A9FED3C7A3C4C99
:100F00004FF47A7603F5E16306FB03F302F5E16241
:100F100006FB02F285FB03761E44DB1785FB027598
:100F2000C3EBE62377EEC77A089E2478069415442F
:100F3000D2173446C2EBE522FDEEE77A3546A3F53B
:100F4000FA73A646AD882489ADF8483017EE903A7A
:100F5000401AA2F5FA726D1A641A3788ADF83E008D
:100F60007688ADF84A20ADF83630BEF80A20BEF8D3
:100F70000C30BEF80E00ADF83C50ADF840401D4DB1
:100F8000069C7F1A761A521A5B1A401A0021ADF895
:100F90003870ADF83A60ADF84220ADF84430ADF8A5
:100FA000460029606960A960E960002C01F0E680D4
:100FB000114FDFF84C80114E07958946CDF824A0DB
:100FC0005EE000BF98560020502E00208C2E00209E
:100FD000A42E0020605700202432002070570020EB
:100FE000BC8300202C5F0020C5B3A2910080BB44CD
:100FF00090500020402E002094500020E457002004
:101000002024002018AB03EB440030F9300CA8F882
:10101000000097F902E001230D4403FA04F4A94B00
:1010200056F825501EFB00F083FB003EC017019BC5
:101030002C42C0EB6E100CBF01244FF0FF349842DD
:101040000EDB039B02FB03F29E4B83FB0253D21782
:10105000C2EB6313A3EB0C031BB28342A8BF03468E
:10106000079830F8112003FB042320F81130069B69
:1010700009F10109994507F1070708F102084FDA5C
:10108000BB79002B35D1397897F9052003924D00B3
:10109000681806EB800097F90430C288808897F8BA
:1010A00003E07C78121A92B2864802FB03F380FBBD
:1010B00003C0DB17C3EB60134FEA520CA3EB0C0326
:1010C0001BB20193BEF1000F9CD018AB03EB440A96
:1010D000B8F900003AF930AC504513DA864470454F
:1010E00003DCF2455046A8BF704600B2A8F80000E5
:1010F0008FE71633D8B204F0D1FF0028C3D1A8F887
:101100000000B4E785DDA0EB0E0ED64503DB70458D
:10111000A8BF704682460FFA8AF0A8F8000078E768
:10112000079DDDF824A096F90A002B88654A6649D8
:1011300010FB03F3F07A097882FB0342FF284FEAA1
:10114000E373C3EB621200F04886814240F24586A9
:10115000089B33F9100096F916406B8810442880DC
:10116000584AF07D14FB03F382FB0342FF284FEA49
:10117000E373C3EB621200F02C86814240F22986B1
:10118000089B33F9100096F92240AB881044688020
:101190004C4A96F8230014FB03F382FB0342FF281A
:1011A0004FEAE373C3EB621200F00F86814240F214
:1011B0000C86089B33F9100096F92E40EB881044FA
:1011C000A880404A96F82F0014FB03F382FB0342E9
:1011D000FF284FEAE373C3EB621200F0F28581420D
:1011E00040F2EF85089B33F9100096F93A402B89BD
:1011F0001044E880334A96F83B0014FB03F382FB6B
:101200000342FF284FEAE373C3EB621200F0D58577
:10121000814240F2D285089B33F9100096F946408E
:101220006B8910442881274A96F8470014FB03F382
:1012300082FB0342FF284FEAE373C3EB621200F024
:10124000B885814240F2B585089B33F9100096F9C4
:101250005240AB89104468811A4A96F8530014FB37
:1012600003F382FB0342FF284FEAE373C3EB6212EE
:1012700000F09B85814240F29885089B33F910006D
:1012800096F95E40EB891044A8810E4A96F85F00FB
:1012900014FB03F382FB0342FF284FEAE373C3EB23
:1012A000621300F07E85884280F07B85089A32F9CF
:1012B00010200099096801911344EB810B46FDF75A
:1012C000B9BA00BF1F85EB51345F0020FDEEE77A0D
:1012D00017EE105A17EE906AFDEEE57AB54217EE5A
:1012E000901A17EE104AA8BF3446B142C8BF0C4648
:1012F00007EE904AF8EEE77A012AC0ED007A3DF455
:101300005AAE93ED047ADDED0D7AE7EE267AB0EE73
:10131000647AA6EE277AFDEEC77A17EE906A17EE8A
:10132000904AAE42A8BF2C468E42B8BF0C4607EE8C
:10133000904AF8EEE77A022AC0ED017A3DF43BAE1E
:1013400093ED087ADDED0E7AE7EE267AB0EE647A58
:10135000A6EE277AFDEEC77A17EE906A17EE904A4E
:10136000AE42A8BF2C468E42B8BF0C4607EE904A4C
:10137000F8EEE77A032AC0ED027A3DF41CAE93ED55
:101380000C7ADDED0F7AE7EE267AB0EE647AA6EEFF
:10139000277AFDEEC77A17EE906A17EE904AAE42B2
:1013A000A8BF2C468E42B8BF0C4607EE904AF8EE16
:1013B000E77A042AC0ED037A3DF4FDAD93ED107A8F
:1013C000DDED107AE7EE267AB0EE647AA6EE277AA3
:1013D000FDEEC77A17EE906A17EE904AAE42A8BFAC
:1013E0002C468E42B8BF0C4607EE904AF8EEE77ADC
:1013F000052AC0ED047A3DF4DEAD93ED147ADDEDFF
:10140000117AE7EE267AB0EE647AA6EE277AFDEE40
:10141000C77A17EE906A17EE904AAE42A8BF2C46E4
:101420008E42B8BF0C4607EE904AF8EEE77A062ADD
:10143000C0ED057A3DF4BFAD93ED187ADDED127A7B
:10144000E7EE267AB0EE647AA6EE277AFDEEC77A4A
:1014500017EE906A17EE904AAE42A8BF2C468E4215
:10146000B8BF0C4607EE904AF8EEE77A072AC0EDBF
:10147000067A3DF4A0AD93ED1C7ADDED137AE7EE2C
:10148000267AB0EE647AA6EE277AFDEEC77A17EEDA
:10149000906A17EE904AAE42A8BF2C468E42B8BF63
:1014A0000C4607EE904AF8EEE77A082AC0ED077A74
:1014B0003DF481AD93ED207ADDED147AE7EE267AE6
:1014C000B0EE647AA6EE277AFDEEC77A17EE906A40
:1014D00017EE904AAE42A8BF2C468E42B8BF0C46CB
:1014E00007EE904AF8EEE77A092AC0ED087A3DF453
:1014F00062AD93ED247ADDED157AE7EE267AB0EE53
:10150000647AA6EE277AFDEEC77A17EE906A17EE98
:10151000904AAE42A8BF2C468E42B8BF0C4607EE9A
:10152000904AF8EEE77A0A2AC0ED097A3DF443AD15
:1015300093ED287ADDED167AE7EE267AB0EE647A3E
:10154000A6EE277AFDEEC77A17EE906A17EE904A5C
:10155000AE42A8BF2C468E42B8BF0C4607EE904A5A
:10156000F8EEE77A0B2AC0ED0A7A3DF424AD93ED4C
:101570002C7ADDED177AE6EE877AE6EE274AFDEE65
:10158000E47AFFF717BBE7EE267AEC48BDEEE47A83
:1015900017EE105AB0EE447AA3EE277A2C46F0EEFE
:1015A000477AF4EEC47AF1EE10FAB8BFF0EE657A3D
:1015B000FDEEE77ABDEEE57A17EE906A17EE101AA7
:1015C000B542A8BF3446B142C8BF0C4607EE904AA8
:1015D000F8EEE77A012AC0ED007A3DF4ECAC93ED29
:1015E000047ADDED0D7AE7EE267AB0EE447AA3EECA
:1015F000277AB4EEC47AF1EE10FAF0EE477AB8BF6B
:10160000F0EE657AFDEEE77A17EE906A17EE904AF3
:10161000AE42A8BF2C468E42B8BF0C4607EE904A99
:10162000F8EEE77A022AC0ED017A3DF4C4AC93EDFE
:10163000087ADDED0E7AE7EE267AB0EE447AA3EE74
:10164000277AB4EEC47AF1EE10FAF0EE477AB8BF1A
:10165000F0EE657AFDEEE77A17EE906A17EE904AA3
:10166000AE42A8BF2C468E42B8BF0C4607EE904A49
:10167000F8EEE77A032AC0ED027A3DF49CAC93EDD4
:101680000C7ADDED0F7AE7EE267AB0EE447AA3EE1F
:10169000277AB4EEC47AF1EE10FAF0EE477AB8BFCA
:1016A000F0EE657AFDEEE77A17EE906A17EE904A53
:1016B000AE42A8BF2C468E42B8BF0C4607EE904AF9
:1016C000F8EEE77A042AC0ED037A3DF474AC93EDAA
:1016D000107ADDED107AE7EE267AB0EE447AA3EECA
:1016E000277AB4EEC47AF1EE10FAF0EE477AB8BF7A
:1016F000F0EE657AFDEEE77A17EE906A17EE904A03
:10170000AE42A8BF2C468E42B8BF0C4607EE904AA8
:10171000F8EEE77A052AC0ED047A3DF44CAC93ED7F
:10172000147ADDED117AE7EE267AB0EE447AA3EE74
:10173000277AB4EEC47AF1EE10FAF0EE477AB8BF29
:10174000F0EE657AFDEEE77A17EE906A17EE904AB2
:10175000AE42A8BF2C468E42B8BF0C4607EE904A58
:10176000F8EEE77A062AC0ED057A3DF424AC93ED55
:10177000187ADDED127AE7EE267AB0EE447AA3EE1F
:10178000277AB4EEC47AF1EE10FAF0EE477AB8BFD9
:10179000F0EE657AFDEEE77A17EE906A17EE904A62
:1017A000AE42A8BF2C468E42B8BF0C4607EE904A08
:1017B000F8EEE77A072AC0ED067A3DF4FCAB93ED2C
:1017C0001C7ADDED137AE7EE267AB0EE447AA3EECA
:1017D000277AB4EEC47AF1EE10FAF0EE477AB8BF89
:1017E000F0EE657AFDEEE77A17EE906A17EE904A12
:1017F000AE42A8BF2C468E42B8BF0C4607EE904AB8
:10180000F8EEE77A082AC0ED077A3DF4D4AB93ED01
:10181000207ADDED147AE7EE267AB0EE447AA3EE74
:10182000277AB4EEC47AF1EE10FAF0EE477AB8BF38
:10183000F0EE657AFDEEE77A17EE906A17EE904AC1
:10184000AE42A8BF2C468E42B8BF0C4607EE904A67
:10185000F8EEE77A092AC0ED087A3DF4ACAB93EDD7
:10186000247ADDED157AE7EE267AB0EE447AA3EE1F
:10187000277AB4EEC47AF1EE10FAF0EE477AB8BFE8
:10188000F0EE657AFDEEE77A17EE906A17EE904A71
:10189000AE42A8BF2C468E42B8BF0C4607EE904A17
:1018A000F8EEE77A0A2AC0ED097A3DF484AB93EDAD
:1018B000287ADDED167AE7EE267AB0EE447AA3EECA
:1018C000277AB4EEC47AF1EE10FAF0EE477AB8BF98
:1018D000F0EE657AFDEEE77A17EE906A17EE904A21
:1018E000AE42A8BF2C468E42B8BF0C4607EE904AC7
:1018F000F8EEE77A0B2AC0ED0A7A3DF45CAB93ED83
:101900002C7ADDED177AE7EE267AB0EE447AA7EE70
:10191000837AB4EEC74AF0EE477AF1EE10FAC8BF08
:10192000F0EE657AFDEEE77AFFF744B98223FEF721
:1019300034BDDFED037AFEF7FCBC00BF502E002063
:1019400000000243B4EEE74AF1EE10FAC8BFF0EE31
:10195000657AFDEEE77A17EE105A17EE906AFDEE03
:10196000E57AAE4217EE901A3446A8BF2C46B14233
:10197000C8BF0C4607EE904AF8EEE77A012AC0EDA0
:10198000007A3DF418AB93ED047ADDED0D7AE7EEC5
:10199000267AB0EE647AA7EEC37AB4EEC47AF1EE9A
:1019A00010FAF0EE477AB8BFF0EE657AFDEEE77A0E
:1019B00017EE906A17EE904AAE42A8BF2C46B1428D
:1019C000C8BF0C4607EE904AF8EEE77A022AC0ED4F
:1019D000017A3DF4F0AA93ED087ADDED0E7AE7EE98
:1019E000267A2C46B0EE647AA7EEC37AB4EEC47AB7
:1019F000F1EE10FAF0EE477AB8BFF0EE657AFDEE40
:101A0000E77A17EE906AB542A8BF3446B142C8BF24
:101A10000C4607EE904AF8EEE77A032AC0ED027A08
:101A20003DF4C9AA93ED0C7ADDED0F7AE7EE267A44
:101A3000B0EE647AA6EE277AB4EEC47AF1EE10FA2C
:101A4000F0EE477AB8BFF0EE657AFDEEE77A17EE72
:101A5000906A17EE904AAE42A8BF2C468E42B8BF9D
:101A60000C4607EE904AF8EEE77A042AC0ED037AB6
:101A70003DF4A1AA93ED107ADDED107AE7EE267A17
:101A8000B0EE647AA6EE277AB4EEC47AF1EE10FADC
:101A9000F0EE477AB8BFF0EE657AFDEEE77A17EE22
:101AA000906A17EE904AAE42A8BF2C46B142C8BF1A
:101AB0000C4607EE904AF8EEE77A052AC0ED047A64
:101AC0003DF479AA93ED147ADDED117AE7EE267AEA
:101AD0002C46B0EE647AA6EE277AB4EEC74AF1EE51
:101AE00010FAF0EE477AC8BFF0EE657AFDEEE77ABD
:101AF00017EE906AB542A8BF3446B142C8BF0C4643
:101B000007EE904AF8EEE77A062AC0ED057A3DF432
:101B100052AA93ED187ADDED127AE6EE877A2C461A
:101B2000B0EE647AA6EE277AB4EEC74AF1EE10FA68
:101B3000F0EE477AC8BFF0EE657AFDEEE77A17EE71
:101B4000906AB542A8BF3446B142C8BF0C4607EE02
:101B5000904AF8EEE77A072AC0ED067A3DF42BAA00
:101B600093ED1C7ADDED137AE6EE877A2C46B0EE23
:101B7000647AA6EE277AB4EEC74AF1EE10FAF0EED8
:101B8000477AC8BFF0EE657AFDEEE77A17EE906A05
:101B9000B542A8BF3446B142C8BF0C4607EE904AD2
:101BA000F8EEE77A082AC0ED077A3DF404AA93ED2F
:101BB000207ADDED147AE6EE877A2C46B0EE647A70
:101BC000A6EE277AB4EEC74AF1EE10FAF0EE477AA5
:101BD000C8BFF0EE657AFDEEE77A17EE906AB5427F
:101BE000A8BF3446B142C8BF0C4607EE904AF8EE93
:101BF000E77A092AC0ED087A3DF4DDA993ED247A4D
